:020000040001F9
:10000000B869022099020100A5CB0100D586010044
:10001000E3C90100E5350100C94D02000000000000
:10002000000000000000000000000000BD270200EA
:100030006D5401000000000039080200353602004E
:10004000C5960100D5960100E5960100F5960100E0
:1000500005970100159701002597010035970100CC
:1000600045970100559701006597010075970100BC
:100070008597010095970100A5970100B5970100AC
:10008000C5970100D5970100E5970100F59701009C
:100090000598010015980100259801003598010088
:1000A0004598010055980100659801007598010078
:1000B0008598010095980100A5980100B598010068
:1000C000C5980100D9980100ED980100019901003F
:1000D00015990100299901003D99010051990100EC
:1000E00065990100799901008D990100A19901009C
:1000F000B5990100C9990100DD990100F19901004C
:10010000059A0100199A01002D9A0100419A0100F7
:10011000559A0100699A01007D9A0100919A0100A7
:10012000A59A0100B99A0100CD9A0100E19A010057
:10013000F59A0100099B01001D9B0100319B010004
:10014000459B0100599B01006D9B0100819B0100B3
:10015000959B0100A99B0100BD9B0100D19B010063
:10016000E59B0100F99B01000D9C0100219C010011
:10017000359C0100499C01005D9C0100719C0100BF
:10018000859C0100999C0100AD9C0100C19C01006F
:10019000D59C0100E99C0100FD9C0100119D01001E
:1001A000259D0100399D01004D9D0100619D0100CB
:1001B000759D0100899D01009D9D0100B19D01007B
:1001C000C59D0100D99D0100ED9D0100019E01002A
:1001D000159E0100299E01003D9E0100519E0100D7
:1001E000659E0100799E01008D9E0100A19E010087
:1001F000B59E0100C99E0100DD9E0100F19E010037
:10020000059F0100199F01002D9F0100419F0100E2
:10021000559F0100699F01007D9F0100919F010092
:10022000A59F0100B99F0100CD9F0100E19F010042
:10023000F59F010009A001001DA0010031A00100EF
:10024000DB020100DB020100DB020100DB02010036
:10025000DB020100DB020100DB020100DB02010026
:10026000DB020100DB020100DB020100DB02010016
:10027000DB020100DB020100DB020100DB02010006
:10028000DFF810D000F004FC00480047759C020025
:10029000AFF30080B869022010484FF07701016089
:1002A0000F484FF0770101600E484FF4885101600C
:1002B0000A484FF07601016009484FF0760101606D
:1002C0000948804709480047FEE7FEE7FEE7FEE7EA
:1002D000FEE7FEE7FEE7FEE7FEE7FEE7040805406F
:1002E0000C08054000080540F536020081020100B7
:1002F0002DE9F05F0546002092469B46884606465B
:10030000814640241BE0284641464746224600F0ED
:1003100089FA53465A46C01A914110D311461846DD
:10032000224600F016F82D1A67EB01084F462246C8
:100330000120002100F00DF817EB00094E41201EAE
:10034000A4F10104DFDC484631462A464346BDE8B5
:10035000F09F202A04DB203A00FA02F100207047C7
:100360009140C2F1200320FA03F3194390407047F3
:10037000202A06DBCB17203A41FA02F043EAE07369
:1003800006E041FA02F3D040C2F120029140084356
:100390001946704740EA01039B0703D009E008C9EA
:1003A000121F08C0042AFAD203E011F8013B00F83A
:1003B000013B521EF9D27047D2B201E000F8012B86
:1003C000491EFBD270470022F6E710B513460A46D5
:1003D00004461946FFF7F0FF204610BD2DE9FE4FF9
:1003E000804681EA0300C00F0C46009021F00041D6
:1003F00023F00045B8EB0200A94105D24046214652
:1004000090461C460B46024623F00040104347D05E
:10041000270DC7F30A00C3F30A510290401A019056
:1004200040286BDAC3F3130040F4801B0098924617
:1004300020B10023D2EB030A63EB0B0B0198594662
:10044000C0F140025046FFF784FF06460D46504675
:100450005946019AFFF78CFF10EB08006141002418
:1004600087EA115284EAE7731A4340D0009A62B3D4
:10047000019A012A4FEA075215DC001B61EB0201C9
:100480004FF0004202EA0752CDE90042001C41F55C
:10049000801132462B4600F01BFA03B0BDE8F08F06
:1004A00040462146F9E7001B61EB0201001C41F5C3
:1004B000801300185B412018A2F5001747EB0301D9
:1004C00040EAD570B6196D4111E06D084FEA360665
:1004D00045EAC0754FEA0752001B61EB0201001CA0
:1004E00041F5801149084FEA300000195141324668
:1004F0002B4603B0BDE8F04F00F0DBB900980122B5
:1005000040000023D0EB020263EBE0730098214629
:100510004FEAE074B8EB000061EB0401E9E783F017
:1005200000435BE781F0004158E72DE9FE4F81EA87
:10053000030404F0004421F0004100944FF0000B4C
:1005400023F0004350EA01045ED052EA03045BD07A
:10055000C3F30A54C1F30A552C44A4F2F3340194B2
:10056000A0FB0254C1F3130141F48011C3F3130340
:1005700043F4801301FB024400FB034E840A970AF4
:1005800044EA815447EA8357A4FB076802958D0A21
:1005900005FB07854FEA932C04FB0C542705029DAD
:1005A0004FEA065847EA1637B5EB08056EEB070C1D
:1005B000870E920E47EA811742EA8312A7FB0201D7
:1005C000B6EB0B0164EB00042B0D43EA0C335E1811
:1005D00044EB1C50DA465146E7FB0201C5F3130415
:1005E0004FEA0B3343EA14534FEA0432019C43EAC7
:1005F0000603A4F10C040294009CCDE900B400F0C1
:1006000067F903B0BDE8F08F00200146F9E72DE956
:10061000F04D81EA030404F0004B21F0004514463C
:100620004FF0000A23F0004150EA050220D054EABE
:1006300001021DD0C5F30A570246C5F31303C1F3E7
:100640001300C1F30A5640F4801543F48013A7EB5E
:100650000608101BD64608F2FD3873EB050002D3DE
:1006600008F1010801E092185B41B8F1000F03DACC
:1006700000200146BDE8F08D00204FF480110646B1
:1006800084460EE0171B73EB050705D3121B63EBC3
:10069000050306434CEA010C49084FEA3000921862
:1006A0005B4150EA0107EDD152EA030012D082EA21
:1006B000040083EA0501084305D0101BAB4106D2B4
:1006C0000122002306E000224FF0004302E06FF019
:1006D000010253101AEB06004CEB085110EB0A0014
:1006E00041EB0B01BDE8F04D00F0E3B80EB540F270
:1006F000334102910021CDE900110A460B4600F07A
:10070000E7F803B000BDC1F30A5210B5C1F31301FD
:1007100040F2FF3341F480119A4201DA002010BD0B
:1007200040F233439A42A2F2334203DC524200F0D9
:1007300079F810BD904010BD00F0004230F000404C
:100740000AD0C10D01F56071C0F3160042EA0151F3
:10075000C20840071143704700200146704700005F
:1007600030B5041E71F1000404DB4FF00044404238
:1007700064EB0101141E73F1000405DB1C464FF00D
:100780000043524263EB04038B4208BF824230BDF8
:1007900030B5041E71F1000404DB4FF00044404208
:1007A00064EB0101141E73F1000405DB1C464FF0DD
:1007B0000043524263EB0403994208BF904230BDAC
:1007C00001F0004330B421F0004150EA010206D0AC
:1007D0000A0DA2F56072C1F31301002A02DC30BCDD
:1007E00000207047440F44EAC104C100E01830BC47
:1007F00000EBC25000F026B830B50B460146002091
:100800002022012409E021FA02F59D4205D303FAD2
:1008100002F5491B04FA02F52844151EA2F1010253
:10082000F1DC30BD202A04DB203A21FA02F000215D
:10083000704721FA02F3D040C2F1200291400843F0
:10084000194670470029A8BF7047401C490008BFDF
:1008500020F00100704710B4B0FA80FC00FA0CF0F0
:1008600050EA010404BF10BC704749B1CCF1200428
:1008700021FA04F411FA0CF118BF012121430843B5
:10088000A3EB0C01CB1D4FEA00614FEA102042BFE1
:10089000002010BC704700EBC35010440029A4BFD7
:1008A00010BC7047401C490008BF20F0010010BC7C
:1008B000704710B5141E73F1000408DA401C41F1B2
:1008C000000192185B411A4301D120F0010010BDD4
:1008D0002DE9F04D92469B4611B1B1FA81F202E04A
:1008E000B0FA80F220329046FFF733FD04460F46FF
:1008F00040EA0A0041EA0B0153465A46084313D026
:10090000114653EA010019D0C8F140025046FFF7E2
:1009100089FF05460E46504659464246FFF719FDE7
:10092000084305D0012004E020463946BDE8F08D9B
:100930000020054346EAE0762C4337430A986305D6
:10094000E40AA0EB08000022FD0A44EA47540A30FA
:1009500002D500200146E9E7010510196941DDE9EA
:10096000084500196941BDE8F04DA2E770B521F0D6
:10097000004303430CD0C1F30A550024D5EB040512
:1009800064EB0403D617AD1AB34102DB0020014625
:1009900070BD201841EB025170BD2DE9F04D0023D0
:1009A0001A461B1A8A4103DB00200146BDE8F08D80
:1009B000C1F30A52C1F3130141F480154FF0000B4B
:1009C000D10702D100186D41521E0027044640F2A3
:1009D000FF11384601EB620A3E468046024600207F
:1009E0004FF48011FFF71EFFC2197141BB1846EB8F
:1009F0000100B4EB030C75EB000C04D3E41A65EBB7
:100A0000000517460E46241908F101006D41804685
:100A10003428E3DDF91946EB0600091BA84103D28F
:100A20004FF0FF32134601E0002213461BEB070094
:100A300046EB0A51BDE8F04DFFF73BBF0EB5C10FC5
:100A400080EAE0700844CA07002140F233438DE891
:100A50000E000A460B46FFF73BFF03B000BDC1F393
:100A60000A52C1F3130140F2FF3341F480119A425C
:100A700002DA00200146704740F233439A42A2F264
:100A8000334202DC5242FFF7CDBEFFF762BC0000EA
:100A9000064C074D06E0E06840F0010394E80700CB
:100AA00098471034AC42F6D3FFF7EEFBDC8F03001F
:100AB0000C90030070B58C1810F8015B15F007035B
:100AC00001D110F8013B2A1106D110F8012B03E0E7
:100AD00010F8016B01F8016B5B1EF9D12B0705D4EF
:100AE0000023521E0DD401F8013BFAE710F8013B38
:100AF000CB1A921C03E013F8015B01F8015B521E54
:100B0000F9D5A142D8D3002070BD48F25B0CC1F6E4
:100B1000FF7C604748F2390CC1F6FF7C604748F221
:100B2000010CC1F6FF7C604748F2A51CC1F6FF7CB2
:100B30006047000070B504460D460420002C43D0E9
:100B4000002D41D0297901293ED8204EB44207D04A
:100B50001F48844204D040F25A211EA004F038FC01
:100B6000B44214D12868C0F31000297939B1218A20
:100B700001432182618A41EA104161820FE0A1892B
:100B80000143A181E18941EA1041E18107E0288820
:100B9000C0F30800297931B1218A01432182002163
:100BA000002220340EE0A1890143A181F7E7C307A9
:100BB00005D01346AE68521CD2B2F35C63544008B1
:100BC000491CC9B20028F2D170BD000000000440E9
:100BD000000404402E2E5C2E2E5C2E2E5C2E2E5CED
:100BE0002E2E5C6472697665725C7372635C6863F6
:100BF0003332663436305F6164632E630000000078
:100C000070B504460D460420002C1ED00F4EB44291
:100C100007D00F48844204D040F221310DA004F0E7
:100C2000D7FBB44202D1C5F3100001E0C5F30800C0
:100C30004FEA1041A28A42EA0002A28203D1E08A6E
:100C400040EA0100E0824FF0000070BD0000044067
:100C5000000404402E2E5C2E2E5C2E2E5C2E2E5C6C
:100C60002E2E5C6472697665725C7372635C686375
:100C70003332663436305F6164632E6300000000F7
:100C800070B504460D46002C10D00948844207D0A8
:100C90000848844204D040F2F24107A004F098FBD7
:100CA00014F8460F0121A9408843207070BD000050
:100CB00000000440000404402E2E5C2E2E5C2E2EDC
:100CC0005C2E2E5C2E2E5C6472697665725C73728B
:100CD000635C68633332663436305F6164632E630D
:100CE0000000000010B500F0D3FB00F07FFB00F027
:100CF00053FCBDE8104004F0BDBB000070B50446D5
:100D00000D460420002C18D00C48844207D00C4813
:100D1000844204D040F2FE210AA004F059FB3DB108
:100D2000681E062804D940F2FF2106A004F050FBFB
:100D3000608865F30A206080002070BD00000440D8
:100D4000000404402E2E5C2E2E5C2E2E5C2E2E5C7B
:100D50002E2E5C6472697665725C7372635C686384
:100D60003332663436305F6164632E630000000006
:100D700070B504460D46002C07D0601E0D2804D91E
:100D800040F22A410AA004F023FB012D05D025B131
:100D900040F22B4106A004F01BFB1048018864F3CD
:100DA00003010180818965F30001818170BD00002C
:100DB0002E2E5C2E2E5C2E2E5C2E2E5C2E2E5C6437
:100DC00072697665725C7372635C68633332663431
:100DD00036305F6164632E6300000000C20004408F
:100DE00010B502220021064804F020F8054C2046E8
:100DF00000F07CFA2046BDE810400021FFF740BF1C
:100E0000003005400000044070B504460D46042043
:100E1000002C1AD00D4EB44207D00D48844204D0A5
:100E200040F2A7210BA004F0D3FA280CA189A94312
:100E3000A181218AA9432182B44205D1E18981435C
:100E4000E181618A81436182002070BD000004401D
:100E5000000404402E2E5C2E2E5C2E2E5C2E2E5C6A
:100E60002E2E5C6472697665725C7372635C686373
:100E70003332663436305F6164632E6300000000F5
:100E80002DE9F0470546884617461C46042005F123
:100E90005006002D2AD0002F28D0002C26D0DFF8B5
:100EA00050904D4507D01348854204D040F2AB51D5
:100EB00011A004F08DFA4D4502D1C8F3100001E0F5
:100EC000C8F30800002100230CE0C20707D036F861
:100ED000112027F813205B1CDBB2641EE4B240082B
:100EE000491CC9B208B1002CEFD10020BDE8F08741
:100EF00000000440000404402E2E5C2E2E5C2E2E9A
:100F00005C2E2E5C2E2E5C6472697665725C737248
:100F1000635C68633332663436305F6164632E63CA
:100F20000000000070B504460E46002509488442C2
:100F300007D00948844204D040F2D64107A004F00B
:100F400047FA94F846000121B140084200D001253B
:100F5000284670BD00000440000404402E2E5C2E84
:100F60002E5C2E2E5C2E2E5C2E2E5C6472697665B5
:100F7000725C7372635C68633332663436305F610F
:100F800064632E630000000070B504460D46042023
:100F9000002C56D0002D54D02A48844206D02A482E
:100FA000844203D0F82129A004F012FA28780228FC
:100FB00006D0012804D018B1F92124A004F008FAC1
:100FC000687828B1012803D0FA2120A004F000FAA3
:100FD000A878012804D018B1FB211CA004F0F8F96E
:100FE000E87848B1012807D0022805D0032803D0AB
:100FF000FC2116A004F0ECF9287928B1012803D0CF
:10100000FD2112A004F0E4F9002020702A78618804
:1010100062F3051161806A78618862F3C7116180AB
:10102000AA78618862F386116180EA78618862F348
:10103000010161802A79A18862F38201A18084F88C
:10104000470070BD00000440000404402E2E5C2EBA
:101050002E5C2E2E5C2E2E5C2E2E5C6472697665C4
:10106000725C7372635C68633332663436305F611E
:1010700064632E630000000010B50446002C06D007
:10108000012C04D040F23C4109A004F0A1F913481E
:10109000012C05D030F8C01F21F00F01018010BDD8
:1010A00030F8C01F21F00F010E31018010BD00008B
:1010B0002E2E5C2E2E5C2E2E5C2E2E5C2E2E5C6434
:1010C00072697665725C7372635C6863333266342E
:1010D00036305F6164632E6300000000000004404E
:1010E00010B50446002C17D0012C15D0022C13D0BB
:1010F000042C11D0082C0FD0102C0DD0202C0BD08C
:10110000402C09D0802C07D0B4F5807F04D040F269
:10111000574103A004F05CF90C48048010BD0000A6
:101120002E2E5C2E2E5C2E2E5C2E2E5C2E2E5C64C3
:1011300072697665725C7372635C686333326634BD
:1011400036305F6164632E6300000000CC00044011
:101150003EB5434C204600F09BF800212046FFF7A7
:10116000E1FE0028F9D006236A4640F23B112046F2
:10117000FFF786FE00212046FFF782FDBDF80A003A
:101180009FED381A00EE100A384CF8EE400A81EE56
:10119000200ADFED350A20EE200A84ED000ABDF8B2
:1011A000060001EE100AF8EE411A81EEA01A21EEB7
:1011B000001A84ED031ABDF8080001EE100AF8EEDB
:1011C000411A81EEA01A21EE000A84ED020ABDF850
:1011D000000000EE100AB8EE400A84ED040ABDF8E3
:1011E000020000EE100AB8EE400A84ED050ABDF8D0
:1011F000040000EE100AB8EE400A70EEC00A00EEDD
:10120000100AB8EE401A80EE810A10EE100AFFF7BD
:1012100093FA41EC100B13F06FFF9FED151B51EC8F
:10122000100B53EC112BFFF780F99FED131B53ECC0
:10123000112BFFF7D3F841EC100B53EC102B9FED63
:10124000100B51EC100BFFF7E2F99FED0F1B53EC65
:10125000112BFFF764F9FFF7B3FA60603EBD0000A1
:1012600000040440BE9F8A3F00F07F458083FF1F3B
:101270000000006066A272400000000000F4AA4076
:101280000000000013642F410000006066127140EE
:1012900010B504460420002C0DD00748844207D026
:1012A0000648844204D040F2944105A004F090F82E
:1012B00001202070002010BD000004400004044004
:1012C0002E2E5C2E2E5C2E2E5C2E2E5C2E2E5C6422
:1012D00072697665725C7372635C6863333266341C
:1012E00036305F6164632E630000000038B5044649
:1012F000042100250095002C19D00E48844207D007
:101300000D48844204D040F2B1410CA004F060F8D2
:10131000002142F2107207E025700098401C0090F6
:10132000904201D9092102E020780128F4D0084632
:1013300038BD000000000440000404402E2E5C2E46
:101340002E5C2E2E5C2E2E5C2E2E5C6472697665D1
:10135000725C7372635C68633332663436305F612B
:1013600064632E630000000070B504460E46154607
:101370000420002C1AD0012E18D80F48844207D020
:101380000E48844204D04FF4F3710DA004F020F80D
:1013900035B1012D04D040F2E71109A004F018F88E
:1013A0002EB1608965F3CF306081002070BD608907
:1013B00065F3C7106081F8E70000044000040440B2
:1013C0002E2E5C2E2E5C2E2E5C2E2E5C2E2E5C6421
:1013D00072697665725C7372635C6863333266341B
:1013E00036305F6164632E630000000030B587B063
:1013F00022A00068039022A003C8CDE901010020CB
:101400000590042104918DF8140003A806901E4C49
:101410000222204600F05EF804A92046FFF78AFB6E
:1014200001210020FFF7A4FC0420FFF759FE012052
:10143000FFF722FE40F23B14049401A80690134DDE
:1014400002222146284600F045F804A92846FFF765
:1014500071FB04212846FFF751FC21462846FFF77F
:10146000CFFB012108020FF06BF9102002F036FDCE
:1014700001200FF09FF907B030BD000011000000FF
:1014800050505050505000000000044000040440F0
:101490001CB50024009401948DF800408DF80140A3
:1014A00001208DF80300012108460FF049F9694633
:1014B0000648FFF769FD0094012102200FF040F972
:1014C00069460348FFF760FD1CBD000000000440B2
:1014D000000404402DE9F0411746002500260B4A80
:1014E000904201D18CB20CE0CCB2042609E0E007B6
:1014F00004D0A819C0B2394600F00AF864086D1C7F
:10150000EDB2002CF3D1BDE8F081000000000440F2
:101510007CB504460D4600200121012200230093E2
:1015200001938DF800508DF80430102C2DD2DFE897
:1015300004F02D080A0C0E10121416181B1D20237F
:101540002629022122E0042120E008211EE01021AA
:101550001CE020211AE0402118E0802116E0012043
:1015600014E00120022111E002200FE002200221FC
:101570000CE00220042109E00220082106E00220FC
:10158000102103E00220202100E00022002A02D0E6
:101590006A460EF009FC7CBD70B5012148040FF0CD
:1015A0001BF80C4C002211462046FFF7DDFE0A4DC9
:1015B000002211462846FFF7D7FE002201212046CF
:1015C000FFF7D2FE2846BDE8704000220121FFF758
:1015D000CBBE000000000440000404402DE9F04FA1
:1015E0002DED048B83B0FE490A780020FD4EDFF814
:1015F000F893FE4FDFF8F883062A06D00A78042A0B
:101600000ED00A78052A0DD00DE03880A8F8000029
:1016100001223280F74A108089F80000087002E049
:10162000087000E00870502548F610440A2246234E
:1016300000211046CDE9004500F070FC142246233D
:1016400000211046CDE9004500F068FC1E2246232B
:1016500000211046CDE9004500F060FC2822462319
:1016600000211046CDE9004500F058FC3222462307
:1016700000211046CDE9004500F050FC3C224623F5
:1016800000211046CDE9004500F048FC46231A46EB
:1016900000211846CDE9004500F040FC50224623C9
:1016A00000211046CDE9004500F038FC5A224623BF
:1016B00000211046CDE9004500F030FC64224623AD
:1016C00000211046CDE9004500F028FC6E2246239B
:1016D00000211046CDE9004500F020FC7822462389
:1016E00000211046CDE9004500F018FC8222462377
:1016F00000211046CDE9004500F010FC8C22462365
:1017000000211046CDE9004500F008FC9622462352
:1017100000211046CDE9004500F000FC0A239F227D
:1017200019460020CDE9004500F0F8FB14239F2264
:1017300019460020CDE9004500F0F0FB1E239F2252
:1017400019460020CDE9004500F0E8FB28239F2240
:1017500019460020CDE9004500F0E0FB32239F222E
:1017600019460020CDE9004500F0D8FB3C239F221C
:1017700019460020CDE9004500F0D0FB4FF0FF0AEC
:10178000CDE9004A002146230122084600F0C6FBAD
:10179000CDE9004A002101239F22084600F0BEFB4C
:1017A000CDE9004A46239F2200219E2000F0B6FB8F
:1017B000CDE9004A46239F224521002000F0AEFBE0
:1017C0000C2001F0CBFB8C48008801F0CDFB4621BA
:1017D000002001F0BDFB8949894C91ED000A10EE13
:1017E000100AA04205DA022091ED000A01F0F8FA91
:1017F00004E0012091ED000A01F0F2FA81A001F06D
:1018000059F84621242001F0A3FB7F4991ED000AFD
:1018100010EE100AA04205DA022091ED000A01F054
:10182000DFFA04E0012091ED000A01F0D9FA77A077
:1018300001F040F84621482001F08AFB744991EDFF
:10184000000A10EE100AA04205DA022091ED000A0B
:1018500001F0C6FA11E091ED000A6E4A10EE100A8E
:10186000904205DA012091ED000A01F0B9FA04E096
:10187000002091ED000A01F0B3FA67A001F01AF818
:101880004621762001F064FB30880321400001F0FE
:1018900019FB62A001F00EF80024DFF884B1DFED3F
:1018A000618A9FED618A614D9FED619A614ED9E039
:1018B000401E844238D13BF81400FF2300EE100A8A
:1018C00038882A88B8EE400A60EE280A00EE100A2E
:1018D000B8EE401A80EE810A38EE400ABCEEC00A2B
:1018E00010EE100AC1B2204600F0F8FA5248FF2369
:1018F000328830F8140000EE100AB8F80000B8EE94
:10190000400A60EE090A00EE100AB8EE401A80EEB6
:10191000810A38EE400ABCEEC00A10EE100AC1B2CD
:10192000204600F0DBFA9BE004F1010922463BF877
:10193000190000EE100A3888B8EE400A60EE280A56
:1019400000EE100AB8EE401A80EE810A38EE400A26
:10195000BCEEC00A10EE101A8BB23BF8141000EE69
:10196000101AB8EE400A60EE280A00EE100AB8EE2F
:10197000401A80EE810A38EE400ABCEEC00A10EE32
:10198000100AC1B22888CDE9000A204600F0C6FA44
:101990002949DFED2A0A31F8190031F8141000EE58
:1019A000100AB8F80000B8EE400A60EE200A00EE17
:1019B000100AB8EE401A80EE810A38EE400ABCEEFA
:1019C000C00A10EE102A00EE101A93B2B8EE400AC8
:1019D00060EE090A00EE100AB8EE401A30E000008E
:1019E0006083FF1FC28EFF1FBB8EFF1FBC8EFF1FB9
:1019F000BE8EFF1FC08EFF1FAE83FF1F3483FF1FED
:101A000000002041560000003C83FF1F4100000001
:101A10004083FF1F0000C84257000000532F64009E
:101A2000786002200000704200008C42A883FF1FF3
:101A300000000C42AA83FF1FB86102200000204270
:101A400080EE810A224638EE400ABCEEC00A10EE53
:101A5000100AC1B23088CDE9000A204600F05EFAD3
:101A6000641CE4B2244800788442FFF421AF288843
:101A700001F07AFA388842F21074A04204D20021B0
:101A80007F2001F065FA03E00021782001F060FA80
:101A900038889FED1A8A00EE100A0220F8EE400AFC
:101AA00080EE880A01F09CF9AFF2A80000F002FF76
:101AB000308801F059FAB8F80000A04204D214218D
:101AC0007F2001F045FA03E01421782001F040FA6C
:101AD000B8F8000000EE100A0220F8EE400A80EE8E
:101AE000880A01F07DF9AFF2DC0003B0BDEC048B95
:101AF000BDE8F04F00F0DEBEBB8EFF1F00007A4451
:101B00001CB50021009101918DF8001001228DF883
:101B100001208DF802108DF803208DF804000221B9
:101B20008DF805108DF80600684602F01DF81CBD02
:101B30002DE9F04107468846164600240021384624
:101B400012F012FA05460121384612F00DFA012E64
:101B500006D04146384612F007FA012806D006E0C2
:101B6000012D01D0012802D1012400E00124012C23
:101B70000BD10020064942F21072096801E000BF53
:101B8000401CB1FBF2F38342F9D8BDE8F0810000BC
:101B9000B482FF1F2DE9FC4100F0FCF8102001F099
:101BA000DDF96748008801F0DFF90021084601F0FF
:101BB000CFF964A000F006FB0024DFF89881644EA2
:101BC0001927A8F56575308801F0CEF907EB0410E8
:101BD000C1B2002001F0BCF9687B844212D102211D
:101BE000002000F069F90C2001F0B8F95A4800888B
:101BF00001F0BAF959A000F05DFE6FF0010100207C
:101C000000F05AF9102001F0A9F908EB84100068DF
:101C100000F0D8FA24B1012C63D0022C70D168E016
:101C2000A87B08286CD2DFE800F00F1A25303B466D
:101C300051044BA000F0C6FA0021022000F03CF94C
:101C400048A000F0BFFA5BE049A000F0BBFA002119
:101C5000022000F031F947A000F0B4FA50E046A0AD
:101C600000F0B0FA0021022000F026F941A000F0B7
:101C7000A9FA45E041A000F0A5FA0021022000F0F9
:101C80001BF93FA000F09EFA3AE03FA000F09AFA5C
:101C90000021022000F010F939A000F093FA2FE0A3
:101CA0003AA000F08FFA0021022000F005F934A0DC
:101CB00000F088FA24E036A000F084FA0021022027
:101CC00000F0FAF82EA000F07DFA19E02AA000F04A
:101CD00079FA0021022000F0EFF829A000F072FA52
:101CE0000EE01FA000F06EFA0021E87B01F0EAF898
:101CF00006E01BA000F066FA0021287C01F0E2F863
:101D0000641CE4B2032CFFF45EAFFF243088CDE9FD
:101D100000049E224F230021104600F0FFF8308877
:101D2000CDE90004687B9F22C0EBC00101EB4013AA
:101D30005B1C00219D2000F0F1F8BDE8FC81000053
:101D4000AC83FF1FB1B3B9E2C9E8D6C300000000FD
:101D5000AA83FF1F4487FF1FA883FF1F3E000000C8
:101D60003A000000B1A3B3D6BFAAC6F40000000039
:101D70003A313500C3EB00003A3330003A3100000D
:101D8000B7D6D6D3000000003A3200003A35000042
:101D90003A3130002DE9F041434D2F78434C002675
:101DA000042FA17B227C637BE07B12D02F780A2F4B
:101DB0000FD02F78052F27D02F780B2F24D095F810
:101DC00000C03B4FBCF1060F37D02878092855D00A
:101DD0005EE023B1012B07D0022B59D10CE007297B
:101DE00056D2491CA17353E0642801D2401CE07311
:101DF000E07B08F02DFF4BE0824201D2521C22749E
:101E0000207C08F025FF43E023B1012B06D0022BF4
:101E10003ED10BE089B3491EA17339E0012801D9F5
:101E2000401EE073E07B08F013FF31E00AB1521E60
:101E30002274207C08F00CFF2AE05B1CDBB2637389
:101E4000032B25D12378C3B902236373F97038714A
:101E5000824200D92074207C787105F02BFF3879FC
:101E600008F0F6FE13480168A26B891AB1F5487FA5
:101E70000ED9012121700068A06309E013B15B1E37
:101E8000637304E0387908F0E3FE112060702E706F
:101E90002878062805D02878052802D02878042834
:101EA00000D12E70BDE8F0816083FF1FB083FF1F5B
:101EB000F86202207C83FF1F034A937818449070D5
:101EC000D0780844D07070479C83FF1F024A9070FE
:101ED000D0780844D07070479C83FF1F30B504460B
:101EE0001046A02C16D8502914D801EB81020A49BB
:101EF00001EB821535F814201AB1110A01EB022109
:101F00008AB20146962014F03BFE010201EB10203C
:101F100025F8140030BD0000D0D601202DE9F04F87
:101F20008046DDF824B016461F46B8F1A00F32D225
:101F3000502930D2A02E2ED2502F2CD2B04503D90A
:101F4000404606F0FF080646B94202D90846F9B2F3
:101F500007460D46DFF844A01BE0444615E005EBBC
:101F600085000AEB801939F814201AB1100A00EB29
:101F7000022082B259460A9814F002FE010201EBD7
:101F8000102029F81400641CE4B2B442E7D96D1C97
:101F9000EDB2BD42E1D9BDE8F08F0000D0D60120FE
:101FA0002DE9FF4F92B0DDE91F96219F484400F0D4
:101FB000FF0A01EB0900C0B21390C9F1000002EB67
:101FC0004001CAB2149203EB4001C9B200244D464D
:101FD000032202EB4008149A0AEB020005901398C2
:101FE0000844049099E01398AAEB040B401B11904D
:101FF0000BF0FF01C0B23B463246FFF76FFFAAEB82
:102000000500C1B2109013983B46001B0F90C0B260
:102010003246FFF763FF0498C0B2039003980BF0B9
:10202000FF0128440E900D90C0B23B463246FFF7A8
:1020300055FF10983B46C1B20398324620440C909D
:102040000B90C0B2FFF74AFF0598C0B20290029809
:102050003B4620440A90C1B209900E983246C0B265
:10206000FFF73CFF02983B462844C1B208900C9809
:102070003246C0B2FFF732FF0A980790C1B21198FA
:102080003B46C0B23246FFF729FF08980690C1B21E
:102090000F983B46C0B23246FFF720FF1198CDE9BA
:1020A000006783B2079882B21198C1B20BF0FF00AB
:1020B000FFF734FFCDE900670F9883B2069882B22C
:1020C0000F98C1B21098C0B2FFF728FF0D98CDE964
:1020D000006783B2099882B20D98C1B20BF0FF007D
:1020E000FFF71CFFCDE900670B9883B2069882B218
:1020F0000B98C1B21098C0B2FFF710FF641CB8F182
:10210000000F04DA08EB840808F1060805E0601BFC
:1021100008EB800808F10A086D1EAC427FF763AF38
:10212000AAEB0904CDE90067A2B2E0B2049B1399BF
:10213000FFF7F4FECDE9006714980AEB09010A18CD
:10214000D0B2049B1399FFF7E9FE1398CDE900671D
:10215000A0EB090083B2C1B25046059AFFF7DEFE3C
:102160000498CDE9006700EB0903D9B25046059AFF
:10217000FFF7D4FECDE90067DDE9043000EB09028A
:10218000641CE0B21399FFF7C9FE16B0BDE8F08FEA
:1021900010B50021020A02EB0020094C82B2002097
:1021A00001EB810304EB831323F81020401C80B261
:1021B000A028F9D3491C89B25029F0D310BD0000E2
:1021C000D0D601202DE9FE4F07460024DFF8B48366
:1021D000D1E17E297ED98C23787800EB012081B271
:1021E0000020E94A13E032F830608E420DD802EB4D
:1021F000C00676888E4208D332F8303002EBC00039
:10220000C91A8088084485B203E0401C80B2984215
:10221000E9D3BF1CDD48DE4A30F835109078C1F1B3
:10222000A003834202DA4FF0A00A02E0084400F063
:10223000FF0A92F80390B9F1400F02D950200090A4
:102240003BE009F11000C0B2009036E0D04886783B
:102250001EE009EB890008EB801B3BF816201AB141
:10226000100A00EB022082B2C848CA4900EBC50040
:1022700021444068405CC649C98814F081FC0102D1
:1022800001EB10202BF81600641CA4B2761CF6B2E9
:102290005645DED3BAF1A00F0BD1BC4830F835005B
:1022A000B4FBF0F100FB1141C9B211B12044401A56
:1022B00084B209F1010909F0FF0900988145C5D3ED
:1022C0000024B24810F83510B1488278114481706A
:1022D00051E1FFE7AE4A5078102807D01C2875D08E
:1022E0000C2872D109260020AB4BF0E0112600200B
:1022F000AA4B14E033F830C061450ED303EBC00C99
:10230000BCF802C0614508D833F8305003EBC00078
:10231000491B8088084485B203E0401C80B2B0426B
:10232000E8D37F1C9D489178883030F83500C0F1A3
:10233000A0038B4202DA4FF0A00A02E0084400F04A
:10234000FF0A92F80390B9F1420F02D95020009091
:102350002DE009F10E00C0B2009028E08C4886788C
:102360001FE009EB890008EB801B3BF816201AB12F
:10237000100A00EB022082B288488949883000EBBD
:10238000C50021444068405C8149C98814F0F8FBCD
:10239000010201EB10202BF81600641CA4B2761C7D
:1023A000F6B25645DDD309F1010909F0FF0900989D
:1023B0008145D3D300247948883010F8351074480B
:1023C000827811448170D6E000E0D8E00426002035
:1023D000744B14E033F830C061450ED303EBC00CEE
:1023E000BCF802C0614508D833F8305003EBC00098
:1023F000491B8088084485B203E0401C80B2B0428B
:10240000E8D37F1C6748203030F835109078C1F150
:10241000A003834202DA4FF0A00A02E0084400F071
:10242000FF0A92F80390B9F1370F02D94FF0500B21
:102430002CE009F1190000F0FF0B27E054488678E2
:10244000584909EB8900203101EBC50108EB8010E8
:10245000CDE9010114E002984168524890302044CF
:10246000085C4B490A89C98814F08AFB010201EB18
:102470001020019921F81600641CA4B2761CF6B253
:102480005645E8D309F1010909F0FF09D945D5D32B
:1024900000244448203010F835103D48827811441B
:1024A000817068E033F830C061450ED303EBC00C97
:1024B000BCF802C0614508D833F8305003EBC000C7
:1024C000491B8088084485B203E0401C80B2B042BA
:1024D000E8D37F1C30489178483030F83500C0F19F
:1024E000A0038B4202DA4FF0A00A02E0084400F099
:1024F000FF0A92F80390B9F1450F02D950200090DD
:102500002AE009F10B00C0B2009025E0204886784F
:102510001CE009EB890008EB801B3BF8160088B92A
:102520001D482149483000EBC50021444068405C0B
:1025300017490A89C98814F023FB010201EB102016
:102540002BF81600641CA4B2761CF6B25645E0D3F4
:1025500009F1010909F0FF0900988145D6D300244B
:102560000D480B49483010F835008A781044C0B245
:1025700088709F2803D8397800297FF42AAEBDE8F7
:10258000FE8F0000D0D60120C0DC020020E1020056
:102590009C83FF1F88E502007846030038B80200DC
:1025A000D8BA02003CA30200F84803000EB509297E
:1025B0003BD2DFE801F0050B11171D23292F350051
:1025C00002461CA1684612F00BFD2EE002461AA13D
:1025D000684612F005FD28E0024619A1684612F08F
:1025E000FFFC22E0024618A1684612F0F9FC1CE04C
:1025F000024617A1684612F0F3FC16E0024616A147
:10260000684612F0EDFC10E0024615A1684612F093
:10261000E7FC0AE0024614A1684612F0E1FC04E07F
:10262000024613A1684612F0DBFC684600F042F94E
:102630000EBD000025580000253031580000000074
:1026400025303258000000002530335800000000CB
:1026500025303458000000002530355800000000B7
:1026600025303658000000002530375800000000A3
:1026700025303858000000002DE9FF4F07468846F6
:10268000002403E138787E287ED98C2317F8011CBA
:1026900001EB002080B200227F4913E031F8326064
:1026A00086420DD801EBC2067688864208D331F8FF
:1026B000323001EBC201C01A8988084485B203E0B8
:1026C000521C92B29A42E9D3BF1E7448744A30F841
:1026D00035109078C1F1A003834202DA4FF0A00ACE
:1026E00002E0084400F0FF0A92F80390B9F1400FAD
:1026F00002D94FF0500B3AE009F1100000F0FF0B47
:1027000035E0674A96786548664900EBC500039056
:1027100009EB890001EB8010029013E003984168F7
:1027200061482044085C5E490A89C98814F028FA87
:10273000010201EB1020029921F81600641CA4B2DA
:10274000761CF6B25645E9D3BAF1A00F0BD1534827
:1027500030F83500B4FBF0F100FB1141C9B211B102
:102760002044401A84B209F1010909F0FF09D94552
:10277000C7D3002449484A4910F835008A781044E4
:102780008870A8F1020800E002E008F0FF087DE090
:1027900011230022454913E031F83260B0420DD3D5
:1027A00001EBC2067688B04208D831F8323001EB2E
:1027B000C201C01A8988084485B203E0521C92B253
:1027C0009A42E9D37F1E3948354A883030F83500BF
:1027D0009178C0F1A0038B4202DA4FF0A00A02E028
:1027E000084400F0FF0A92F80390B9F1420F02D9B1
:1027F0004FF0500B3BE009F10E0000F0FF0B36E00C
:10280000274A9678274909EB890001EB801001904F
:102810002648883000EBC500009013E0009841681E
:1028200023482044085C1E490A89C98814F0A8F985
:10283000010201EB1021019820F81610641CA4B2CB
:10284000761CF6B25645E9D3BAF1A00F0BD1134866
:1028500030F83500B4FBF0F100FB1141C9B211B101
:102860002044401A84B209F1010909F0FF09D94551
:10287000C6D300240D48883010F8351008488278F7
:1028800011448170A8F1010808F0FF08B8F1000FA9
:102890007FF4F8AEBDE8FF8FC0DC020020E102004B
:1028A0009C83FF1FD0D6012088E5020038B80200C3
:1028B000D8BA02002DE9F84F06460024FE4A907867
:1028C000D178A046A02870D850296ED878E2FA486E
:1028D0004278102A0FD01C2A68D00C2A67D0422ACE
:1028E00063D18C237E297DD9727802EB01218AB2D3
:1028F0000021F24FF5E111237E291FD9727802EBF6
:1029000001218AB20021EE4F14E037F831C094451E
:102910000ED807EBC10CBCF802C0944508D337F8B9
:10292000313007EBC101D21A898811448DB203E01E
:10293000491C89B29942E8D3B61C1AE00022E04F44
:1029400014E037F832C061450ED307EBC20CBCF877
:1029500002C0614508D837F8323007EBC202C91A05
:10296000928811448DB203E0521C92B29A42E8D38D
:10297000761CD3498278883131F83510C1F1A00333
:10298000934207DA4FF0A00AC2F1A002891A01F0BF
:10299000FF0802E0114401F0FF0A90F80390B9F13A
:1029A000420F05D95021009141E00DE24CE0DFE0FB
:1029B00009F10E01C9B2009139E0BF48877821E0E2
:1029C000C04809EB890100EB811B3BF817201AB1C5
:1029D000100A00EB022082B2B948883000EBC50033
:1029E000406800E081E1B8492144405CB249C988AF
:1029F00014F0C6F8010201EB10202BF81700641C3C
:102A00007F1CFFB25745DBD3BAF1A00F0BD1AC4806
:102A1000883030F8350094FBF0F100FB1141C9B269
:102A200009B12044441A09F1010909F0FF0900988D
:102A30008145C2D30024A248883010F835109E4842
:102A4000827811448170BBE104237E291FD97278FA
:102A500002EB01218AB200219C4F14E037F831C00B
:102A600094450ED807EBC10CBCF802C0944508D3BE
:102A700037F8313007EBC101D21A898811448DB281
:102A800003E0491C89B29942E8D3B61C1AE000223F
:102A90008E4F14E037F832C061450ED307EBC20CFD
:102AA000BCF802C0614508D837F8323007EBC202E3
:102AB000C91A928811448DB203E0521C92B29A4214
:102AC000E8D3761C81498278203131F83510C1F184
:102AD000A003934207DA4FF0A00AC2F1A002891ABC
:102AE00001F0FF0802E0114401F0FF0A90F80390A2
:102AF000B9F1370F02D94FF0500B2DE009F1190150
:102B000001F0FF0B28E06C4887781FE06F486F49A1
:102B1000203000EBC500903140682144405C66499C
:102B20000A89C98814F02CF8010201EB10206549CC
:102B300009EB890201EB821121F81700AAF10100CB
:102B4000874200D14444641C7F1CFFB25745DDD34B
:102B500009F1010909F0FF09D945D4D300245B48E4
:102B6000203010F83510544882781144817027E1E4
:102B700009237E291FD9727802EB01218AB2002134
:102B8000534F14E037F831C094450ED807EBC10C11
:102B9000BCF802C0944508D337F8313007EBC101C7
:102BA000D21A898811448DB203E0491C89B2994236
:102BB000E8D3B61C1AE00022454F14E037F832C0C3
:102BC00061450ED307EBC20CBCF802C0614508D8C2
:102BD00037F8323007EBC202C91A928811448DB21D
:102BE00003E0521C92B29A42E8D3761C38498278AC
:102BF000483131F83510C1F1A003934207DA4FF0A4
:102C0000A00AC2F1A002891A01F0FF0802E01144F3
:102C100001F0FF0A90F80390B9F1450F02D94FF087
:102C2000500B2CE009F10B0101F0FF0B27E02248CB
:102C300087781EE026482749483000EBC50021442C
:102C40004068405C1C490A89C98813F099FF010259
:102C500001EB10201B4909EB890201EB821121F8DD
:102C60001700AAF10100874200D14444641C7F1C74
:102C7000FFB25745DED309F1010909F0FF09D94533
:102C8000D5D300241248483010F835100A4882780D
:102C90001144817094E037F831C094451FD807EB98
:102CA000C10CBCF802C0944519D337F8313007EB9A
:102CB000C101D21A89880FE09C83FF1FC0DC02008B
:102CC00038B80200D0D60120D8BA02003CA30200D6
:102CD00078460300F848030011448DB203E0491C14
:102CE00089B29942D7D3B61C1AE00022374F14E0BC
:102CF00037F832C061450ED307EBC20CBCF802C0F6
:102D0000614508D837F8323007EBC202C91A9288F9
:102D100011448DB203E0521C92B29A42E8D3761C61
:102D20002B49827831F83510C1F1A003934207DABC
:102D30004FF0A009C2F1A002891A01F0FF0802E0D9
:102D4000114401F0FF09C778402F02D94FF0500A13
:102D50002CE007F1100101F0FF0A27E01D4890F870
:102D600002B01FE01A481C4900EBC500214440682E
:102D7000405C18490A89C98813F002FF010201EB7F
:102D80001020164907EB870201EB821121F81B0086
:102D9000A9F10100834500D14444641C0BF1010BEF
:102DA0000BF0FF0BCB45DDD37F1CFFB25745D5D3CE
:102DB0000024074810F835100648827811448170C5
:102DC000317800297FF483ADBDE8F88FC0DC0200C4
:102DD00020E102009C83FF1F88E50200D0D601207D
:102DE0000EB5062851D2DFE800F003101D2A374443
:102DF00010EE100AFDF7A0FC41EC100B25A153ECDE
:102E0000102B684612F0ECF83FE010EE100AFDF7C8
:102E100093FC41EC100B21A153EC102B684612F0EF
:102E2000DFF832E010EE100AFDF786FC41EC100BE3
:102E30001CA153EC102B684612F0D2F825E010EEDE
:102E4000100AFDF779FC41EC100B18A153EC102B84
:102E5000684612F0C5F818E010EE100AFDF76CFC99
:102E600041EC100B13A153EC102B684612F0B8F88C
:102E70000BE010EE100AFDF75FFC41EC100B0FA108
:102E800053EC102B684612F0ABF86846FFF712FDC2
:102E90000EBD0000252E306600000000252E316694
:102EA00000000000252E326600000000252E33664B
:102EB00000000000252E346600000000252E356637
:102EC000000000000EB5062927D2DFE801F0030953
:102ED0000F151B21024613A1684612F081F81CE071
:102EE000024611A1684612F07BF816E0024610A1D6
:102EF000684612F075F810E002460FA1684612F01D
:102F00006FF80AE002460EA1684612F069F804E084
:102F100002460DA1684612F063F86846FFF7CAFC46
:102F20000EBD000025640000253031640000000063
:102F300025303264000000002530336400000000BA
:102F400025303464000000002530356400000000A6
:102F5000014A9070D17070479C83FF1F01494870EF
:102F6000704700009C83FF1F0149C8807047000024
:102F70009C83FF1F2DE9FF4F89B006468846174600
:102F8000002453E21798102812D017981C2874D0E8
:102F900017980C2872D01798422870D18C227E2B5B
:102FA0006ED9787800EB032081B20020F84BC6E19F
:102FB00011227E2B1FD9787800EB032081B20020EC
:102FC000F44B14E033F830C08C450ED803EBC00C42
:102FD000BCF802C08C4508D333F8302003EBC000A6
:102FE000891A8088084485B203E0401C80B2904270
:102FF000E8D3BF1C1AE00020E64914E031F830C0E5
:1030000063450ED301EBC00CBCF802C0634508D881
:1030100031F8302001EBC0009A1A8088104485B244
:1030200003E0401C80B29042E8D37F1CD94888302E
:1030300030F83500C0F1A001B14202DA4FF0A00B28
:1030400002E0304400F0FF0BB8F1420F02D95020EB
:10305000009003E008F10E00C0B20090C2462AE0E2
:10306000B146CC48CC49883000EBC50008900AEB4B
:103070008A0001EB8010079017E027E0B1E0D9E16A
:1030800061E108980C9A4168C4482044085C16998C
:1030900013F076FD010201EB1020079921F81900C9
:1030A000641C09F1010909F0FF09D945E9D30AF1C6
:1030B000010A0AF0FF0A00988245D1D30024B548DE
:1030C000883010F835003044C6B2AFE104227E2BC0
:1030D0001FD9787800EB032081B20020B04B14E0B8
:1030E00033F830C08C450ED803EBC00CBCF802C0DE
:1030F0008C4508D333F8302003EBC000891A808850
:10310000084485B203E0401C80B29042E8D3BF1C63
:103110001AE00020A24914E031F830C063450ED314
:1031200001EBC00CBCF802C0634508D831F8302070
:1031300001EBC0009A1A8088104485B203E0401C5D
:1031400080B29042E8D37F1C9548203030F835009B
:10315000C0F1A001B14202DA4FF0A00B02E030440E
:1031600000F0FF0BB8F1370F02D95020009003E0B8
:1031700008F11900C0B20090C24627E0B146884865
:103180008549203000EBC50006900AEB8A0001EB70
:103190008010059014E006980C9A416880489030A1
:1031A0002044085C169913F0EBFC010201EB10209F
:1031B000059921F81900641C09F1010909F0FF09BA
:1031C000D945E8D30AF1010A0AF0FF0A00988245BE
:1031D000D4D300247248203010F835003044C6B2F1
:1031E00024E109227E2B1FD9787800EB032081B2DD
:1031F00000206C4B14E033F830C08C450ED803EB44
:10320000C00CBCF802C08C4508D333F8302003EB67
:10321000C000891A8088084485B203E0401C80B24F
:103220009042E8D3BF1C1AE000205E4914E031F858
:1032300030C063450ED301EBC00CBCF802C063453F
:1032400008D831F8302001EBC0009A1A8088104469
:1032500085B203E0401C80B29042E8D37F1C514805
:10326000483030F83500C0F1A001B14202DA4FF029
:10327000A00B02E0304400F0FF0BB8F1450F02D97B
:103280005020009003E008F10B00C0B20090C2464D
:1032900035E0B14643484049483000EBC500049052
:1032A0000AEB8A0001EB8010039013E004980C9A5B
:1032B00041683D482044085C169913F061FC010206
:1032C00001EB1020039921F81900641C09F1010990
:1032D00009F0FF09D945E9D3BBF1A00F0BD1314863
:1032E000483030F8350094FBF0F100FB1141C9B2D1
:1032F00009B12044441A0AF1010A0AF0FF0A0098B1
:103300008245C6D300242748483010F835003044A1
:10331000C6B28BE033F830C08C450ED803EBC00C3E
:10332000BCF802C08C4508D333F8302003EBC00052
:10333000891A8088084485B203E0401C80B290421C
:10334000E8D3BF1C1AE00020114914E031F830C066
:1033500063450ED301EBC00CBCF802C0634508D82E
:1033600031F8302001EBC0009A1A8088104485B2F1
:1033700003E0401C80B29042E8D37F1C0B4830F839
:103380003500C0F1A001B14212DA4FF0A00B12E0FB
:10339000C0DC020038B80200D0D60120D8BA020042
:1033A0003CA3020078460300F848030020E1020035
:1033B000304400F0FF0BB8F1400F02D950200090CC
:1033C00003E008F11000C0B20090C24625E0B1460B
:1033D0001A490AEB8A0001EB80100290184800EBB2
:1033E000C500019013E001980C9A416815482044EB
:1033F000085C169913F0C4FB010201EB102002993E
:1034000021F81900641C09F1010909F0FF09D945E7
:10341000E9D30AF1010A0AF0FF0A00988245D6D3DF
:103420000024074810F835003044C6B23B78002B22
:103430007FF4A8AD0DB0BDE8F08F0000D0D601201C
:1034400020E1020088E502002DE9F04186B0064641
:10345000DDE90C450F469846062A51D2DFE802F016
:1034600003101D2A374410EE100AFDF765F941ECF0
:10347000100B29A153EC102B03A811F0B1FD3FE074
:1034800010EE100AFDF758F941EC100B24A153EC93
:10349000102B03A811F0A4FD32E010EE100AFDF786
:1034A0004BF941EC100B20A153EC102B03A811F0A9
:1034B00097FD25E010EE100AFDF73EF941EC100BE8
:1034C0001BA153EC102B03A811F08AFD18E010EE9D
:1034D000100AFDF731F941EC100B17A153EC102B3A
:1034E00003A811F07DFD0BE010EE100AFDF724F9A2
:1034F00041EC100B12A153EC102B03A811F070FD3E
:10350000434603AA39463046CDE90045FFF732FD70
:1035100006B0BDE8F0810000252E306600000000F6
:10352000252E316600000000252E326600000000C6
:10353000252E336600000000252E346600000000B2
:10354000252E3566000000002DE9F04186B00646C4
:10355000DDE90C850E9C0F46062B21D2DFE803F037
:1035600003080D12171C14A103A811F039FD17E070
:1035700012A103A811F034FD12E012A103A811F06A
:103580002FFD0DE011A103A811F02AFD08E011A103
:1035900003A811F025FD03E010A103A811F020FD00
:1035A000CDE90054434603AA39463046FFF7E2FC12
:1035B00006B0BDE8F08100002564000025303164CC
:1035C0000000000025303264000000002530336424
:1035D0000000000025303464000000002530356410
:1035E0000000000010B5AFF3008010BD10B5044618
:1035F000002C0CD0012C0AD0022C08D0032C06D0B1
:10360000042C04D04FF4C86111A001F0E1FE1B4866
:1036100054B1012C0DD0022C10D0032C13D090F8F3
:103620004100C0F3000010BD90F83C00C0F3000062
:1036300010BD90F83C00C0F3C00010BD90F83C00F5
:10364000C0F3401010BD90F83C00C0F3801010BDD6
:103650002E2E5C2E2E5C2E2E5C2E2E5C2E2E5C646E
:1036600072697665725C7372635C68633332663468
:1036700036305F636C6B2E63000000000040054035
:10368000F8B50546002000900024284EB6F8FE0349
:103690004AF201510843A6F8FE03002D06D0012D81
:1036A00004D040F2252122A001F092FE4DB196F8FF
:1036B000360020F0010086F8360009244FF48055CA
:1036C00025E096F8260040070ED0D6F80001000647
:1036D0000ED596F82A00C00708D096F8360040F0BC
:1036E000010086F8360015E0012413E0012411E002
:1036F00096F8360040F0010086F836000AE0002017
:10370000FFF774FF01280FD00098401C009000982C
:10371000A842F4D3B6F8FE0320F0010040F425409F
:10372000A6F8FE032046F8BD0024F3E7004005405C
:103730002E2E5C2E2E5C2E2E5C2E2E5C2E2E5C648D
:1037400072697665725C7372635C68633332663487
:1037500036305F636C6B2E6300000000F8B50546E1
:10376000002000900024002D06D0012D04D040F24E
:1037700036311EA001F02CFE274EB6F8FE034AF2A9
:1037800001510843A6F8FE034DB196F82A0020F037
:10379000010086F82A0009244FF4805516E096F8B7
:1037A000260000F00700052806D096F82A0040F011
:1037B000010086F82A000CE001240AE00220FFF74D
:1037C00015FF01280FD00098401C00900098A842D7
:1037D000F4D3B6F8FE0320F0010040F42540A6F82B
:1037E000FE032046F8BD0024F3E700002E2E5C2ED9
:1037F0002E5C2E2E5C2E2E5C2E2E5C6472697665FD
:10380000725C7372635C68633332663436305F6354
:103810006C6B2E63000000000040054010B50446AC
:10382000002C5BD02068801E0E2804D940F20531A0
:103830002BA001F0CDFD6068401E0F2804D940F296
:10384000063127A001F0C4FDA068801E0E2804D90F
:1038500040F2073122A001F0BBFDE0681438B0F55A
:10386000E67F04D94FF442711DA001F0B1FD20693B
:10387000401E172804D940F2093119A001F0A8FD13
:103880002248B0F8FE124AF201521143A0F8FE128B
:1038900021780268491E61F31F7202602179026873
:1038A000491E61F31B620260217A0268491E61F3BE
:1038B00017520260A1890268491E61F3102202605A
:1038C000217C0268491E61F304020260B0F8FE1216
:1038D00021F0010141F42541A0F8FE1210BD0000C5
:1038E0002E2E5C2E2E5C2E2E5C2E2E5C2E2E5C64DC
:1038F00072697665725C7372635C686333326634D6
:1039000036305F636C6B2E630000000000410540A1
:1039100010B50446002C08D0A4F10800052804D9ED
:1039200040F243510BA001F053FD1549B1F8FE03DD
:103930004AF202521043A1F8FE03088A64F303001E
:103940000882B1F8FE0320F0020040F42540A1F8FF
:10395000FE0310BD2E2E5C2E2E5C2E2E5C2E2E5CB9
:103960002E2E5C6472697665725C7372635C686348
:103970003332663436305F636C6B2E6300000000B8
:103980000040054010B50446002C06D0012C04D0A0
:1039900040F2E5210BA001F01BFD1549B1F8FE0234
:1039A0004AF201521043A1F8FE02086864F3C710FE
:1039B0000860B1F8FE0220F0010040F42540A1F8B3
:1039C000FE0210BD2E2E5C2E2E5C2E2E5C2E2E5C4A
:1039D0002E2E5C6472697665725C7372635C6863D8
:1039E0003332663436305F636C6B2E630000000048
:1039F0000041054070B586B00446002605962E4D60
:103A00002868049068680390A8680290E8680190AC
:103A1000002C07D0601E042804D940F2DD3127A015
:103A200001F0D6FC30482861304991F826004A154B
:103A300000F00700052801D0052C0BD12C48286088
:103A4000C0126860A860E8600598401C0590059861
:103A50009042F9D32631B1F8D8034AF20153184302
:103A6000A1F8D803087864F302000870B1F8D8030D
:103A700020F0010040F42540A1F8D80305960598F0
:103A8000401C059005989042F9D30498286003984B
:103A900068600298A8600198E8601348401E286199
:103AA00005960598401C059005989042F9D306B0FC
:103AB000BDE870400FF0C8BD008004402E2E5C2E83
:103AC0002E5C2E2E5C2E2E5C2E2E5C64726976652A
:103AD000725C7372635C68633332663436305F6382
:103AE0006C6B2E63000000000100A5A5004005409E
:103AF000EEFAFFFF10B50446A01E022807D9801F6A
:103B0000052804D940F227510BA001F061FC1549AA
:103B1000B1F8DA034AF201521043A1F8DA03087847
:103B200064F307100870B1F8DA0320F0010040F4E4
:103B30002540A1F8DA0310BD2E2E5C2E2E5C2E2E11
:103B40005C2E2E5C2E2E5C6472697665725C7372DC
:103B5000635C68633332663436305F636C6B2E634C
:103B60000000000024400540F0B585B00446002662
:103B70000496434D2868039068680290A8680190F5
:103B8000E86800903F482861002C76D02178E278E0
:103B900091421BD86379994218D8A079814215D8EF
:103BA000A178914212D8994210D821790A1A032A91
:103BB00011D0022A0FD0012A0DD081420BD0401A19
:103BC000012808D0022806D0032804D040F23C4146
:103BD0002DA001F0FDFB374991F826004A1500F0B1
:103BE000070005280BD134482860C0126860A8601F
:103BF000E8600498401C049004989042F9D3B1F80E
:103C0000FE034AF201531843A1F8FE03A078E378BB
:103C1000677940EA031023791B0243EA073318430C
:103C2000A37940EA0340637840EA0353207843EAEB
:103C3000006343EA00700862B1F8FE0320F001005F
:103C400040F42540A1F8FE0304960498401C04901B
:103C500004989042F9D3039828600298686001980C
:103C6000A8600098E8600748401E28610496049800
:103C7000401C049004989042F9D305B0F0BD0000B8
:103C8000008004400100A5A52E2E5C2E2E5C2E2E59
:103C90005C2E2E5C2E2E5C6472697665725C73728B
:103CA000635C68633332663436305F636C6B2E63FB
:103CB0000000000000400540EEFAFFFF38B5044662
:103CC000002C06D0012C04D040F29F3122A001F03C
:103CD0007FFB2C49B1F8FE034AF201521043A1F8D0
:103CE000FE03012C04D091F82E0040F0010003E007
:103CF00091F82E0020F0010081F82E00B1F8FE03AB
:103D000020F0010040F42540A1F8FE0300204FF40C
:103D100080550CB1009017E0009007E00098401C1F
:103D200000900098A84201D9092038BD0320FFF770
:103D30005DFC0028F2D10CE00098401C0090009837
:103D4000A84201D9092038BD0320FFF74FFC012804
:103D5000F2D1002038BD00002E2E5C2E2E5C2E2EBF
:103D60005C2E2E5C2E2E5C6472697665725C7372BA
:103D7000635C68633332663436305F636C6B2E632A
:103D8000000000000040054070B50446002C7CD0C7
:103D90002068801E0E2804D940F26F313EA001F049
:103DA00017FB6068801E0E2804D94FF45C713AA09E
:103DB00001F00EFBA068801E0E2804D940F271317C
:103DC00035A001F005FBE0681438B0F5E67F04D9B2
:103DD00040F2723130A001F0FBFA2069801E1628F3
:103DE00004D940F273312CA001F0F2FA354DD5F828
:103DF0000001000601D4344801E03448006821691C
:103E0000B0FBF1F0E6684643314908443149884245
:103E100004D940F27A3120A001F0DAFA2E482E4976
:103E200030444942884204D940F27B311AA001F063
:103E3000CFFA05F58275B5F8FA024AF20151084346
:103E4000A5F8FA0220782968401E60F31F712960E6
:103E500020792968401E60F31B612960207A296857
:103E6000401E60F317512960A0892968401E60F345
:103E700010212960207C2968401E60F3040129601C
:103E8000B5F8FA0220F0010000E003E040F425401C
:103E9000A5F8FA0270BD00002E2E5C2E2E5C2E2E90
:103EA0005C2E2E5C2E2E5C6472697665725C737279
:103EB000635C68633332663436305F636C6B2E63E9
:103EC000000000000040054000127A00B082FF1F91
:103ED000C0BDF0FFC0F35E0100E4B1F10421012890
:103EE00003D0022801D0102805D104494FF4AA427A
:103EF0000A80088000210846704700000CA1044099
:103F000038B521480090002003F05AFF00F0070167
:103F100020FA01F2884010441C49884203D91C4908
:103F20000844400803E01A4949420844400019493E
:103F3000194C0968814203D1012084F8240038BD5E
:103F40001649009808441549009A0939114412E0AD
:103F500002787AB10278082302E052085B1EDBB2D5
:103F6000D507FAD00099401AC01C03EBC00084F8B2
:103F7000230002E0401E8842EAD294F8230008B1F0
:103F8000012038BD002038BD53AE004333DDD3538C
:103F900034DDD3D3D890FF1FB083FF1FC65DFFBFB2
:103FA00070B5002500F0D6F81020FEF7D7FF4F4877
:103FB0000088FEF7D9FF00210846FEF7C9FF4CA094
:103FC000FEF778FC00210420FDF776FF4BA0FEF7FA
:103FD00071FC4B4C2088FEF7C7FF10210020FEF734
:103FE000B7FF48A0FEF766FC48A0FEF763FC002080
:103FF00003F0E6FE0821FEF7D9FA20210020FEF7A3
:10400000A7FF43A0FEF7DEF840210020FEF7A0FF47
:104010002088FEF7A9FF424C94F8230040B141A04C
:10402000FEF7D0F8002194F82300FEF74BFF05E0DF
:104030003FA0FEF7C7F840A0FEF73CFC41480088CF
:10404000FEF792FF94F825003F4C082835D2DFE8B0
:1040500000F034040B121920272E20680121000FD4
:1040600003F0CEFE054628E020680221000E03F092
:10407000C7FE054621E020680321000D03F0C0FEC5
:1040800005461AE020680421000C03F0B9FE05463D
:1040900013E020680521000B03F0B2FE05460CE09A
:1040A00020680621000A03F0ABFE054605E0206803
:1040B0000721000903F0A4FE054624A003F006FF33
:1040C0002844C0B23221FEF743FF21A0FEF7F2FBE5
:1040D00030210020FEF73CFF1CA0FEF7EBFB206820
:1040E000BDE870400821FEF761BA0000AC83FF1FF5
:1040F00069444B4D65746572000000003032430026
:10410000AA83FF1F532F4E3A0000000030780000B2
:10411000C7EBCAE4C8EBD7A2B2E1C2EB3A00000099
:10412000B083FF1F52656D61696E5573653A00007B
:104130005151C8BA3A000000373838303133313283
:1041400030000000A883FF1FD890FF1F3E3078008A
:104150005F000000F8B571480090714E3278714CE4
:10416000714F0025206897F82510042A15D0327861
:104170000A2A12D03278052A54D032780B2A51D02C
:104180003078062871D032783846092A90F8230012
:104190006CD031780C296AD0B4E0624A1268D243FC
:1041A00008290AD2DFE801F0040A121A222A323959
:1041B000110F02D000F180502060A3E06FEA10617F
:1041C000090702D000F1807020609BE06FEA105177
:1041D000090702D000F58010206093E06FEA1041DB
:1041E000090702D000F5803020608BE06FEA1031C3
:1041F000090702D000F58050206083E06FEA1021AB
:1042000009077FD000F5807020607BE06FEA101115
:10421000090777D01030206074E0110772D0401C7D
:1042200020606FE008296DD2DFE801F0040A111860
:1042300022293036010F65D0A0F18050206061E066
:10424000010E09075ED0A0F1807020605AE0010DD8
:10425000090757D0A0F58010206053E0010C090732
:1042600050D0A0F5803020604CE01AE03EE047E0FE
:10427000010B090746D0A0F58050206042E0010AFA
:1042800009073FD0A0F5807020603BE001090907D5
:1042900038D01038206035E0010733D0401E206050
:1042A00030E0491CC8B287F8250008282AD187F8D1
:1042B0002550FFF725FE97F8240058B17D7087F848
:1042C000215087F82250194A00982168104403F0C1
:1042D00045FD17E016480168BA6B891AB1F5487FA9
:1042E00010D9022139700068B8630BE019B1491E7A
:1042F00087F8251002E008B111207870357001E0D0
:1043000000B17D703078062805D03078052802D0BD
:104310003078042800D13570F8BD000053AE00435A
:104320006083FF1FD890FF1FB083FF1FB55DFFBFE5
:104330007C83FF1F2DE9FC4100F088F81020FEF778
:104340000DFE3C4EB08EFEF70FFE00210846FEF734
:10435000FFFD39A0FDF736FF708EFEF705FE102138
:104360000020FEF7F5FD002406F23477708EFEF78C
:10437000FBFD601C05460007010E0020FEF7E8FD6E
:1043800096F82000844211D102210020FDF794FD0F
:104390000C20FEF7E3FD308EFEF7E6FD2AA0FEF7C7
:1043A00089FA6FF001010020FDF786FD1020FEF76D
:1043B000D5FD04EB041057F82000FDF703FFECB225
:1043C000042CD3D3FF24308ECDE900042023842293
:1043D00010216420FDF7A2FD708ECDE90004352385
:1043E000842225216420FDF799FDB08ECDE90004DB
:1043F0004A2384223A216420FDF790FD708ECDE996
:1044000000049E224F2300211046FDF787FD708E89
:10441000CDE9000496F820009F2200EB800101EB1B
:10442000C000012101EB400300219D20FDF776FD36
:10443000BDE8FC81B083FF1FD6F7CCE2D1D5C9AB74
:10444000C9E8D6C3000000003E00000070B5404E31
:104450003178404C0025042994F8200003D03178AD
:1044600005290AD012E0032803D2401C84F820005A
:1044700001E084F82050357008E018B1401E84F83F
:10448000200002E0032084F82000357094F820001A
:1044900050B14FF6DC514FF6F37201280ED00228CE
:1044A00012D003281FD117E04FF64D30208640F27E
:1044B000796060864DF69A30A08614E02186628687
:1044C0004AF67D70A0860EE04FF638702086618631
:1044D0004EF27350A08606E0228646F2F3706086A4
:1044E0004AF6DC60A0863078062807D030780928A4
:1044F00003D1657511206070357070BD218E282044
:1045000003F018FC618E2A2003F014FCA18E2C20ED
:1045100003F010FC104994F8200081F8320003F0F9
:10452000C9FB0E49208E08800D49608E08800D4918
:10453000A08E08800C480168A26B891AB1F5487FEB
:1045400003D9012121700068A063357070BD00009F
:104550006083FF1FB083FF1FF8620220A883FF1F44
:10456000AA83FF1FAC83FF1F7C83FF1F70B500F081
:10457000ABF81020FEF7F2FC3D480088FEF7F4FC93
:1045800000210846FEF7E4FC3AA0FDF71BFE3C4D77
:104590002888FEF7E9FC10210020FEF7D9FC39A09D
:1045A000FDF710FE3A4C052094ED150AFEF718FCB5
:1045B00020210020FEF7CCFC36A0FDF703FE384991
:1045C000052091ED000AFEF70BFCA07D354C6FF045
:1045D000020628B301284AD130210020FEF7B8FC9A
:1045E00031A0FDF7EFFD2088FEF7BEFC0C20FEF7A2
:1045F000B5FC40210020FEF7ABFC03210020FDF7B5
:104600005BFC2CA0FEF756F931460020FDF754FC68
:104610001020FEF7A3FCBDE8704027A0FDF7D2BD37
:104620002088FEF7A1FC30210020FEF791FC0C2031
:10463000FEF794FC03210020FDF73EFC1DA0FEF7D1
:1046400039F931460020FDF737FC1020FEF786FCD3
:1046500015A0FDF7B7FD2888FEF786FC4021002055
:10466000FEF776FCBDE8704013A0FDF7ABBD70BD52
:10467000AC83FF1FB5E7C1F7D0A3D7BC0000000093
:10468000AA83FF1FD0C2D0A3D7BCB2CECAFD3A00C6
:10469000B083FF1FBEC9D0A3D7BCB2CECAFD3A00BB
:1046A0004883FF1FA883FF1FB1A3B4E6D0C2B2CED8
:1046B000CAFD00003E000000BBD6B8B4C4ACC8CFF1
:1046C000B2CECAFD000000002DE9F0411F4E317846
:1046D0001F4C00250127A07D04290ED03178052923
:1046E0000FD03178062911D03078092803D16575AB
:1046F000192060703570BDE8F08100B9A77535707C
:10470000F9E708B1401EA0753570F4E798B119209B
:1047100003F0C0FA1D2003F017FB03F0CBFA0D489D
:104720000168A26B891AB1F5487F02D92770006829
:10473000A0633570DFE7084894ED150A80ED000AA4
:1047400090ED000A1D2003F0FFFAE6E76083FF1FEB
:10475000B083FF1F7C83FF1F4883FF1F7CB500F0E1
:10476000DBF81020FEF7FAFB4F480088FEF7FCFB51
:1047700000210846FEF7ECFB4CA0FDF723FD4E4D53
:104780002888FEF7F1FB4D48007830B14FF40071F6
:1047900000200BF0A7FA002833D018210020FEF7E4
:1047A000D7FB2888FEF7E0FB45A0FDF70BFD28218D
:1047B0000020FEF7CDFB47A0FDF704FD484E042086
:1047C00096ED140AFEF70CFB46A0FEF773F83821AD
:1047D0000020FEF7BDFB44A0FDF7F4FC4549042092
:1047E00091ED000AFEF7FCFA3EA0FEF763F8717D3A
:1047F0004148FF2405293ED2DFE801F00C16202AAB
:10480000340028210020FEF7A3FBBDE87C403BA03C
:10481000FDF7D8BC0088CDE90004372339223621C2
:104820003120FDF77BFB26E00088CDE9000437232B
:10483000472236213F20FDF771FB1CE00088CDE9BF
:1048400000043723502236214820FDF767FB12E091
:104850000088CDE900043723592236215120FDF785
:104860005DFB08E00088CDE9000437236222362191
:104870005A20FDF753FB2888CDE900049E224F23E0
:1048800000211046FDF74AFB2888CDE90004707D21
:104890009F2200EB400101EB0013DB1C00219D2057
:1048A000FDF73CFB7CBD0000AC83FF1FB5E7C1F703
:1048B000D0A3D7BC00000000AA83FF1F3083FF1FD6
:1048C000C7EBC9E8D6C3B1EAD7BCB5E7C1F7D6B5DF
:1048D0003A000000B1EAD7BCB5E7C1F73A000000E2
:1048E000B083FF1F41000000B5B1C7B0B5E7C1F705
:1048F0003A0000003883FF1FA883FF1FC7EBCAB927
:10490000D3C3B9ABCDB7CAE4C8EBBBF2CDE2BDD3DC
:10491000484944D0A3D7BC0070B52DED028B5C4D47
:104920002978B7EE008A9FED5B2ADFED5B0ADFEDA9
:104930005B1A9FED5B1A5B4C0026042994ED140A68
:10494000607D0CD029780A2909D0297805292ED034
:1049500029780B292BD02878062850D059E0052833
:104960001CD2DFE800F003080D12170030EE080A31
:1049700084ED140A12E030EE020A84ED140A0DE010
:1049800030EE200A84ED140A08E030EE210A84EDAE
:10499000140A03E030EE010A84ED140A4249206D46
:1049A000884268DDB1EE040A84ED140A63E005284C
:1049B0001CD2DFE800F003080D12170030EE480AA1
:1049C00084ED140A12E030EE420A84ED140A0DE080
:1049D00030EE600A84ED140A08E030EE610A84EDDE
:1049E000140A03E030EE410A84ED140A206DB0F1A0
:1049F0007C5F40DAB6EE000A84ED140A3BE02B48F7
:104A0000007850B14FF4007100200BF06BF90128D1
:104A100003D02878092826D02DE0607D401CC0B244
:104A20006075052827D166752148224A90ED000A55
:104A300010EE101A914211DDD4ED140A90ED001A17
:104A400080EE810A84ED150A10EE100A51420844E6
:104A50001949884204D384ED158A01E084ED158A52
:104A60001A20607007E0607D10B1401E607501E0A3
:104A7000112060702E702878062805D02878052827
:104A800002D02878042800D12E70BDEC028B70BDB6
:104A90006083FF1FCDCCCC3D0AD7233C6F12833AF5
:104AA00017B7D138B083FF1F0000A0403083FF1F2D
:104AB0003883FF1F9A99993E6766A60170B506462E
:104AC0000D4614465F48864207D05F48864204D0B0
:104AD00040F2D1715DA000F07BFC55B1012D08D0F2
:104AE000022D06D0032D04D040F2D27157A000F061
:104AF0006FFC207840B1012806D0022804D040F293
:104B0000D37152A000F064FC607840B1012806D057
:104B1000022804D040F2D4714CA000F059FCA078D7
:104B200030B1012804D040F2D57148A000F050FC0B
:104B3000E07830B1012804D040F2D67143A000F0F3
:104B400047FC207930B1012804D040F2D7713FA052
:104B500000F03EFC607930B1012804D04FF4FB61D5
:104B60003AA000F035FCA07940B1012806D0022817
:104B700004D040F2D97135A000F02AFCE07930B1C0
:104B8000012804D040F2DA7130A000F021FC207A34
:104B900030B1012804D040F2DB712CA000F018FCE9
:104BA000607A30B1012804D040F2DC7127A000F017
:104BB0000FFC06EB8510C16D227821F00301114333
:104BC000C165C16D627821F00C0141EA8201C165C5
:104BD000C16DA27821F0100141EA0211C165C16DD9
:104BE000E27821F0200141EA4211C165C16D2279CC
:104BF00021F0400141EA8211C165C16D627921F065
:104C0000800141EAC211C165C16DA27921F44071F0
:104C100041EA0221C165C16DE27921F4806141EA76
:104C20008221C165C16D227A21F4006141EAC2216D
:104C3000C165C16D627A21F4805141EA0231C165DA
:104C400070BD000000300540003405402E2E5C2E63
:104C50002E5C2E2E5C2E2E5C2E2E5C647269766588
:104C6000725C7372635C68633332663436305F64DF
:104C70006D61632E630000002DE9F04704460D4688
:104C8000174600265B48844207D05B48844204D024
:104C900040F2872159A000F09BFB55B1012D08D0AF
:104CA000022D06D0032D04D04FF4227153A000F042
:104CB0008FFB37B1012F04D040F289214FA000F0C3
:104CC00087FB5949087810B10120BDE8F08701231E
:104CD0000B70E069AB409843002290B3E0694FF05D
:104CE0000A0CC0074FF4A04817D0B5B1A06C000C57
:104CF000D4F86890BCEB194F0FD3D4F86890B0EBA0
:104D0000194F07D809E0761CB6B2464502D90A7099
:104D10000920DAE7E069C007F5D1E06980071BD513
:104D2000012D19D0D4F88800000CD4F8A860BCEB91
:104D3000164F11D3D4F8A860B0EB164F0CD9002051
:104D400007E03AE0401C80B2404502D90A700920D1
:104D5000BBE7E669B607F5D4E06940071AD5022D2E
:104D600018D00020D4F8C860360CD4F8E890BCEB1A
:104D7000194F0FD3D4F8E890B6EB194F07D809E0D4
:104D8000401C80B2404502D90A7009209DE7E669BF
:104D90007607F5D4E06900071AD5032D18D0002056
:104DA000D4F808512D0CD4F82861BCEB164F0FD362
:104DB000D4F82861B5EB164F07D809E0401C80B243
:104DC000404502D90A7009207FE7E5692D07F5D42F
:104DD0003FB1012F0AD1E06903F00F031843E061EE
:104DE00004E0E0690F259D432840E0610A7000203F
:104DF0006BE7000000300540003405402E2E5C2E8D
:104E00002E5C2E2E5C2E2E5C2E2E5C6472697665D6
:104E1000725C7372635C68633332663436305F642D
:104E20006D61632E63000000F090FF1F2DE9F041DB
:104E300005460C46164600272548854207D02548DA
:104E4000854204D040F24E2123A000F0C1FA54B1B3
:104E5000012C08D0022C06D0032C04D040F24F21A4
:104E60001DA000F0B5FA56B1012E08D0022E06D0D2
:104E7000032E04D04FF4147117A000F0A9FA3CB12E
:104E8000012C05D0022C03D0032C01D004270CE008
:104E90000120A04066B110340121A140012E0BD0A9
:104EA000022E0DD0032E0FD004273846BDE8F08126
:104EB000696901436961F8E7686908436861F4E773
:104EC000A9690143A961F0E7A8690843A861ECE773
:104ED00000300540003405402E2E5C2E2E5C2E2E18
:104EE0005C2E2E5C2E2E5C6472697665725C737229
:104EF000635C68633332663436305F646D61632EA1
:104F00006300000070B504460D460C48844207D08B
:104F10000B48844204D04FF4C1710AA000F058FA43
:104F200035B1012D04D040F2831106A000F050FAF3
:104F3000206865F30000206070BD0000003005406F
:104F4000003405402E2E5C2E2E5C2E2E5C2E2E5C08
:104F50002E2E5C6472697665725C7372635C686342
:104F60003332663436305F646D61632E6300000057
:104F700070B506460D4614463A48864207D03A4870
:104F8000864204D040F6120138A000F021FA55B153
:104F9000012D08D0022D06D0032D04D040F61301B8
:104FA00032A000F015FA2088800A04D040F61401DF
:104FB0002EA000F00DFAA089800A04D040F6160158
:104FC0002AA000F005FAE089800A04D040F6170113
:104FD00026A000F0FDF901213046FFF793FF06EB14
:104FE0008513D86D20F48050D86560681864A06877
:104FF0005864986C21886FF30900084398646188AD
:10500000986C61F31F409864D86CA1896FF3090014
:105010000843D864D86C20490840E18940EA01403F
:10502000D864186D61696FF3130008431865218B0C
:10503000186D61F31F501865586DE1696FF3130027
:1050400008435865218C586D61F31F5058652069DD
:10505000986504F1240229463046BDE87040FFF708
:105060002DBD000000300540003405402E2E5C2E82
:105070002E5C2E2E5C2E2E5C2E2E5C647269766564
:10508000725C7372635C68633332663436305F64BB
:105090006D61632E63000000FFFF00FC2DE9F0410D
:1050A00080460D461646002400271548804507D047
:1050B0001448804504D040F2354113A000F088F92F
:1050C00055B1012D08D0022D06D0032D04D040F299
:1050D00036410DA000F07CF908EB85114E644FF4C9
:1050E000805006E0641CA4B2844201D9092700E084
:1050F0004E644A6EB242F5D13846BDE8F0810000F8
:1051000000300540003405402E2E5C2E2E5C2E2EE5
:105110005C2E2E5C2E2E5C6472697665725C7372F6
:10512000635C68633332663436305F646D61632E6E
:10513000630000002DE9F04180460D46164600242C
:1051400000271548804507D01448804504D040F218
:10515000F33113A000F03CF955B1012D08D0022D18
:1051600006D0032D04D04FF47D710DA000F030F96E
:1051700008EB85110E644FF4805006E0641CA4B265
:10518000844201D9092700E00E640A6EB242F5D1CB
:105190003846BDE8F081000000300540003405408D
:1051A0002E2E5C2E2E5C2E2E5C2E2E5C2E2E5C6403
:1051B00072697665725C7372635C686333326634FD
:1051C00036305F646D61632E630000002DE9F041AD
:1051D00080460D461646002400271848804507D013
:1051E0001748804504D040F2BB4116A000F0F0F80B
:1051F00055B1012D08D0022D06D0032D04D040F268
:10520000BC4110A000F0E4F808EB8511886C66F34F
:105210001F4088644FF4805009E0641CA4B28442AB
:1052200001D9092703E08A6C66F31F428A648A6EFB
:10523000B6EB124FF1D13846BDE8F08100300540A1
:10524000003405402E2E5C2E2E5C2E2E5C2E2E5C05
:105250002E2E5C6472697665725C7372635C68633F
:105260003332663436305F646D61632E6300000054
:105270002DE9F0410446884615460C4E0C4FB442C9
:1052800006D0BC4204D040F247710AA000F0A0F85A
:105290001349B44201EB880003D1C0F81458BDE8AB
:1052A000F081BC42FBD1C0F82458F8E7003005403B
:1052B000003405402E2E5C2E2E5C2E2E5C2E2E5C95
:1052C0002E2E5C6472697665725C7372635C6863CF
:1052D0003332663436305F646D61632E63000000E4
:1052E0000000014010B54FF4007101200AF034FEB7
:1052F0001021BDE8104001200AF02EBE10B54FF479
:10530000007101200AF05CFE1021BDE81040012070
:105310000AF022BE10B54FF4007101200AF050FED1
:105320001021BDE8104001200AF04ABE10B54FF42C
:10533000807101200AF010FE0821BDE81040012014
:105340000AF00ABE10B54FF4807101200AF038FE51
:105350000821BDE8104001200AF0FEBD10B54FF451
:10536000807101200AF02CFE0821BDE810400120C8
:105370000AF026BE1CB50020009001908DF80000B8
:105380006A464FF4807101200AF00EFD6A4608213A
:1053900001200AF009FD4FF400746A4621460120FD
:1053A0000AF002FD6A46102101200AF0FDFC6A465F
:1053B000214600200AF0F8FC6A46210100200AF08C
:1053C000F3FC6A46610100200AF0EEFC1CBD0000FF
:1053D00010B50A46014602A00FF0F2FDFEE70000FC
:1053E00057726F6E6720706172616D65746572735C
:1053F0002076616C75653A2066696C65202573209E
:105400006F6E206C696E652025640D0A0000000037
:1054100008B5084942F210720968B1FBF2F304E0E2
:10542000009300994A1E0092FBD2401E411CF7D106
:1054300008BD0000B482FF1F08B50A490A4A09687E
:1054400091420BD9B1FBF2F304E0009300994A1E9C
:105450000092FBD2401E411CF7D108BD401E411CEA
:10546000FCD108BDB482FF1F8096980010B5AFF341
:10547000008010BD30B58FB0302103A8FAF7A3FF2C
:10548000002401940294012188030BF0A5F8012166
:1054900048040BF0A1F80125ADF80C504FF4A060C2
:1054A000ADF80E0032480490324805900794ADF8EC
:1054B00024400894ADF82C400A948DF830408DF8C3
:1054C00031508DF834408DF835408DF836508DF8D8
:1054D00037408DF83950284C03AA00212046FFF7A9
:1054E00047FD4FF4E07200212046FFF7C1FE012185
:1054F0002046FFF707FD012200212046FFF7BCFBF5
:105500000520ADF806001D4802902020ADF80400EB
:1055100001A812F04DFBBDF90600F021002804DBC4
:1055200000F1E02080F8001405E000F00F0000F129
:10553000E02080F8141DBDF90600002809DB00F00A
:105540001F0105FA01F14009800000F1E020C0F8D8
:105550008012BDF90600002808DB00F01F018D4015
:105560004009800000F1E020C0F800510FB030BDCC
:1055700054000440D0CC012000300540E10D010072
:1055800010B50446002C05D0012C03D0BB2107A088
:10559000FFF71EFF1049012C03D0086840F00100FE
:1055A00002E0086820F00100086010BD2E2E5C2E7D
:1055B0002E5C2E2E5C2E2E5C2E2E5C64726976651F
:1055C000725C7372635C68633332663436305F6575
:1055D000666D2E63000000000404014010B504460F
:1055E000012C11D0022C0FD0042C0DD0082C0BD084
:1055F000102C09D0202C07D0B4F5807F04D040F2C5
:10560000951105A0FFF7E4FE0E480068204201D086
:10561000012010BD002010BD2E2E5C2E2E5C2E2EE3
:105620005C2E2E5C2E2E5C6472697665725C7372E1
:10563000635C68633332663436305F65666D2E6353
:10564000000000001004014004480168012903D152
:1056500043F2102101600160704700000004014026
:105660000FB50649009106490A6801924A680292FC
:105670008968039101A90EC90EC00FBD3FCA02403F
:105680005004014010B50446002C21D0012C1FD03D
:10569000022C1DD0032C1BD0042C19D0052C17D0A4
:1056A000062C15D0072C13D0082C11D0092C0FD0A4
:1056B0000A2C0DD00B2C0BD00C2C09D00D2C07D0A4
:1056C0000E2C05D00F2C03D0DC2104A0FFF780FEA8
:1056D0000D48016864F30711016010BD2E2E5C2E89
:1056E0002E5C2E2E5C2E2E5C2E2E5C6472697665EE
:1056F000725C7372635C68633332663436305F6544
:10570000666D2E6300000000080401402DE9F0479B
:1057100005460F4600260024244885420BD2234824
:105720003830854207D92248854204D940F21B21EE
:1057300020A0FFF74DFE3F20FBF7E7F9DFF8A09030
:10574000D9F80000C0F30048D9F8000020F48030F8
:10575000C9F800000120FBF7DDF909F10402106827
:1057600020F07000103010602F609114101D04E0C4
:10577000641CA4B28C4200D909260368DB05F7D566
:10578000BF4200D001261020FBF7BFF9106820F0BF
:10579000700010600020FBF7BDF9D9F8000068F335
:1057A0001040C9F800003046BDE8F087C00F000384
:1057B000DFFF07002E2E5C2E2E5C2E2E5C2E2E5C24
:1057C0002E2E5C6472697665725C7372635C6863CA
:1057D0003332663436305F65666D2E63000000003C
:1057E00008040140034840F22311016043F21021F4
:1057F000016070470004014010B50446217800297B
:1058000021D001291FD002291DD003291BD0042932
:1058100019D0052917D0062915D0072913D0082932
:1058200011D009290FD00A290DD00B290BD00C2932
:1058300009D00D2907D00E2905D00F2903D06D21DD
:105840000BA0FFF7C5FD2078164901EB80016278B7
:10585000086862F3C7100860A278086862F3051050
:105860000860E278086862F301000860002010BD5B
:105870002E2E5C2E2E5C2E2E5C2E2E5C2E2E5C642C
:1058800072697665725C7372635C68633332663426
:1058900036305F6578696E745F6E6D695F737769C6
:1058A0002E6300001010054003498A6D01238340D8
:1058B0001A438A65002070470010054070B50F211B
:1058C0000B2002F031F90421022002F02DF94FF4EF
:1058D000005102200AF006FA0125164C01280BD0CF
:1058E0000220FFF795FD402000F099F9C0F3401128
:1058F00000F0030019B106E02570012070BD10B161
:105900002570012070BD0821022002F00DF902204F
:10591000FFF77EFD402000F082F9C0F3401100F057
:10592000030000B109B1002070BD022020700120E9
:1059300070BD00002083FF1F70B50F210B2002F007
:10594000F3F80721022002F0EFF84FF40051022093
:105950000AF0C8F90125164C01280BD00220FFF7E8
:1059600057FD402000F05BF9C0F3401100F0030048
:1059700019B106E02570012070BD10B1257001201D
:1059800070BD0B21022002F0CFF80220FFF740FD8E
:10599000402000F044F9C0F3401100F0030000B1D2
:1059A00009B1002070BD02202070012070BD0000F0
:1059B0002083FF1F10B503210C2002F0B5F804214D
:1059C000022002F0B1F80D49002008704870C8703C
:1059D000087128210A48FAF7F6FC38210948FAF735
:1059E000F2FC4FF486710848FAF7EDFC074801789D
:1059F000092901D10821017010BD00002083FF1F7B
:105A0000A8CC0120C8B6FF1F68B8FF1FB183FF1FD5
:105A100010B500F091F84FF4804102200AF062F9CD
:105A200018B1BDE8104000F00BB800F043F8024890
:105A300000680249C86110BD7C83FF1FC8B6FF1F04
:105A400010B5FFF73BFF00282ED0FF210E2002F0FB
:105A50006BF801210F2002F067F8E7210A2002F01D
:105A600063F80021062002F05FF810480078012852
:105A700002D0022809D010E00421022002F054F8DC
:105A80004121032002F050F807E00821022002F033
:105A90004BF84221032002F047F80121072002F0D1
:105AA00043F803490220887310BD00002083FF1FC4
:105AB000C8B6FF1F10B5FFF73FFF00282DD0FF210C
:105AC0000E2002F031F8E7210A2002F02DF8002123
:105AD000062002F029F811480078012802D0022897
:105AE00009D010E00521022002F01EF82121032038
:105AF00002F01AF807E00A21022002F015F822212C
:105B0000032002F011F80121072002F00DF80449EA
:105B10000320887303491420087010BD2083FF1FE1
:105B2000C8B6FF1FB183FF1F10B500F08DF8BDE8A8
:105B300010400C20FFF7B8BE70B586B00024059465
:105B400003940494019402940C268DF814600125AA
:105B50008DF815508DF816508DF8174005A8FFF7F1
:105B60004BFE019402948DF804408DF806508DF898
:105B7000085001AA290301200AF016F9ADF80C60BB
:105B80000420ADF80E001948049003A812F010F894
:105B9000BDF90E00002809DB00F01F0105FA01F134
:105BA0004009800000F1E020C0F88012BDF90E002D
:105BB000F021002804DB00F1E02080F8001405E06B
:105BC00000F00F0000F1E02080F8141DBDF90E0078
:105BD000002808DB00F01F018D404009800000F123
:105BE000E020C0F8005106B070BD0000295B010044
:105BF00038B505460C46002C10D0432000902220DA
:105C000003F0FEF918B90121684603F06FF903F0BB
:105C100015FA22462946222003F0E0F838BD01B5E6
:105C200082B0222003F0ECF918B9012102A803F098
:105C30005DF903F003FA012201A9222003F0CEF856
:105C40009DF804000EBD00002DE9FC479F4D6889BA
:105C50009F4E00EBC00006EB80000121FFF7C8FF5C
:105C6000A6F138094FF0020801270FE168890221E7
:105C700000EBC00006EB8000801CFFF7B9FF6889CD
:105C800000EBC00016F82000DF2838D84FF4005190
:105C900002200AF027F8012830D16878012818D0AE
:105CA000688900EBC00006EB80004088C0F38110DB
:105CB000A8702878012802D0022805D008E0012128
:105CC000032001F031FF03E00221032001F02CFF4B
:105CD0006F70688900EBC00006EB8000408800F020
:105CE0001F00012861D0688900EBC00006EB80002E
:105CF0004088C0F34220288100F088F955E0687898
:105D0000022852D0688900EBC00006EB8000408872
:105D1000C0F38110A87099F80E00012802D0022863
:105D20002CD042E0688900EBC00006EB8000408880
:105D3000C0F34220288100F031F9688900EBC000EF
:105D400006EB800080F820702878012802D0022815
:105D500009D010E0A878052101EB4010C1B2032062
:105D600001F0E2FE07E0A878062101EB4010C1B285
:105D7000032001F0D9FE85F8018016E0287801287B
:105D800002D0022808D00EE0A87807EB4010C1B27C
:105D9000032001F0C9FE06E0A87808EB4010C1B26C
:105DA000032001F0C1FE85F80180688900EBC00086
:105DB00006EB80004088C0F30230698901EBC10125
:105DC00006EB81014988C90B3BD0012839D9401E17
:105DD00084B26889022100EBC00006EB800000EB72
:105DE0008400001DFFF704FF688900EBC00006EB8C
:105DF000800000EB8400406810F4F04F12D00221C4
:105E00006846FFF7F5FEA006010E688900EBC000AA
:105E100006EB8000001DFFF7EBFE04216846FFF74C
:105E2000E7FE1CE0A006010E688900EBC00006EB4F
:105E30008000001DFFF7DCFE06216846FFF7D8FE54
:105E40000DE08006010E688900EBC00006EB8000C3
:105E5000001DFFF7CDFE04216846FFF7C9FE6889E3
:105E600000EBC00006EB800080F821706889401CC0
:105E7000688168890A2801D1002068816889012128
:105E800000EBC00006EB8000FFF7B2FE688900EB74
:105E9000C00016F82000C028BFF4E8AE3F20FFF78E
:105EA000BEFEC0070CD0688940B16889401E00EB77
:105EB000C00006EB800080F8207001E086F8647175
:105EC000BDE8FC474220FFF7AABE00002083FF1F69
:105ED00000B7FF1F3EB5044600212B4A6B46505CBD
:105EE0005854491C0A29FADB9DF8060000F0F1001D
:105EF0008DF806002549A4B11B208DF802008DF80D
:105F000003009DF8050040F0400001220B7942EAB1
:105F100043028DF80620897840EA81108DF805004B
:105F20000BE0CA7840EA42008DF806009DF80500B3
:105F3000897840EA81108DF805000A21684601F051
:105F4000DDFDECB109F0D6FD114B124AE0241888B2
:105F500000EB400102F821409DF805409DF80650F5
:105F600002EB810104EB05244C8042F20F71884260
:105F700001D2401C188008480168491C01603EBDE0
:105F800009F0ACFDE0E70000DAA202002083FF1F69
:105F90007083FF1F74B9FF1F7883FF1F0EB50020A9
:105FA00015496A460B5C1354401CC0B20A28F9D349
:105FB0009DF8070000F0F10010499DF806208B784D
:105FC00042EA83128DF80620098940EA41008DF8E3
:105FD00007000A21684601F091FD0948094A01219C
:105FE000008800EB400002EB80000172064908685F
:105FF000401C08600EBD0000C0A002002083FF1FEF
:106000007083FF1F74B9FF1F7883FF1F0EB5002038
:1060100011496A460B5C1354401CC0B20A28F9D3DC
:106020009DF8070000F0F1000C49098940EA4100A1
:106030008DF807000A21684601F060FD0848094A0A
:106040000121008800EB400002EB8000017206484D
:106050000168491C01600EBDB6A002002083FF1F2D
:106060007083FF1F74B9FF1F7883FF1F3EB50020A8
:1060700021496A460B5C1354401C0A28FADB9DF840
:10608000060000F0F1001D49CA7840EA42008DF890
:1060900006009DF80500897840EA8110C0B28DF8AD
:1060A00005001749C97D012903D140F020008DF872
:1060B00005000A21684601F021FD09F00FFD114A93
:1060C000114BE024108800EB400103F821409DF8BB
:1060D00005409DF8065003EB810104EB05244C803C
:1060E00042F20F71884201D2401C108007480168BB
:1060F000491C01603EBD00006EA102002083FF1F0D
:10610000A8CC01207083FF1F74B9FF1F7883FF1F85
:106110007FB50020244A6946135C0B54401C0E28AE
:10612000FADB9DF8060000F0F1002049CA7840EA49
:1061300042008DF806009DF80500897840EA81103C
:106140008DF805001A4800681A4948620E21684611
:1061500001F0D4FC09F0C2FC174A184BE024108867
:1061600000EB400103F821409DF805409DF80650E2
:1061700003EB810104EB05244C809DF807309DF86A
:106180000A409DF8085003EB04639DF8094024047D
:1061900004EB052423444B6042F20F71884201D284
:1061A000401C10807FBD000012A302002083FF1F4F
:1061B0007C83FF1FC8B6FF1F7083FF1F74B9FF1FCA
:1061C0007FB50020244A6946135C0B54401C0E28FE
:1061D000FADB9DF8060000F0F1002049CA7840EA99
:1061E00042008DF806009DF80500897840EA81108C
:1061F0008DF805000E21684601F080FC09F06EFC68
:10620000174B184AE024188800EB400102F821409F
:106210009DF805409DF8065002EB810104EB052432
:106220004C809DF807209DF80A409DF8085002EB2D
:1062300004629DF80940240404EB052422444A60CA
:1062400042F20F71884201D2401C18800648016852
:10625000491C01607FBD0000E4A202002083FF1FF3
:106260007083FF1F74B9FF1F7883FF1F2DE9F04172
:1062700088B0FE4C694694F820200B2A5ED2DFE8F5
:1062800002F05D060E172029323B444C55000020D9
:10629000F74B1D5C0D54401C0E28FADB4EE000202D
:1062A000F34B8C331D5C0D54401C0E28FADB45E08B
:1062B0000020EF4B9A331D5C0D54401C0E28FADB76
:1062C0003CE00020EA4BA8331D5C0D54401C0E2816
:1062D000FADB33E00020E64BB6331D5C0D54401C66
:1062E0001E28FADB2AE00020E14BD4331D5C0D545C
:1062F000401C1E28FADB21E00020DD4BF2331D5C40
:106300000D54401C1228FADB18E00020D94B1D5C0C
:106310000D54401C1228FADB10E00020D54B12333C
:106320001D5C0D54401C1E28FADB07E00020D14BF9
:1063300030331D5C0D54401C1228FADB9DF806001A
:1063400000F0F100CC49CB7840EA43008DF806001C
:106350009DF80500897840EA81108DF805000B2A28
:1063600038D2DFE802F037060B10151A1F24292E49
:1063700033000E21684601F0C1FB2BE00E21684678
:1063800001F0BCFB26E00E21684601F0B7FB21E0DE
:106390000E21684601F0B2FB1CE01E21684601F0A8
:1063A000ADFB17E01E21684601F0A8FB12E01221A8
:1063B000684601F0A3FB0DE01221684601F09EFB48
:1063C00008E01E21684601F099FB03E012216846AF
:1063D00001F094FB09F082FBA84FA94AE02338881A
:1063E00000EB400102F821309DF805309DF8065081
:1063F00002EB810103EB05234B8094F820C0A14BF5
:10640000A14A4FF4FA75BCF10B0F16D2DFE80CF07D
:106410001506162636469AF3F1F0EF009DF8072090
:106420009DF80A309DF8085002EB03629DF8093090
:106430001B0403EB05231A444A60B5E19DF80720CD
:106440009DF80A309DF8085002EB03629DF8093070
:106450001B0403EB05231A444A60A5E19DF80720BD
:106460009DF80A309DF8085002EB03629DF8093050
:106470001B0403EB05231A444A6095E19DF80720AD
:106480009DF80A309DF8085002EB03629DF8093030
:106490001B0403EB05231A444A6085E11688AE42CB
:1064A000CBD29DF807109DF80A509DF8088001EBAB
:1064B00005619DF809502D0405EB08250D4403EBFB
:1064C00046114D609DF80B309DF80E509DF80C80E4
:1064D00003EB05639DF80D502D0405EB08252B44B7
:1064E0008B609DF80F309DF812509DF8108003EBE3
:1064F00005659DF811301B0403EB08232B44CB608A
:106500009DF813309DF816509DF8148003EB056339
:106510009DF815502D0405EB08252B440B619DF8C3
:1065200017309DF81A509DF8188003EB05639DF80D
:1065300019502D0405EB08252B444B610880761C6F
:10654000168031E11688AE4287D29DF807109DF87B
:106550000A509DF8088001EB05619DF809502D0453
:1065600005EB08250D4403EB46114D609DF80B30FB
:106570009DF80E509DF80C8003EB05639DF80D50BF
:106580002D0405EB08252B448B609DF80F309DF8FA
:1065900012509DF8108003EB05639DF811502D04F7
:1065A00005EB08252B44CB609DF813309DF8165061
:1065B0009DF8148003EB05639DF815502D0405EB41
:1065C00008252B440B619DF817309DF81A5003EBFA
:1065D00005659DF819304FEA03489DF8183008EB1F
:1065E00003232B444B610880761C1680DCE0B5E069
:1065F00060E027E0FFE71188A94222D29DF807500A
:106600009DF80A609DF8088005EB06659DF8096015
:1066100003EB4113360406EB082635445D609DF814
:106620000B509DF80E609DF80C8005EB06659DF8FB
:106630000D60360406EB082635449D601880491C21
:106640001180B1E01188A94233D29DF807509DF81E
:106650000A609DF8088005EB06659DF8096003EB6C
:106660004113360406EB082635440FE0A8CC012080
:1066700078A102007CA202002083FF1F7083FF1F0D
:1066800074B9FF1F288E01207283FF1F5D609DF883
:106690000B509DF80E609DF80C8005EB06659DF88B
:1066A0000D60360406EB082635449D601880491CB1
:1066B000118079E01688AE4276D29DF807109DF8D9
:1066C0000A509DF8088001EB05619DF809502D04E2
:1066D00005EB08250D4403EB46114D609DF80B308A
:1066E0009DF80E509DF80C8003EB05639DF80D504E
:1066F0002D0405EB08252B448B609DF80F309DF889
:1067000012509DF8108003EB05639DF811502D0485
:1067100005EB08252B44CB609DF813309DF81650EF
:106720009DF8148003EB05639DF815502D0405EBCF
:1067300008252B440B619DF817309DF81A509DF8E1
:10674000188003EB05639DF819502D0405EB08250F
:106750002B444B610880761C168025E01188A942E5
:1067600022D29DF807509DF80A609DF8088005EB3D
:1067700006659DF8096003EB4113360406EB082615
:1067800035445D609DF80B509DF80E609DF80C80BF
:1067900005EB06659DF80D60360406EB08263544CA
:1067A0009D601880491C118042F20F71884201D20D
:1067B000401C388005480168491C01600CF1010C3F
:1067C00084F820C008B0BDE8F08100007883FF1F86
:1067D0002DE9F04188B0FE4C694694F82020072A44
:1067E00039D2DFE802F038040C151E2730000020F3
:1067F000F84B1D5C0D54401C0E28FADB2BE00020EA
:10680000F44B0E331D5C0D54401C1E28FADB22E0B5
:106810000020F04B2C331D5C0D54401C1E28FADB6D
:1068200019E00020EB4B4A331D5C0D54401C12282C
:10683000FADB10E00020E74B5C331D5C0D54401C7C
:106840001E28FADB07E00020E24B7A331D5C0D5472
:10685000401C1228FADB9DF8060000F0F100DE492A
:10686000CB7840EA43008DF806009DF80500897852
:1068700040EA81108DF80500072A26D2DFE802F0F1
:106880002504090E131821000E21684601F036F97F
:106890001BE01E21684601F031F916E01E21684612
:1068A00001F02CF911E01221684601F027F90CE003
:1068B0001E21684601F022F9C8480068C849C8622C
:1068C00003E01221684601F019F909F007F9C54DF6
:1068D000C54AE023288800EB400102F821309DF8EA
:1068E00005309DF8066003EB062602EB81035E800F
:1068F00094F82060BD49BE4A4FF4FA77072E14D2AF
:10690000DFE806F01304146CC5F0EE009DF80710E4
:106910009DF80A209DF8087001EB02619DF809209E
:10692000120402EB07221144596070E11388BB4244
:10693000FBD29DF807709DF80AC09DF8088007EB10
:106940000C679DF809C001EB43114FEA0C4C0CEBAE
:10695000082C67444F609DF80B709DF80EC09DF8A1
:106960000C8007EB0C679DF80DC04FEA0C4C0CEB4C
:10697000082C67448F609DF80F709DF812C09DF839
:10698000108007EB0C679DF811C04FEA0C4C0CEB24
:10699000082C6744CF609DF813709DF816C09DF8D1
:1069A000148007EB0C679DF815C04FEA0C4C0CEBFC
:1069B000082C67440F619DF817709DF81AC007EB0B
:1069C0000C689DF819709DF818C03F0407EB0C2760
:1069D00047444F6108805B1C138018E11388BB4259
:1069E00054D29DF807709DF80AC09DF8088007EB07
:1069F0000C679DF809C001EB43114FEA0C4C0CEBFE
:106A0000082C67444F609DF80B709DF80EC09DF8F0
:106A10000C8007EB0C679DF80DC04FEA0C4C0CEB9B
:106A2000082C67448F609DF80F709DF812C09DF888
:106A3000108007EB0C679DF811C04FEA0C4C0CEB73
:106A4000082C6744CF609DF813709DF816C09DF820
:106A5000148007EB0C679DF815C04FEA0C4C0CEB4B
:106A6000082C67440F619DF817709DF81AC09DF8B7
:106A7000188007EB0C679DF819C04FEA0C4C0CEB23
:106A8000082C67444F6108805B1C1380BFE01388AB
:106A9000BB4224D29DF807709DF80AC09DF808807B
:106AA00007EB0C679DF809C001EB43114FEA0C4C52
:106AB0000CEB082C67444F609DF80B709DF80EC0DE
:106AC0009DF80C8007EB0C679DF80DC04FEA0C4C4D
:106AD0000CEB082C67448F6008805B1C138096E0E9
:106AE00059E0FFE71388BB4254D29DF807709DF828
:106AF0000AC09DF8088007EB0C679DF809C001EB00
:106B000043114FEA0C4C0CEB082C67444F609DF886
:106B10000B709DF80EC09DF80C8007EB0C679DF87C
:106B20000DC04FEA0C4C0CEB082C67448F609DF8AD
:106B30000F709DF812C09DF8108007EB0C679DF850
:106B400011C04FEA0C4C0CEB082C6744CF609DF849
:106B500013709DF816C09DF8148007EB0C679DF824
:106B600015C04FEA0C4C0CEB082C67440F619DF8E4
:106B700017709DF81AC09DF8188007EB0C679DF8F8
:106B800019C04FEA0C4C0CEB082C67444F6108808D
:106B90005B1C13803BE01388BB4238D29DF8077022
:106BA0009DF80AC09DF8088007EB0C679DF809C0A6
:106BB00001EB43114FEA0C4C0CEB082C67444F607F
:106BC0009DF80B709DF80EC007EB0C6712E00000FB
:106BD000A8CC012078A102002083FF1F7C83FF1F27
:106BE000C8B6FF1F7083FF1F74B9FF1F288E0120D6
:106BF0007283FF1F9DF80DC09DF80C804FEA0C4C6E
:106C00000CEB082C67448F6008805B1C138042F2F9
:106C10000F71884201D2401C288005480168491C38
:106C20000160761C84F8206008B0BDE8F0810000A7
:106C30007883FF1F70B586B00020344A01A9135C29
:106C40000B54401CC0B21228F9D39DF80A0000F082
:106C5000F1002F49CA7840EA42008DF80A009DF8F9
:106C60000900897840EA81108DF80900122101A8F5
:106C700000F044FF08F032FF264D274AE023288821
:106C800000EB400102F821309DF809309DF80A40E0
:106C900002EB810103EB04234B809DF80B209DF850
:106CA0000E109DF80C3002EB01619DF80D201204CE
:106CB00002EB03228C1819490C609DF80F209DF8F7
:106CC00012309DF8106002EB03629DF811301B0436
:106CD00003EB062313444B60114E3188B1F5FA7F64
:106CE00007D2104A02EB4112546093601080491C95
:106CF000318042F20F71884201D2401C28800A493B
:106D00000868401C086006B070BD00002AA302009D
:106D10002083FF1F7083FF1F74B9FF1FA8CC0120C1
:106D20007283FF1F288E01207883FF1F7FB500200C
:106D3000244A6946135C0B54401C0E28FADB9DF86C
:106D4000060000F0F1002049CA7840EA42008DF8C0
:106D500006009DF80500897840EA81108DF805004D
:106D60000E21684600F0CAFE08F0B8FE174B184A1C
:106D7000E024188800EB400102F821409DF805400E
:106D80009DF8065002EB810104EB05244C809DF830
:106D900007209DF80A409DF8085002EB04629DF818
:106DA0000940240404EB052422444A6042F20F7196
:106DB000884201D2401C188006480168491C0160C5
:106DC0007FBD0000F2A202002083FF1F7083FF1F1F
:106DD00074B9FF1F7883FF1F2DE9F04F85B0DFF8EE
:106DE000C89399F8287099F829103944491E8142AE
:106DF0003EDBEE4CEE4D216A2A68511A502937D3FA
:106E0000A17C0126012932D0DFF8A8C3411CCAB2F7
:106E10008CF80520E8496B4691F81AA0BAF1010FE9
:106E200029D00021DFF8948318F801B003F801B0ED
:106E3000491CC9B20E29F7D39DF8061001F0F101E3
:106E40009CF8033041EA43018DF806109DF80510C7
:106E50009CF8023041EA83118DF80510974216D351
:106E60009DF80A1041EA02118DF80A1018E0E67444
:106E700005B0BDE8F08F0021DFF8448318F801B0B9
:106E800003F801B0491CC9B21229F7D3D4E79DF821
:106E90000A10C7F107031A4441EA02118DF80A10DB
:106EA00009EB0001002291F8F830DFEDC60A9FEDF2
:106EB000C60A012B0DD0022B37D0BC4A4FF0090E69
:106EC000032B92F83470117B52895BD0042B78D05D
:106ED000F1E059F820108DF80710C1F3012343EABF
:106EE00081038DF808309DF80930C1F383173B43C7
:106EF0008DF8093084F834202672C1F3892201EE1E
:106F0000102AB8EE411A61EE200AFCEEE00A10EEFB
:106F1000902A2270C1F3090100EE901AF8EE600A7F
:106F200020EE800A84ED010AC5E059F820108DF8A2
:106F30000710C1F3012343EA81038DF808309DF85F
:106F40000930C1F383173B438DF8093084F83420AE
:106F500003222272C1F3892201EE102AB8EE411AEF
:106F600061EE200AFCEEE00A10EE902A2270C1F3D6
:106F7000090100EE901AF8EE600A20EE800A84ED16
:106F8000010A98E059F82080C8F3484303EB8303D3
:106F9000A382C8F3072C0CEB8C0CA4F816C008F0E5
:106FA000FF0884F80D804FF0020B84F808B027B971
:106FB00084F83460854F87F800E09A4202D96381F3
:106FC00003E01CE00AB9FA2262816289624501D2BB
:106FD000A4F80AC0414500D809B984F80C80217B87
:106FE0008DF8071061894A008DF808209DF8092066
:106FF00042EAD1118DF80910296821625BE059F845
:107000002030C3F3484C4FEA8C0CA4F814C0C3F3EF
:1070100007284FEA8808A4F81680637304232372B4
:1070200027B984F83460694B83F800E0624501D9E0
:10703000A4F80AC06289424501D2A4F80A80628994
:1070400002F00303D21A92B2628101EE102A99ED86
:107050003D0AF8EE411A9FED5E1A5E4F21EE812A3D
:10706000C0EE021A11EE903ABB4202DD6423637354
:107070000EE001EE902AF8EE611A61EE811A80EEC0
:10708000211A81EE200ABCEEC00A10EE103A63739A
:10709000637B994200D801B92373217B8DF80710D7
:1070A00051008DF808109DF8091041EAD2118DF8B1
:1070B0000910296821625146DFF81C81DFF81CA104
:1070C000474F42F20F7B012930D00E21684600F075
:1070D00015FD08F003FD3888E02200EB400108F8B8
:1070E00021209DF805209DF8063008EB810102EB78
:1070F00003224A809DF807209DF80A309DF808C0B9
:1071000002EB03629DF809301B0403EB0C231A44C5
:107110004A60584501D2401C3880DAF80000401C13
:10712000CAF80000A67428682063A1E659F8200078
:10713000010E8DF80E10010C8DF80D10010A8DF85E
:107140000C108DF80B00286860621221684600F070
:10715000D5FC08F0C3FC3888E02200EB400108F8B9
:1071600021209DF805209DF8063008EB810102EBF7
:1071700003224A809DF807209DF80A309DF808C038
:1071800002EB03629DF809301B0403EB0C231A4445
:107190004A60584501D2401C3880DAF80000401C93
:1071A000CAF80000BEE7000068B8FF1FC8B6FF1F9E
:1071B0007C83FF1F2083FF1FA8CC0120A8A0020012
:1071C00000A30200CDCC4C3D0AD7233CB183FF1F66
:1071D000CDCCCC3C0000A04074B9FF1F7883FF1FCA
:1071E0007083FF1F2DE9F04389B000208B4901AA6D
:1071F0000B5C1354401CC0B21E28F9D39DF80A0042
:1072000000F0F10086490A7940EA42008DF80A0050
:107210009DF80900897840EA81108DF80900814CB9
:107220009DF81B0021790843617840EA41108DF8F0
:107230001B009DF81C00217840EA4100A17840EA3B
:1072400041108DF81C009DF81D00E17840EA4100D6
:107250008DF81D006279213C00201721062A41D2B9
:10726000DFE802F040030F1C2A37EF208DF80F00F3
:107270008DF81010AA208DF81900A4208DF81A009E
:1072800030E087208DF80F002E208DF810004E2062
:107290008DF8190042208DF81A0023E0E1218DF8C5
:1072A0001E1095218DF80F102D218DF810108DF8DE
:1072B00019008DF81A0015E022208DF80F00D92052
:1072C0008DF8100096208DF8190011208DF81A0005
:1072D00008E08DF80F1027218DF810108DF8190097
:1072E0008DF81A0094F8270028B19DF8120040F09C
:1072F00004008DF812001E2101A800F0FFFB08F029
:10730000F9FBDFF824C1494AC023BCF8001001EBA7
:10731000410002F820309DF809309DF80A5002EB38
:10732000800003EB052343809DF80B009DF80E20A1
:107330009DF80C3000EB02609DF80D20120402EB6A
:10734000032200EB02083A48C0F800809DF80F20A5
:107350009DF812309DF8105002EB03629DF8113039
:107360001B0403EB0523134443609DF813209DF891
:1073700016509DF8146002EB05629DF815502D041F
:1073800005EB0625561986609DF817209DF81A50C2
:107390009DF8187002EB05629DF819502D0405EB5D
:1073A00007251544C5609DF81B209DF81E709DF8AB
:1073B0001C9002EB07629DF81D703F0407EB092744
:1073C0001744076194F82720012A02D0022A03D02B
:1073D00004E00322C27701E00422C277154C228820
:1073E000B2F5FA7F0BD2144800EB4210C0F80480CB
:1073F0008360C660056147610180521C228042F2B1
:107400000F70814202D2491CACF800100B48016891
:10741000491C016009B0BDE8F0830000CAA0020069
:107420002083FF1F196302207083FF1F74B9FF1FA1
:10743000A8CC01207283FF1F288E01207883FF1FB4
:1074400070B586B0002027496A460B5C1354401C77
:10745000C0B21628F9D39DF8060000F0F1002249C9
:107460000A7940EA42008DF806009DF80500897807
:1074700040EA81108DF805001621684600F03EFBB9
:1074800008F038FB194D1A4AC023288800EB400148
:1074900002F821309DF805309DF8064002EB81018D
:1074A00003EB04234B80134C2288B2F5FA7F0CD2F5
:1074B000114B124901EB42111E684E605E688E60EE
:1074C0009B68CB600880521C228042F20F71884278
:1074D00001D2401C28800A480168491C016006B09E
:1074E00070BD0000E8A002002083FF1F7083FF1F13
:1074F00074B9FF1F7283FF1FA8CC0120288E0120C2
:107500007883FF1F70B586B00020304901AA0B5C5C
:107510001354401CC0B21228F9D39DF80A0000F0A1
:10752000F1002B490A7940EA42008DF80A009DF8E3
:107530000900897840EA81108DF80900254890F803
:107540002700012802D0022807D00CE09DF8110086
:1075500040F003008DF8110005E09DF8110040F0A7
:107560000B008DF81100122101A800F0C7FA08F0F5
:10757000C1FA194B194AC024188800EB400102F8DF
:1075800021409DF809409DF80A5002EB810104EB6F
:1075900005244C80124C2188B1F5FA7F0AD2114D96
:1075A000114A02EB41122E6856606D68956010809A
:1075B000491C218042F20F71884201D2401C188080
:1075C0000A480168491C016006B070BDFEA00200B7
:1075D0002083FF1FF86202207083FF1F74B9FF1F12
:1075E0007283FF1FA8CC0120288E01207883FF1F03
:1075F00070B588B0002029496A460B5C1354401CC2
:10760000C0B21E28F9D39DF8060000F0F10024490D
:107610000A7940EA42008DF806009DF80500897855
:1076200040EA81108DF805001E21684600F066FAD8
:1076300008F060FA1B4D1C4AC023298801EB410069
:1076400002F820309DF805309DF8064002EB8000DE
:1076500003EB04234380154C2388B3F5FA7F10D243
:10766000134A144800EB431016684660566886605B
:107670009668C660D66806611269426101805B1C2B
:10768000238042F20F70814201D2491C29800A48AE
:107690000168491C016008B070BD000010A1020023
:1076A0002083FF1F7083FF1F74B9FF1F7283FF1FAA
:1076B000A8CC0120288E01207883FF1F70B588B0E8
:1076C000002029496A460B5C1354401CC0B21E2896
:1076D000F9D39DF8060000F0F10024490A7940EA48
:1076E00042008DF806009DF80500897840EA811077
:1076F0008DF805001E21684600F000FA08F0FAF93E
:107700001B4D1C4AC023298801EB410002F82030A0
:107710009DF805309DF8064002EB800003EB042342
:107720004380154C2388B3F5FA7F10D2134A1448CE
:1077300000EB431016684660566886609668C6601F
:10774000D66806611269426101805B1C238042F2A7
:107750000F70814201D2491C29800A480168491CE6
:10776000016008B070BD00002EA102002083FF1F41
:107770007083FF1F74B9FF1F7283FF1FA8CC012005
:10778000288E01207883FF1F3EB500201C496A46E1
:107790000B5C1354401C0A28FADB9DF8060000F02D
:1077A000F1001849CA7840EA42008DF806009DF8B9
:1077B0000500897840EA81108DF805000A216846A5
:1077C00000F09CF908F08AF90F4A104BE024108869
:1077D00000EB400103F821409DF805409DF806505C
:1077E00003EB810104EB05244C8042F20F718842C7
:1077F00001D2401C108006480168491C01603EBD52
:10780000BEA202002083FF1F7083FF1F74B9FF1FF9
:107810007883FF1F3EB500201C496A460B5C135459
:10782000401C0A28FADB9DF8060000F0F100184918
:10783000CA7840EA42008DF806009DF80500897874
:1078400040EA81108DF805000A21684600F056F9DB
:1078500008F044F90F4A104BE024108800EB400177
:1078600003F821409DF805409DF8065003EB810187
:1078700004EB05244C8042F20F71884201D2401C77
:10788000108006480168491C01603EBD4CA1020001
:107890002083FF1F7083FF1F74B9FF1F7883FF1FB2
:1078A0007FB50021324A6B46545C5C54491C0E295A
:1078B000FADB9DF8061001F0F1012E4AD37841EA77
:1078C00043018DF806109DF80510927841EA821167
:1078D0008DF805108021012802D002280CD015E077
:1078E00002208DF807008DF8081000208DF809009F
:1078F000FF208DF80A0009E003208DF807008DF8BD
:10790000081087208DF809008DF80A100E216846AE
:1079100000F0F4F808F0E2F8174A184BC024108879
:1079200000EB400103F821409DF805409DF806500A
:1079300003EB810104EB05244C809DF807309DF892
:107940000A409DF8085003EB04639DF809402404A5
:1079500004EB052423444B6042F20F71884201D2AC
:10796000401C108006480168491C01607FBD000072
:1079700060A102002083FF1F7083FF1F74B9FF1FE7
:107980007883FF1FF0B585B0002032496A460B5C52
:107990001354401C1228FADB9DF8060000F0F10099
:1079A0002D49CA7840EA42008DF806009DF805008E
:1079B000897840EA81108DF805001221684600F0B0
:1079C0009DF808F08BF8254B254AE024188800EB39
:1079D000400102F821409DF805409DF8065002EB59
:1079E000810104EB05244C801E4C2188B1F5FA7FFF
:1079F00023D29DF807209DF80A509DF8086002EBFD
:107A000005629DF809502D0405EB06251544164A1C
:107A100002EB411255609DF80B509DF80E609DF8E9
:107A20000C7005EB06659DF80D60360406EB072625
:107A3000354495601080491C218042F20F718842C4
:107A400001D2401C188009480168491C016005B03A
:107A5000F0BD0000C8A202002083FF1F7083FF1F3B
:107A600074B9FF1F7283FF1F288E01207883FF1FC8
:107A70003EB500201C496A460B5C1354401C0A2882
:107A8000FADB9DF8060000F0F1001849CA7840EAD8
:107A900042008DF806009DF80500897840EA8110C3
:107AA0008DF805000A21684600F028F808F016F85D
:107AB0000F4A104BE024108800EB400103F82140EE
:107AC0009DF805409DF8065003EB810104EB052469
:107AD0004C8042F20F71884201D2401C108006484F
:107AE0000168491C01603EBD56A102002083FF1FB2
:107AF0007083FF1F74B9FF1F7883FF1F38B50446DA
:107B00000D464320009072B6222001F079FA38B970
:107B10000121684601F0EAF92946204601F0E6F91C
:107B200001F08CFA62B638BD08B58DF800008DF80A
:107B30000110222001F064FA18B105490020887173
:107B400008BD0221684601F0D1F901F077FA08BDBD
:107B50002083FF1F38B53E4800903E483E490068EC
:107B60000860401C00D1086000203C4C810101F5F8
:107B7000FC210978A02937D0401CC0B27F28F5D35A
:107B80001E20E41D04F8030C072004F8040C052053
:107B900060700321A1760220E076012020776077D3
:107BA000A177E0774FF64D31282000F0C3F840F27E
:107BB00079612A2000F0BEF84DF69A312C2000F0B1
:107BC000B9F8B1EE040A092000F0BEF8B1EE040ADB
:107BD0000D2000F0B9F8B7EE000A1D2000F0B4F84F
:107BE000BDE8384000F066B84FF4FC2101EB80118D
:107BF00040221A48F8F7CEFB607800B101201849FE
:107C00000870112000F046F8164880ED000A152093
:107C100000F040F8144880ED000A1D2000F03AF80A
:107C2000124880ED000A282000F028F800280ED025
:107C3000282000F023F80E4908802A2000F01EF8C2
:107C40000C4908802C2000F019F80B49088038BD39
:107C500053AE0043080C0003D890FF1FF8620220C7
:107C6000A683FF1FD88EFF1FDC8EFF1F4883FF1FD8
:107C7000A883FF1FAA83FF1FAC83FF1F08B5002145
:107C800000910349084400880090BDF8000008BD39
:107C9000F862022008B59FED050A8DED000A04493F
:107CA0000844006800909DED000A08BD0000000037
:107CB000F86202202DE9F04100241D4FA0264FF468
:107CC000FC25A10101F5FC210878FF280ED0641CD9
:107CD000E4B27F2CF5D3284600F042F83E702846E7
:107CE000BDE8F04140221249F8F719BF3E7005EB9C
:107CF000841040220E49F8F712FF002C15D0601EA8
:107D0000810101F5FC210978A02907D0A41E05EB0B
:107D10008410BDE8F041002100F039B805EB801077
:107D2000BDE8F041002100F032B8BDE8F08100006C
:107D3000F862022003B503490844BDF8041001802D
:107D40000CBD0000F862022001B52DED020B0249C6
:107D50000844009901600EBDF862022000F017B8D7
:107D600070B50546FDF73EFD0120FDF709FC4FF417
:107D700080742046FDF732FC0128FAD172B62846FD
:107D8000F8F7D2FE62B6BDE87040FDF75DBC70B595
:107D900005460E46FDF726FD0120FDF7F1FB4FF4E9
:107DA00080742046FDF71AFC0128FAD172B63146DC
:107DB0002846FDF7ABFC62B6BDE87040FDF744BC59
:107DC00010B586B004466846FDF74AFC9DE80700FA
:107DD00003AB07C3012C0DD0022C0DD0032C0DD00A
:107DE0000398049980B289B20844059900EB0140D8
:107DF00006B010BD0398FBE70498F9E70598F7E78C
:107E00000EB509293BD2DFE801F0050B11171D2340
:107E1000292F350002461CA168460DF0E1F82EE03E
:107E200002461AA168460DF0DBF828E0024619A1C7
:107E300068460DF0D5F822E0024618A168460DF01C
:107E4000CFF81CE0024617A168460DF0C9F816E00D
:107E5000024616A168460DF0C3F810E0024615A1CF
:107E600068460DF0BDF80AE0024614A168460DF020
:107E7000B7F804E0024613A168460DF0B1F8684671
:107E800000F024F80EBD00002558000025303158C0
:107E90000000000025303258000000002530335823
:107EA000000000002530345800000000253035580F
:107EB00000000000253036580000000025303758FB
:107EC0000000000025303858000000002DE9F04780
:107ED0000023544D544E554FDFF85481DFF854C100
:107EE0009AE07E2925D94FF08C09427802EB0121D6
:107EF0008AB2002114E035F831A092450ED805EB86
:107F0000C10ABAF802A0924508D335F8314005EB12
:107F1000C101121B898811448CB203E0491C89B24B
:107F20004945E8D3801C444931F8341019448BB2D8
:107F300072E098F80120102A06D01C2A27D00C2ABB
:107F400048D00020BDE8F0874FF01109002214E06E
:107F500036F832A051450ED306EBC20ABAF802A099
:107F6000514508D836F8324006EBC202091B928808
:107F700011448CB203E0521C92B24A45E8D3401C33
:107F80002949883131F8341019448BB244E04FF05C
:107F90000409002214E037F832A051450ED307EB54
:107FA000C20ABAF802A0514508D837F8324007EBA8
:107FB000C202091B928811448CB203E0521C92B297
:107FC0004A45E8D3401C1949203131F8341019448E
:107FD0008BB221E04FF00909002214E03CF832A0F6
:107FE00051450ED30CEBC20ABAF802A0514508D88D
:107FF0003CF832400CEBC202091B928811448CB24F
:1080000003E0521C92B24A45E8D3401C094948316A
:1080100031F8341019448BB2017800297FF461AF34
:1080200018468FE7C0DC020038B802003CA302000B
:108030009C83FF1F7846030020E102002DE9F843EE
:108040006B4800906B4C6C4800996C4E084483E080
:10805000217800297FD022781346082502E05B08AA
:108060006D1EEDB2DF07FAD0F82A22D008DC802A94
:1080700027D0C02A23D0E02A1FD0F02A06D11AE048
:10808000FC2A14D0FE2A10D0FF2A0CD000225A4B12
:10809000009F08333B449C421DD31846231A12D03C
:1080A000012B4FD112E0FE22F1E7FC22EFE7F8228C
:1080B000EDE7F022EBE7E022E9E7C022E7E78022E4
:1080C000E5E70022E3E74E4911433BE06FF47F41CF
:1080D00041EA022136E0484B009F1B1D3B444FF014
:1080E000FF0C4FF6FF776FF07F489C4214D3184681
:1080F000231A06D0012B06D0022B07D0032B21D147
:1081000007E011461EE04CEA02211BE007EB0241AA
:1081100018E048EA026115E0844213D3231A06D01E
:10812000012B06D0022B08D0032B0BD108E01146FF
:1081300008E04CEA022105E00DE007EB024101E016
:1081400048EA0261FFF70AFE0098201A133005EB97
:10815000C000B07003E0641E8442BFF479AFB07811
:108160000324B8B327480179427901EB02218279CF
:10817000C079120402EB0060084430610020FFF770
:108180001FFE00F0070120FA01F2884010441E494A
:10819000884203D91D490844400803E01B4949426D
:1081A0000844400031690125814216D1124A0098E5
:1081B000383A1044FFF7D2FD154900980844316958
:1081C000D0F8B50D884206D112480570124900203A
:1081D000087006E003E0F47003E0F57001E00220AF
:1081E000F07020467471BDE8F84300F015B9000046
:1081F00053AE0043490C0003ED5DFFBFB882FF1F83
:108200000000FFFF3865022033DDD35334DDD3D3C4
:108210000050FFBFD483FF1FB183FF1F0449052215
:108220000A7011224A7009228A70C87070470000D3
:108230007865022010B5094CE079032809D86079E7
:1082400000F0EAF8E079401CE071054800686061E0
:1082500010BD0020A071E07110BD0000B882FF1FAA
:108260007C83FF1F00200321044A535C1844C0B2E2
:10827000491CC9B23F29F8D3704700003865022075
:1082800006480178052905D14178112902D1817864
:10829000092901D000207047C07870473865022056
:1082A0002DE9F041594C0027A771A07A0125584EBD
:1082B000002802D0FFF7E4FF98B1FFF7D3FF96F84C
:1082C0003F1088427ED1FFF7DBFF69287FD02BDC8F
:1082D000652848D023DC78B3012875D0642830D1D4
:1082E0003BE0E089217A884203D9F420607100F0F4
:1082F00093F80020474BE289315CA7890F44A7819E
:1083000000EB8217D955401CC0B24028F4D3521C50
:10831000E28128466571BDE8F04100F07DB867282C
:108320003BD068280DD12BE0F1285ED005DC6A280F
:1083300053D0F02805D154E009E0F22859D0FF28A5
:1083400061D0F1206071BDE8F04100F065B8F02027
:108350006071BDE8F04100F05FB838466771BDE874
:10836000F04100F059B8A781E78130792072707927
:1083700060722846A5726071BDE8F04100F04CB80B
:10838000A781E78130792072707960722846A572E2
:108390006071BDE8F04100F03FB8A772A089317963
:1083A000C2B2914209D17179B1EB102F05D10220EF
:1083B0006071BDE8F04100F02FB8F3206071BDE8B6
:1083C000F04102E019E002E01DE000F025B8284687
:1083D0006571BDE8F04100F01FB8BDE8F041FFF75E
:1083E0002DBEBDE8F041FFF725BFBDE8F041FFF726
:1083F00021BFBDE8F041FFF71DBFF2206071BDE86D
:10840000F04100F009B8BDE8F0810000B882FF1F1C
:1084100038650220C491FF1F10B50446402125484D
:10842000F7F7D1FFF12C27D00BDC022C1CD003DC9A
:1084300084B1012C33D110E0032C12D0F02C2ED1BA
:1084400016E0F22C1CD0F32C1ED0F42C20D0FF2CE4
:1084500025D121E000F034F821E0012000F064F89B
:108460001DE000F083F81AE0022000F05DF816E04D
:10847000F02000F059F812E0F12000F055F80EE07D
:10848000F22000F051F80AE0F32000F04DF806E089
:10849000F42000F049F802E0FF2000F045F8012C3C
:1084A00007D0FF2C05D00448016804484161012130
:1084B000817110BD786502207C83FF1FB882FF1F89
:1084C00070B5154D2878002825D0144890F8DC00A8
:1084D000032820D10020FFF773FC03460020FFF79C
:1084E0009DFE0F4C012020716371180AA071180CB9
:1084F000E071180E20720B4800786072CB20A072D9
:1085000000F062F884F83F0040222146034811F051
:108510002DFD0020287070BDB882FF1FC4B1FF1F61
:1085200078650220D483FF1F70B504460C4D29786E
:10853000002914D00B4991F8DC1003290FD1002039
:10854000FFF73EFC2046FFF769FE074880F83F40F2
:1085500001464022034811F009FD0020287070BD3B
:10856000B882FF1FC4B1FF1F7865022070B5124C9E
:10857000207800281FD0114890F8DC0003281AD179
:108580000020FFF71DFC0320FFF748FE0C4803788E
:108590000C480371A1784171E2788271C578114469
:1085A0002B44194480F83F1001464022034811F043
:1085B000DDFC0020207070BDB882FF1FC4B1FF1F1A
:1085C000D483FF1F7865022000200321044A535CF6
:1085D0001844C0B2491CC9B23F29F8D37047000003
:1085E0007865022010B5134C2078002820D012485E
:1085F00090F8DC0003281BD10020FFF7E1FB0346C5
:108600000020FFF70BFE0D49012008714B71180A7D
:108610008871180CC871180E0872094800784872E1
:10862000C92088724022044811F0A0FC002020706C
:1086300010BD0000B882FF1FC4B1FF1F7865022083
:10864000D483FF1F70B51C481C4D1D4C90F833009F
:10865000002824D02868B0F57A7F20D94FF4007123
:10866000002007F03FFB012819D1607838B9154B7D
:10867000154A164916480FF045FD01206070207913
:1086800001280CD1124890F8DC00032807D1002003
:10869000207100231A4681210D480FF0B5FEA07904
:1086A000002808D028686169401A642803D9BDE809
:1086B0007040FFF7BFBD70BDF86202207C83FF1FD2
:1086C000B882FF1F0483FF1F9091FF1FD082FF1FFE
:1086D000C4B1FF1F10B5AFF3008010BD70B50446E4
:1086E0000D460D4884420AD00C48844207D00C48FD
:1086F000844204D04FF457710AA0FCF769FE35B1EB
:10870000012D04D040F25D3106A0FCF761FE206827
:1087100065F38A20206070BD00E0044000E404405E
:1087200000E804402E2E5C2E2E5C2E2E5C2E2E5C3D
:108730002E2E5C6472697665725C7372635C68632A
:108740003332663436305F6932632E6300000000D6
:108750002DE9F04704462DED028B0D46904600268C
:1087600000274FF002099FED648A002D45D0B8F133
:10877000000F42D0614884420AD06148844207D049
:108780006048844204D04FF496715FA0FCF720FE4D
:1087900068496868884204D940F22D115AA0FCF754
:1087A00017FE286890B1012810D002280ED00328A7
:1087B0000CD004280AD0052808D0062806D007289F
:1087C00004D04FF4977150A0FCF702FE5A48006A9B
:1087D000C0F3023159480068C8402A68012191401D
:1087E000D5ED020A95ED011A236BDB0603D5236B49
:1087F00003F003077F1C12B103E0042670E04FF082
:10880000030900EE100AB8EE412AB8EE400AC0EEA5
:10881000021A00EE101AB8EE402A81EE820A01EE2A
:10882000909AF8EE600AB8EE612AF0EE001A62EE55
:10883000212A02EE107AB8EE422A42EE212A32EEC6
:10884000A02A70EE421AFCEEC00AF8EE602A30EE62
:10885000620A10EE103AB3F17C5F06DBB8EE600AF4
:10886000F7EE000A30EE200A01E0B8EE600AB4EE3E
:10887000C20AF1EE10FA01D8042631E011EE903A66
:108880002F4DAB4201DD04262AE0BCEEC00A10EEFB
:10889000103AB0FBF3F0B0FBF1F000EE100AF8EE86
:1088A000410AB8EE400A70EEC00A00EE100AB8EEB7
:1088B000400A80EE808AE06A62F31240E062BCEE19
:1088C000E10A10EE100A4108E06A61F30400E06278
:1088D00010EE100AA0EB5001E06A61F30C20E06298
:1088E000B8F1000F02D00EB988ED008A3046BDEC19
:1088F000028BBDE8F08700000000000000E00440AB
:1089000000E4044000E804402E2E5C2E2E5C2E2E47
:108910005C2E2E5C2E2E5C6472697665725C7372BE
:10892000635C68633332663436305F6932632E636A
:1089300000000000801A060000400540B482FF1FBE
:108940000000784270B504460D460A4884420AD0B9
:108950000948844207D00948844204D040F2F521F6
:1089600007A0FCF735FD206A10490D40284320621E
:1089700070BD000000E0044000E4044000E8044052
:108980002E2E5C2E2E5C2E2E5C2E2E5C2E2E5C64EB
:1089900072697665725C7372635C686333326634E5
:1089A00036305F6932632E6300000000DF56F0004E
:1089B00070B504460D460D4884420AD00C488442E6
:1089C00007D00C48844204D040F2FF110AA0FCF703
:1089D000FFFC35B1012D04D04FF4007106A0FCF767
:1089E000F7FC206865F30000206070BD00E00440E3
:1089F00000E4044000E804402E2E5C2E2E5C2E2E57
:108A00005C2E2E5C2E2E5C6472697665725C7372CD
:108A1000635C68633332663436305F6932632E6379
:108A2000000000001FB5002331224FF40041012057
:108A300007F0FAFA002330224FF48041012007F0BA
:108A4000F3FA0121402007F007FE0A4C204600F00F
:108A500015F8002101910391074902916A4601A985
:108A6000204600F019F901212046FFF7A1FF04B0CC
:108A7000284610BD00E80440801A060010B50446E0
:108A80000B4884420AD00B48844207D00A488442EB
:108A900004D04FF4BD7109A0FCF79AFC206820F0C7
:108AA00001002060206840F400402060002010BDDC
:108AB00000E0044000E4044000E804402E2E5C2E58
:108AC0002E5C2E2E5C2E2E5C2E2E5C6472697665DA
:108AD000725C7372635C68633332663436305F692C
:108AE00032632E630000000070B504460D460C484A
:108AF000844209D00B48844206D00B48844203D0FC
:108B0000D5210AA0FCF764FC2DB1012D03D0D6219C
:108B100006A0FCF75DFC206865F30820206070BDAE
:108B200000E0044000E4044000E804402E2E5C2EE7
:108B30002E5C2E2E5C2E2E5C2E2E5C647269766569
:108B4000725C7372635C68633332663436305F69BB
:108B500032632E630000000070B504460D460C48D9
:108B6000844209D00B48844206D00B48844203D08B
:108B7000F8210AA0FCF72CFC2DB1012D03D0F9211E
:108B800006A0FCF725FC206865F34920206070BD35
:108B900000E0044000E4044000E804402E2E5C2E77
:108BA0002E5C2E2E5C2E2E5C2E2E5C6472697665F9
:108BB000725C7372635C68633332663436305F694B
:108BC00032632E630000000070B505460C46002697
:108BD000234885420AD02348854207D0224885424F
:108BE00004D040F2CD2121A0FCF7F2FB012C31D0C2
:108BF000022C2FD0042C2DD0082C2BD0102C29D0B7
:108C0000402C27D0802C25D0B4F5007F22D0B4F59D
:108C1000806F1FD0B4F5805F1CD0B4F5804F19D0A1
:108C2000B4F5803F16D0B4F5003F13D0B4F5802FD3
:108C300010D0B4F5801F0DD0B4F5001F0AD0B4F5E4
:108C4000800F07D0B4F5000F04D040F2CE2107A06A
:108C5000FCF7BEFBE869204200D00126304670BD1B
:108C600000E0044000E4044000E804402E2E5C2EA6
:108C70002E5C2E2E5C2E2E5C2E2E5C647269766528
:108C8000725C7372635C68633332663436305F697A
:108C900032632E630000000070B504460D46164690
:108CA000002D4BD0002C49D0254884420AD02548BD
:108CB000844207D02448844204D040F2A31123A068
:108CC000FCF786FB2C496868884204D94FF4D271BE
:108CD0001EA0FCF77DFB286890B1012810D0022867
:108CE0000ED003280CD004280AD0052808D0062866
:108CF00006D0072804D040F2A51114A0FCF768FBA9
:108D0000206820F001002060206840F400402060CE
:108D1000206840F001002060324629462046FFF7D7
:108D200017FD216821F040012160216821F40041F4
:108D30002160216821F00101216070BD042070BD17
:108D400000E0044000E4044000E804402E2E5C2EC5
:108D50002E5C2E2E5C2E2E5C2E2E5C647269766547
:108D6000725C7372635C68633332663436305F6999
:108D700032632E6300000000801A060010B504461E
:108D8000084884420AD00848844207D007488442F1
:108D900004D040F24B3106A0FCF71AFB94F82800EF
:108DA00010BD000000E0044000E4044000E804407E
:108DB0002E2E5C2E2E5C2E2E5C2E2E5C2E2E5C64B7
:108DC00072697665725C7372635C686333326634B1
:108DD00036305F6932632E63000000002DE9F05FDA
:108DE00007460E4691464FF47A7AD0463E4D012111
:108DF000284600F085F80021284600F081F84FF45D
:108E0000003B07E0B8F1010804D200F017F9002098
:108E1000BDE8F09F59462846FFF7D6FE0128F1D05D
:108E200001212846FFF760FE5446D84641462846B1
:108E3000FFF7CAFE834601212846FFF7C5FEBBF1B6
:108E4000000F05D020B1012000EB4700C7B206E0BB
:108E5000641E601CEAD1DBE7641E601C0ED080211A
:108E60002846FFF7B1FE0028F6D02C4639462046AA
:108E700000F0F2F957464FF4806504E00020C7E7A0
:108E80007F1E781C0AD029462046FFF79DFE012848
:108E9000F6D00025A9F1010827461AE000F0CEF827
:108EA0000020B5E7454503D101213846FFF716FC00
:108EB000544602E0641E601C11D040213846FFF782
:108EC00083FE0028F6D03846FFF758FF06F8010B5E
:108ED0006D1C4D45E6D300F0B1F8012098E700F095
:108EE000ADF8002094E7000000E804400A4601467F
:108EF0004FF47A73014800F037B9000000E80440ED
:108F000070B504460D460D4884420AD00C48844290
:108F100007D00C48844204D040F205310AA0FCF787
:108F200057FA35B1012D04D040F2063106A0FCF706
:108F30004FFA206865F3CF30206070BD00E0044038
:108F400000E4044000E804402E2E5C2E2E5C2E2E01
:108F50005C2E2E5C2E2E5C6472697665725C737278
:108F6000635C68633332663436305F6932632E6324
:108F70000000000070B504460D46124884420AD035
:108F80001148844207D01148844204D040F28F3106
:108F90000FA0FCF71DFA2B4600224FF400312046AB
:108FA00000F046F900280BD101212046FFF79CFD77
:108FB0002B462046BDE870400122104900F038B928
:108FC00070BD000000E0044000E4044000E80440FC
:108FD0002E2E5C2E2E5C2E2E5C2E2E5C2E2E5C6495
:108FE00072697665725C7372635C6863333266348F
:108FF00036305F6932632E6300000000010002001A
:1090000070B506460C4C01212046FFF779FF002180
:109010002046FFF775FF4FF47A7529462046FFF783
:10902000A9FF002807D12B4631462046BDE87040F5
:10903000002200F02DB870BD00E804402DE9F04199
:109040004FF47A752C464FF40037104E02E0641E40
:10905000601C0BD039463046FFF7B6FD0028F6D02D
:10906000344601212046FFF777FD05E00020BDE8EA
:10907000F0816D1E681C07D010212046FFF7A4FD6B
:109080000028F6D00120F2E70020F0E700E80440D5
:109090002DE9F04106460F4615469846244886427B
:1090A0000AD02448864207D02348864204D040F2A2
:1090B000C93122A0FCF78CF97F2F04D940F2CA31C4
:1090C0001EA0FCF785F9012D05D025B140F2CB316A
:1090D0001AA0FCF77DF9434601228021304600F0BA
:1090E000A7F8044604BB45EA4700C1B2304600F089
:1090F000B3F84DB1434600224FF48021304600F0D2
:1091000097F8044644B10FE0434601220821304657
:1091100000F08EF80446F5E74FF480613046FFF723
:1091200053FD012800D101242046BDE8F081000054
:1091300000E0044000E4044000E804402E2E5C2ED1
:109140002E5C2E2E5C2E2E5C2E2E5C647269766553
:10915000725C7372635C68633332663436305F69A5
:1091600032632E63000000002DE9F84305460E46E9
:1091700017469946204885420AD02048854207D0A4
:109180001F48854204D040F24B411EA0FCF720F955
:1091900000240020009056B34FF480581CE04B464A
:1091A00001228021284600F043F80446A4B9009823
:1091B000315C284600F050F84B4601220821284631
:1091C00000F036F8044641462846FFF7FDFC01282A
:1091D00008D00098401C00900098B84208D0002C9D
:1091E000DDD005E041462846FFF7ACFB00E0042453
:1091F0002046BDE8F883000000E0044000E404409D
:1092000000E804402E2E5C2E2E5C2E2E5C2E2E5C52
:109210002E2E5C6472697665725C7372635C68633F
:109220003332663436305F6932632E6300000000EB
:1092300030B505460920EC690C40012A01D1A14254
:1092400001D0144300D10020002803D0002B01D00E
:109250005B1EF0E730BD000070B504460D460848BF
:1092600084420AD00748844207D00748844204D089
:1092700040F23D3105A0FCF7ABF884F8245070BDF6
:1092800000E0044000E4044000E804402E2E5C2E80
:109290002E5C2E2E5C2E2E5C2E2E5C647269766502
:1092A000725C7372635C68633332663436305F6954
:1092B00032632E630000000010B5042000F0CFF9E7
:1092C00001040FD5401EC04380B2F7F70FFA9FED9F
:1092D0000C1B53EC112BF7F728F9F7F771FA00EE96
:1092E000100A10BDF7F702FA9FED071B53EC112B84
:1092F000F7F71BF9F7F764FA00EE100A10BD00004B
:10930000FCA9F1D24D6240BFFCA9F1D24D62403FB1
:1093100010B5022000F0A3F9F7F7E8F99FED051B5F
:1093200053EC112BF7F701F9F7F74AFA00EE100AA0
:1093300010BD00007B14AE47E17A543F10B540EAFF
:109340000102072A1DD844F2070242EA402080B2F7
:1093500040EA811040EAC101002000F099F94FF481
:109360008061062000F094F94FF40061052000F0C0
:109370008FF90448006804494861BDE8104000F0D6
:109380000DB810BD7C83FF1F3083FF1F10B500F0A8
:1093900061F8BDE810400820FCF786BA70B586B0C9
:1093A00000240594039404940194029408268DF8F3
:1093B000146001258DF815508DF816508DF8174062
:1093C00005A8FCF719FA019402948DF804408DF871
:1093D00006508DF8085001AA2902002006F0E4FC8E
:1093E000ADF80C600320ADF80E001948049003A8F6
:1093F0000EF0DEFBBDF90E00002809DB00F01F01B6
:1094000005FA01F14009800000F1E020C0F8801267
:10941000BDF90E00F021002804DB00F1E02080F807
:10942000001405E000F00F0000F1E02080F8141DAA
:10943000BDF90E00002808DB00F01F018D40400937
:10944000800000F1E020C0F8005106B070BD0000BF
:109450008D93010070B5FFF75BFF744C84ED010A3A
:10946000FFF72AFF84ED020A00F0F6F894ED020AF5
:109470006F4910EE100A884202D80120207001E0E6
:109480000020207094ED020A10EE100AF7F754F94C
:1094900041EC100B0BF024FE51EC100BF7F790F998
:1094A00000EE100A84ED020A94ED020A614910EE02
:1094B000100A884204DD94ED020A84ED030A03E0F9
:1094C0009FED5D0A84ED030A94ED060AB5EEC00A2D
:1094D000F1EE10FA0ED094ED060A10EE100AB0F17B
:1094E0007E5F07D094ED030AD4ED060A20EE200A31
:1094F00084ED030A94ED010AD4ED030A20EE200A5C
:1095000084ED040A4D4D28686169D4ED040A401ABF
:1095100000EE100AB8EE400A60EE200A9FED481AED
:1095200080EE810A10EE100AF7F706F994ED081B99
:1095300053EC112BF6F752FF41EC100B84ED080BA6
:1095400094ED010A3F4A10EE100A90421DDC286893
:109550006169D4ED030A401A00EE100A9FED3A1A31
:10956000B8EE400A60EE200A80EE810A10EE100A82
:10957000F7F7E2F894ED0A1B53EC112BF6F72EFFE8
:1095800041EC100B84ED0A0B4DE094ED010A2F48DD
:1095900010EE101A914223DD94ED010A10EE101A1C
:1095A00081421DDC28686169D4ED030A401A00EE8F
:1095B000100A9FED271AB8EE400A60EE200A80EEEE
:1095C000810A10EE100AF7F7B7F894ED0A1B53EC76
:1095D000112BF6F703FF41EC100B84ED0A0B22E090
:1095E00094ED010A10EE101A81421CDD28686169B1
:1095F000D4ED030A401A00EE100A9FED161AB8EED9
:10960000400A60EE200A80EE810A10EE100AF7F799
:1096100093F894ED0A1B53EC112BF6F7DFFE41ECA7
:10962000100B84ED0A0B2868606170BD3083FF1F4A
:109630006F1203BBE71DA73B000000007C83FF1FE8
:1096400000BA5B4A0000C040000061450000404194
:109650000000E144000061440620AFF3008001B542
:1096600082B04020FFF7CCFC18B9012102A8FFF717
:109670003DFCFFF7E3FC022201A94020FFF7AEFB0F
:109680009DF805009DF8041000EB012080B20EBD8E
:1096900008B58DF80000080A8DF801008DF8021059
:1096A0004020FFF7ADFC18B105490020487008BD07
:1096B00003216846FFF71AFCFFF7C0FC08BD000055
:1096C0003083FF1F02480068002800D00047704721
:1096D0003863022002484068002800D000477047E5
:1096E0003863022002488068002800D00047704795
:1096F000386302200248C068002800D00047704745
:109700003863022002480069002800D000477047F3
:109710003863022002484069002800D000477047A3
:109720003863022002488069002800D00047704753
:10973000386302200248C069002800D00047704703
:10974000386302200248006A002800D000477047B2
:10975000386302200248406A002800D00047704762
:10976000386302200248806A002800D00047704712
:10977000386302200248C06A002800D000477047C2
:10978000386302200248006B002800D00047704771
:10979000386302200248406B002800D00047704721
:1097A000386302200248806B002800D000477047D1
:1097B000386302200248C06B002800D00047704781
:1097C000386302200248006C002800D00047704730
:1097D000386302200248406C002800D000477047E0
:1097E000386302200248806C002800D00047704790
:1097F000386302200248C06C002800D00047704740
:10980000386302200248006D002800D000477047EE
:10981000386302200248406D002800D0004770479E
:10982000386302200248806D002800D0004770474E
:10983000386302200248C06D002800D000477047FE
:10984000386302200248006E002800D000477047AD
:10985000386302200248406E002800D0004770475D
:10986000386302200248806E002800D0004770470D
:10987000386302200248C06E002800D000477047BD
:10988000386302200248006F002800D0004770476C
:10989000386302200248406F002800D0004770471C
:1098A000386302200248806F002800D000477047CC
:1098B000386302200248C06F002800D0004770477C
:1098C000386302200348D0F88000002800D0004709
:1098D00070470000386302200348D0F88400002855
:1098E00000D0004770470000386302200348D0F8DA
:1098F0008800002800D0004770470000386302202D
:109900000348D0F88C00002800D0004770470000C2
:10991000386302200348D0F89000002800D00047A8
:1099200070470000386302200348D0F894000028F4
:1099300000D0004770470000386302200348D0F889
:109940009800002800D000477047000038630220CC
:109950000348D0F89C00002800D000477047000062
:10996000386302200348D0F8A000002800D0004748
:1099700070470000386302200348D0F8A400002894
:1099800000D0004770470000386302200348D0F839
:10999000A800002800D0004770470000386302206C
:1099A0000348D0F8AC00002800D000477047000002
:1099B000386302200348D0F8B000002800D00047E8
:1099C00070470000386302200348D0F8B400002834
:1099D00000D0004770470000386302200348D0F8E9
:1099E000B800002800D0004770470000386302200C
:1099F0000348D0F8BC00002800D0004770470000A2
:109A0000386302200348D0F8C000002800D0004787
:109A100070470000386302200348D0F8C4000028D3
:109A200000D0004770470000386302200348D0F898
:109A3000C800002800D000477047000038630220AB
:109A40000348D0F8CC00002800D000477047000041
:109A5000386302200348D0F8D000002800D0004727
:109A600070470000386302200348D0F8D400002873
:109A700000D0004770470000386302200348D0F848
:109A8000D800002800D0004770470000386302204B
:109A90000348D0F8DC00002800D0004770470000E1
:109AA000386302200348D0F8E000002800D00047C7
:109AB00070470000386302200348D0F8E400002813
:109AC00000D0004770470000386302200348D0F8F8
:109AD000E800002800D000477047000038630220EB
:109AE0000348D0F8EC00002800D000477047000081
:109AF000386302200348D0F8F000002800D0004767
:109B000070470000386302200348D0F8F4000028B2
:109B100000D0004770470000386302200348D0F8A7
:109B2000F800002800D0004770470000386302208A
:109B30000348D0F8FC00002800D000477047000020
:109B4000386302200348D0F80001002800D0004705
:109B500070470000386302200348D0F80401002851
:109B600000D0004770470000386302200348D0F857
:109B70000801002800D00047704700003863022029
:109B80000348D0F80C01002800D0004770470000BF
:109B9000386302200348D0F81001002800D00047A5
:109BA00070470000386302200348D0F814010028F1
:109BB00000D0004770470000386302200348D0F807
:109BC0001801002800D000477047000038630220C9
:109BD0000348D0F81C01002800D00047704700005F
:109BE000386302200348D0F82001002800D0004745
:109BF00070470000386302200348D0F82401002891
:109C000000D0004770470000386302200348D0F8B6
:109C10002801002800D00047704700003863022068
:109C20000348D0F82C01002800D0004770470000FE
:109C3000386302200348D0F83001002800D00047E4
:109C400070470000386302200348D0F83401002830
:109C500000D0004770470000386302200348D0F866
:109C60003801002800D00047704700003863022008
:109C70000348D0F83C01002800D00047704700009E
:109C8000386302200348D0F84001002800D0004784
:109C900070470000386302200348D0F844010028D0
:109CA00000D0004770470000386302200348D0F816
:109CB0004801002800D000477047000038630220A8
:109CC0000348D0F84C01002800D00047704700003E
:109CD000386302200348D0F85001002800D0004724
:109CE00070470000386302200348D0F85401002870
:109CF00000D0004770470000386302200348D0F8C6
:109D00005801002800D00047704700003863022047
:109D10000348D0F85C01002800D0004770470000DD
:109D2000386302200348D0F86001002800D00047C3
:109D300070470000386302200348D0F8640100280F
:109D400000D0004770470000386302200348D0F875
:109D50006801002800D000477047000038630220E7
:109D60000348D0F86C01002800D00047704700007D
:109D7000386302200348D0F87001002800D0004763
:109D800070470000386302200348D0F874010028AF
:109D900000D0004770470000386302200348D0F825
:109DA0007801002800D00047704700003863022087
:109DB0000348D0F87C01002800D00047704700001D
:109DC000386302200348D0F88001002800D0004703
:109DD00070470000386302200348D0F8840100284F
:109DE00000D0004770470000386302200348D0F8D5
:109DF0008801002800D00047704700003863022027
:109E00000348D0F88C01002800D0004770470000BC
:109E1000386302200348D0F89001002800D00047A2
:109E200070470000386302200348D0F894010028EE
:109E300000D0004770470000386302200348D0F884
:109E40009801002800D000477047000038630220C6
:109E50000348D0F89C01002800D00047704700005C
:109E6000386302200348D0F8A001002800D0004742
:109E700070470000386302200348D0F8A40100288E
:109E800000D0004770470000386302200348D0F834
:109E9000A801002800D00047704700003863022066
:109EA0000348D0F8AC01002800D0004770470000FC
:109EB000386302200348D0F8B001002800D00047E2
:109EC00070470000386302200348D0F8B40100282E
:109ED00000D0004770470000386302200348D0F8E4
:109EE000B801002800D00047704700003863022006
:109EF0000348D0F8BC01002800D00047704700009C
:109F0000386302200348D0F8C001002800D0004781
:109F100070470000386302200348D0F8C4010028CD
:109F200000D0004770470000386302200348D0F893
:109F3000C801002800D000477047000038630220A5
:109F40000348D0F8CC01002800D00047704700003B
:109F5000386302200348D0F8D001002800D0004721
:109F600070470000386302200348D0F8D40100286D
:109F700000D0004770470000386302200348D0F843
:109F8000D801002800D00047704700003863022045
:109F90000348D0F8DC01002800D0004770470000DB
:109FA000386302200348D0F8E001002800D00047C1
:109FB00070470000386302200348D0F8E40100280D
:109FC00000D0004770470000386302200348D0F8F3
:109FD000E801002800D000477047000038630220E5
:109FE0000348D0F8EC01002800D00047704700007B
:109FF000386302200348D0F8F001002800D0004761
:10A0000070470000386302200348D0F8F4010028AC
:10A0100000D0004770470000386302200348D0F8A2
:10A02000F801002800D00047704700003863022084
:10A030000348D0F8FC01002800D00047704700001A
:10A04000386302202DE9FE4F00260321DC22D24F87
:10A05000DFF84893DFF848A3D24DD34C47F6EF33EF
:10A060004FF448784FF07C5B092824D2DFE800F0F9
:10A070002305254497C6FCEEED00CDE901320091A1
:10A0800030237F2210210F20F7F78AFF202135206F
:10A09000F8F75EFF1020F8F761FF3888F8F764FFE3
:10A0A000C2A0F8F78FF82868A16B401A404502D982
:10A0B000112060702670BDE8FE8FCDE9013200915D
:10A0C0003023822210210F20F7F76AFF202132204F
:10A0D000F8F73EFF1020F8F741FF3888F8F744FF03
:10A0E000B5A0F8F76FF82868A16B401A4045E2D98F
:10A0F0001E2060702670DEE7CDE90132009130232A
:10A10000822210210F20F7F74BFF1020F8F726FFCF
:10A11000AC480088F8F728FF10210F20F8F718FF47
:10A12000A948007868B9A9A0F8F7C4FB0021042069
:10A13000F7F7C2FEA7A0F8F7BDFB10210F20F7F735
:10A14000C5FEA648007868B9A5A0F8F7B3FB0021C2
:10A150000420F7F7B1FE9FA0F8F7ACFB10210F2009
:10A16000F7F7B4FE94F8240080B99F48006868B1FE
:10A170009EA0F8F79FFB00210420F7F79DFE95A015
:10A18000F8F798FB10210F20F7F7A0FE2868A16BC5
:10A19000401A41F2883188428DD926708BE7CDE98B
:10A1A000013200913023822210210F20F7F7F8FEB0
:10A1B00020211F20F8F7CCFE1020F8F7CFFE3888BA
:10A1C000F8F7D2FE8AA0F7F7FDFFD9F8000058454E
:10A1D00009DADAF80000584505DD26700B206070BA
:10A1E0000120A07067E72868A16B401AB0F5FA6FEC
:10A1F000D4D9062020702868A0635CE7CDE901323D
:10A2000000913023822210210F20F7F7C9FE202170
:10A210001F20F8F79DFE1020F8F7A0FE3888F8F709
:10A22000A3FE73A0F7F7CEFFD9F8000058450FDA68
:10A23000DAF8000058450BDD267006F099FC0C207A
:10A2400060700120A070207135E76BE029E00BE021
:10A250002868A16B401A40F6C41188429ED9062096
:10A2600020702868A06326E7CDE9013200913023F1
:10A27000822210210F20F7F793FE20213A20F8F7D1
:10A2800067FE1020F8F76AFE3888F8F76DFE5DA0CB
:10A29000F7F798FF2868A16B401A4045A2D92670AD
:10A2A00009E7CDE90132009132221423114637200B
:10A2B000F7F776FE1020F8F751FE3888F8F754FECD
:10A2C0005248807830B101280CD0022812D00328DF
:10A2D0001FD117E035213E20F8F73AFE4CA0F8F7E1
:10A2E000E9FA16E035213920F8F732FE4AA0F8F7EE
:10A2F000E1FA0EE035213920F8F72AFE48A0F8F7F8
:10A30000D9FA06E035213E20F8F722FE46A0F8F7FC
:10A31000D1FA2868A16B401A40F2DC51884293D9E7
:10A320002670C8E6CDE90132009130238222102147
:10A330000F20F7F735FE20212F20F8F709FE102017
:10A34000F8F70CFE3888F8F70FFE3948807B0228B2
:10A3500004D003280AD0012810D016E02021312093
:10A36000F8F7F6FD33A0F7F72DFF0EE020212620A9
:10A37000F8F7EEFD32A0F7F725FF06E020212620B2
:10A38000F8F7E6FD32A0F7F71DFF2868A16B401A29
:10A39000404585D926708EE6AA83FF1F8C83FF1F58
:10A3A0008883FF1F7C83FF1FB083FF1FC9E8D6C3CC
:10A3B000B3C9B9A621000000D7A2B2E1C2EBB4ED47
:10A3C000CEF32100AE83FF1F3183FF1F494E413280
:10A3D000323600004552524F522100002683FF1FA3
:10A3E0004655534233303200D890FF1F4F5450002F
:10A3F000D5FDD4DABDF8C8EB5143D3D5C6AD2E2E6A
:10A400002E000000B2BBD6A7B3D62100F86202200E
:10A4100037535053000000003230535053000000B7
:10A4200035305350530000003353505300000000A8
:10A43000C8B6FF1FD3D5C6ADD2D1BDFBD3C3210053
:10A440005044D3D5C6ADD2D1BDFBD3C3210000004B
:10A450005143D3D5C6ADD2D1BDFBD3C3210000003B
:10A4600010B50121052005F03DFC164A164938B10A
:10A4700010688B68C31A00200F2B06D208701BE0EF
:10A48000106888600220087016E013688C681B1B37
:10A49000FA2B02D2052008700EE013688C681B1B93
:10A4A000FA2B08D312688B68D21AB2F57A7F02D2DF
:10A4B0000820087000E00870BDE810400020FBF79D
:10A4C000F3B900007C83FF1F6083FF1F10B54FF4BA
:10A4D0008041022005F006FC154A164938B1106883
:10A4E000CB68C31A00200F2B06D208701BE010683F
:10A4F000C8600320087016E01368CC681B1BFA2B99
:10A5000002D2062008700EE01368CC681B1BFA2BE1
:10A5100008D31268CB68D21AB2F57A7F02D209202A
:10A52000087000E00870BDE810400E20FBF7BCB9D1
:10A530007C83FF1F6083FF1F10B54FF480610020F4
:10A5400005F0D0FB154A164970B110684B68C31A64
:10A5500000200F2B00D2087013684C681B1BFA2BCD
:10A5600007D20420087013E01068486001200870CA
:10A570000EE013684C681B1BFA2B08D312684B685B
:10A58000D21AB2F57A7F02D20720087000E0087074
:10A59000BDE810400A20FBF787B900007C83FF1F4D
:10A5A0006083FF1FF0B585B00024049402940394E7
:10A5B000009401940A268DF810608DF80040012562
:10A5C0008DF802508DF804506A460121052005F0EF
:10A5D000EBFB6A46A902002005F0E6FB6A46A903E8
:10A5E000022005F0E1FB012300225F0239461046FC
:10A5F00005F01AFD8DF802406A463946002005F044
:10A60000D3FB8DF8115003208DF8120002208DF835
:10A61000130004A8FBF7F0F80E258DF8105004A8DD
:10A62000FBF7EAF88DF8104004A8FBF7E5F8ADF861
:10A6300008600620ADF80A002048039002A80DF03B
:10A64000B7FABDF90A000AF0F7FCBDF90A000F21BC
:10A650000AF026FDBDF90A000AF008FDADF8085021
:10A660000720ADF80A001648039002A80DF0A0FAE2
:10A67000BDF90A000AF0E0FCBDF90A000F210AF05A
:10A680000FFDBDF90A000AF0F1FCADF80840082002
:10A69000ADF80A000B48039002A80DF089FABDF945
:10A6A0000A000AF0C9FCBDF90A000F210AF0F8FC03
:10A6B000BDF90A000AF0DAFC05B0F0BD39A50100C9
:10A6C000CDA4010061A4010010B51248037812491D
:10A6D0004FF47A72032B07D10B68C4681B1B93429B
:10A6E00002D90C21017010BD0378012B07D10B6832
:10A6F00044681B1B934202D90A21017010BD0378E4
:10A70000022BFBD109688368C91A9142F6D90B2143
:10A71000017010BD6083FF1F7C83FF1F10B500F028
:10A72000BFF94FF400442146002005F015FC0A2033
:10A73000FAF782FE2146002005F042FC0AF0A8FA52
:10A7400000F008FA00F05EF9112000F055FAAC486C
:10A75000807901287ED0B12000F04EFA012000F06F
:10A7600061FA2C2000F05EFA2D2000F05BFAB22096
:10A7700000F042FA012000F055FA2C2000F052FAC5
:10A780002D2000F04FFAB32000F036FA012000F03F
:10A7900049FA2C2000F046FA2D2000F043FA01205F
:10A7A00000F040FA2C2000F03DFA2D2000F03AFA9B
:10A7B000B42000F021FA072000F034FAC02000F0A5
:10A7C0001BFAA22000F02EFA022000F02BFA8420BF
:10A7D00000F028FAC12000F00FFAC52000F022FA9C
:10A7E000C22000F009FA0A2000F01CFA002000F054
:10A7F00019FAC32000F000FA8A2000F013FA2A2088
:10A8000000F010FAC42000F0F7F98A2000F00AFAEC
:10A81000EE2000F007FAC52000F0EEF90E2000F05F
:10A8200001FA212000F0E8F93A2000F0E5F90520CE
:10A8300000F0F8F9E02000F0DFF9022000F0F2F972
:10A840001C2000F0EFF9072000F0ECF9122000F0D6
:10A85000E9F900E064E0372000F0E4F9322000F08C
:10A86000E1F9292000F0DEF92D2000F0DBF92920A4
:10A8700000F0D8F9252000F0D5F92B2000F0D2F90E
:10A88000392000F0CFF9002000F0CCF9012000F0D1
:10A89000C9F9032000F0C6F9102000F0C3F9E12047
:10A8A00000F0AAF9032000F0BDF91D2000F0BAF96C
:10A8B000072000F0B7F9062000F0B4F92E2000F0D0
:10A8C000B1F92C2000F0AEF9292000F0ABF92D20D1
:10A8D00000F0A8F92E2000F0A5F92E2000F0A2F932
:10A8E000372000F09FF93F2000F09CF9002000F095
:10A8F00099F9002000F096F9022000F093F9102059
:10A9000000F090F9F02000F077F9012000F08AF9CA
:10A91000132000F071F9BDE81040292000F06CB957
:10A92000B12000F069F9052000F07CF93C2000F02E
:10A9300079F93C2000F076F9B22000F05DF90520AD
:10A9400000F070F93C2000F06DF93C2000F06AF94D
:10A95000B32000F051F9052000F064F93C2000F02C
:10A9600061F93C2000F05EF9052000F05BF93C2025
:10A9700000F058F93C2000F055F9B42000F03CF903
:10A98000032000F04FF9C02000F036F90E2000F04F
:10A9900049F90E2000F046F9042000F043F9C120E7
:10A9A00000F02AF9C52000F03DF9C22000F024F99A
:10A9B0000D2000F037F9002000F034F9C32000F03A
:10A9C0001BF98D2000F02EF92A2000F02BF9C4206D
:10A9D00000F012F98D2000F025F9EE2000F022F9A8
:10A9E000C52000F009F9062000F01CF9202000F035
:10A9F00003F93A2000F000F9552000F013F919E7A7
:10AA0000F862022010B58EB0302102A8F5F7DBFC09
:10AA10000121C80305F0E0FD0121480405F0DCFD3B
:10AA20000120ADF80800ADF80A0000210391194A91
:10AA300004928DF82C008DF82D108DF832108DF8C1
:10AA40003500154C02AA2046FAF792FA4FF49B7291
:10AA500000212046FAF70CFC01212046FAF752FAB1
:10AA60000220ADF802000D4801902420ADF800004E
:10AA700068460DF09DF8BDF902000F210AF020FB99
:10AA8000BDF902000AF0E5FABDF902000AF0FBFA8E
:10AA90000EB010BD000002400034054039AB01008B
:10AAA0001CB500200090019001248DF80040022088
:10AAB0008DF805006A468021012005F075F96A4687
:10AAC000E103002005F070F98DF802406A46042188
:10AAD000052005F069F90421052005F03DFA1CBDAB
:10AAE00010B50B4CA079012804D10A48002101714E
:10AAF00018214171FFF712FE607800B1012000F0CB
:10AB0000DBF8207900F0A4F8BDE8104000F004B8AC
:10AB1000F86202209C83FF1F10B500214F239F2263
:10AB2000084600F0D9F80348BDE810404FF4C8418A
:10AB300000F01EB9D0D6012010B502220021034832
:10AB4000FAF774F902490120087010BD003405407D
:10AB50009C83FF1F10B588B01C2101A8F5F733FCBA
:10AB60000121880405F078FD00232B2240210120DB
:10AB700005F05AFA002328222021012005F054FA7A
:10AB800000208DF812008DF8150004218DF81310A7
:10AB90008DF814008DF810008DF811008DF80F005D
:10ABA00001218DF816108DF817108DF819008DF809
:10ABB0001A008DF81B008DF81C008DF81D008DF813
:10ABC00018108DF804108DF805008DF806108DF81A
:10ABD00007008DF8081005208DF80900054C01A923
:10ABE000204607F0A5FB0121204607F0FFFA08B038
:10ABF00010BD00000000024070B50546084C05215C
:10AC0000204607F02FFB0028F9D08021012005F015
:10AC1000A3F929462046BDE8704007F0B5BD000005
:10AC20000000024070B50546084C0521204607F09B
:10AC300019FB0028F9D08021012005F0C1F929462F
:10AC40002046BDE8704007F09FBD000000000240B4
:10AC500010B504462046F5F749FD9FED101B53EC57
:10AC6000112BF5F7D4FC41EC100B9FED0E1B0AF0F5
:10AC700027FC5CB19FED0D1B51EC100B53EC112B1D
:10AC8000F5F753FCF5F73FFD82B200E00122BDE885
:10AC900010400621074809F07FBD000000000000B9
:10ACA00000005940175D74D14517DD3F00000000DA
:10ACB00000489D40005C014010B504463620FFF777
:10ACC0009BFF24B1BDE81040A820FFF7ABBFBDE853
:10ACD00010406820FFF7A6BF2DE9F04107468846DF
:10ACE00015461E462A20FFF787FF1F4C207938445F
:10ACF000000AFFF797FF20793844C0B2FFF792FFB0
:10AD000020792844C0F30720FFF78CFF20792844DE
:10AD1000C0B2FFF787FF2B20FFF76EFF607940443A
:10AD2000000AFFF77FFF60794044C0B2FFF77AFF67
:10AD300060793044C0F30720FFF774FF6079304436
:10AD4000C0B2FFF76FFF2C20FFF756FF074C05211D
:10AD5000204607F087FA0028F9D02046BDE8F041E8
:10AD6000002107F043BA00009C83FF1F000002404F
:10AD700070B50D460C4C024600212046FAF7DAF970
:10AD80002A4600212046FAF721FA8021012005F009
:10AD900017F9012200212046F9F76EFFBDE8704047
:10ADA0000121024807F022BA0034054000000240A9
:10ADB0002DE9F0412DED028B82B01020F8F7CEF88E
:10ADC00000210846F8F7C4F8C24C2088F8F7CCF800
:10ADD000C1A0F7F7F7F900215820F8F7B9F8C149F1
:10ADE000012091ED000AF7F7FBFFBFA0F7F762FD26
:10ADF000BE4F3878BE4E4FF010053178084208D06B
:10AE00002088CDE900050023BAA219469020F8F762
:10AE1000B1F838783178884308D02088CDE900052A
:10AE20000023B5A219469020F8F7A4F830783978B5
:10AE3000884308D02088CDE900050023AEA219463A
:10AE40009020F8F797F8387850B9307840B92088D2
:10AE5000CDE900050023A7A219469020F8F78AF84B
:10AE6000A649FF2012230988CDE900109F22194628
:10AE70000020F7F753F8A2480088F8F775F8142176
:10AE80000020F8F765F89FA0F7F714FD0C20F8F7FD
:10AE900065F803210020F7F70FF89BA0F7F70AFDEC
:10AEA0006FF0020841460020F7F706F81020F8F787
:10AEB00055F8964F964D97ED000AD5ED000A9FED97
:10AEC000958A954CB4EEE00AF1EE10FA0BDD30EE07
:10AED000600A0520C0EE080A94ED000A20EE800A00
:10AEE000F7F77EFF0AE070EEC00A052080EE880AC0
:10AEF000D4ED000A20EE200AF7F772FF87A0F7F7DB
:10AF0000D9FC00210520F6F7D7FF85A0F7F7D2FC82
:10AF10000C20F8F723F803210020F6F7CDFF81A0DD
:10AF2000F7F7C8FC41460020F6F7C6FF1020F8F7F7
:10AF300015F897ED000A0220C0EE080A94ED000A09
:10AF400020EE800AF7F74CFF74A0F7F7B3FC24213A
:10AF50000120F7F7FDFF74A0F7F7ACFC0C20F7F722
:10AF6000FDFF03210020F6F7A7FF70A0F7F7A2FC72
:10AF700041460020F6F7A0FF1020F7F7EFFF6D4ED7
:10AF8000042096ED000AF7F72BFF6BA0F7F792FC71
:10AF900000210520F6F790FF61A0F7F78BFC0C204D
:10AFA000F7F7DCFF03210020F6F786FF63A0F7F731
:10AFB00081FC41460020F6F77FFF1020F7F7CEFF17
:10AFC00095ED000A0220C0EE080A94ED000A20EE7A
:10AFD000800AF7F705FF51A0F7F76CFC3621002037
:10AFE000F7F7B6FF96ED000A554910EE100A8842B1
:10AFF0005CDD38684FF08A41884202DB286888426D
:10B0000054DA36212020F7F7A3FF1C20F7F7A6FF1C
:10B010004C4D4D494D4C95ED000A10EE100A8842FA
:10B0200003DA0320F7F7DCFE26E010EE100A4849A9
:10B03000884203DA0220F7F7D3FE1DE010EE100A73
:10B04000A04203DA0120F7F7CBFE15E010EE100A5C
:10B0500040499FED411A884207DAC0EE010A0320F9
:10B06000B0EE600AF7F7BCFE06E0C0EE010A02206F
:10B07000B0EE600AF7F7B4FE1020F7F76FFF042177
:10B080000320F6F719FF2868A04207DA02B033A0C0
:10B09000BDEC028BBDE8F041F7F70CBC02B030A06C
:10B0A000BDEC028BBDE8F041F7F704BC392100206C
:10B0B000F7F74EFF4220F7F751FF2A480088F7F7CD
:10B0C00053FF02B028A0BDEC028BBDE8F041F7F7BA
:10B0D000F1BB0000AC83FF1FBFAAB6FBCEC4B2E237
:10B0E000CFDF00008483FF1FA1E600003083FF1F35
:10B0F000A683FF1F3E0000003C000000A883FF1F46
:10B10000AA83FF1F44000000753A00009083FF1FD0
:10B110009483FF1F00F07F458083FF1F56000000CF
:10B1200055000000313A0000490000006275733A92
:10B13000000000003C83FF1F41000000323A000085
:10B14000CDCCCC3E148FFF1F0000204100007A447C
:10B150000000C84200401C4600007A446DA6B800BA
:10B16000A6B80000AE83FF1FC7EBD5FDC8B7BDD39F
:10B17000C8EBBFAAB6FBCEC4B2E2CAD4D2C70000A5
:10B180002DE9F04F2DED028B83B0FE4801780025AC
:10B19000FD4EFE4CDFF8F89304290CD00178052908
:10B1A0000DD0017806290ED001780A290FD0017838
:10B1B0000B2918D01FE00570012060701BE005709E
:10B1C0000220607017E005700A20607013E00570BF
:10B1D000307880F001003070EE494870FFF76CFD68
:10B1E000FCF768FD07E0057099F80E00012811D002
:10B1F00005F0B7FEA5701020F7F7B0FEE64F3888CF
:10B20000F7F7B2FEE5490A783078024236D109787C
:10B2100039B107E072B600210220FCF785FC62B666
:10B22000E9E758B394ED0F0A4121BCEEC00A10EED5
:10B23000100AC0B2F7F78CFED9A0F7F73BFB4FF02E
:10B24000FF0ACDE9005A4F23682241215820F6F722
:10B2500065FEDFF850B39BED000AB5EEC00AF1EED3
:10B2600010FA46DD94ED0F0ACF4910EE100A88421D
:10B2700016DC9FEDCE0A84ED0F0A3EE094ED0F0A36
:10B28000DFEDCB0A30EEC00ABDEEC00A10EE100AA8
:10B290004121C0B2F7F75CFEC6A0F7F70BFBCEE783
:10B2A000DBED000A10EE900AB0F17E5F06DADFED0A
:10B2B000C20A30EE600A84ED0F0A1EE0DBED000AE0
:10B2C000BE4910EE900AF0EE040A88420CDA9BEDBB
:10B2D000001A21EE201ADFEDBA1AC1EE210A30EE73
:10B2E000600A84ED0F0A08E030EE600A84ED0F0A70
:10B2F00003E09FEDB40A84ED0F0AB348DFF8CC8277
:10B300001C2490ED000AB24E10EE101A41450BDAE3
:10B310003188CDE90014002390ED000A042219467B
:10B320001846F8F791F80AE03188CDE900140023B7
:10B3300090ED000A032219461846F8F785F8308880
:10B34000CDE900040023A3A219465320F7F712FE0B
:10B35000A148A24D90ED000A10EE101A41450BDAFB
:10B360002988CDE90014002390ED000A04221B2156
:10B370001846F8F769F80AE02988CDE90014002397
:10B3800090ED000A03221B211846F8F75DF8288883
:10B39000CDE90004002392A21B215320F7F7EAFD18
:10B3A0009BED000A10EE100A40450BDA3888CDE913
:10B3B0000004002304229BED000A37211846F8F709
:10B3C00043F823E09BED000A10EE100A404512DB23
:10B3D0009BED000A834910EE100A88420BDA388888
:10B3E000CDE90004002303229BED000A3721184613
:10B3F000F8F72AF80AE03888CDE900040023022291
:10B400009BED000A37211846F8F71EF83888CDE979
:10B410000004002374A237215320F7F7ABFD2888DE
:10B42000CDE9000A4F23682200216720F6F776FD58
:10B4300099F80800DFED6D8A1024022838D004281E
:10B440007ED03088CDE90004002369A219466C2023
:10B45000F7F790FD3088CDE900046648002302220A
:10B4600090ED000A19468020F7F7EEFF3088CDE90D
:10B470000004002360A211216C20F7F77BFD3088C7
:10B48000CDE900045D480023022290ED000A11215D
:10B490008020F7F7D9FF0CF05FFA801E0C286FD2DE
:10B4A000DFE800F0FBFAF9F8F7F6F5F4F3F2F1F063
:10B4B000B9F80A0000EE100AB8EE400A9FED508A73
:10B4C00020EE080A10EE101A414523DA3088CDE943
:10B4D000000400234BA201216B20F7F74BFD3088BD
:10B4E000CDE90004B9F80A00002300EE100A022298
:10B4F0000121B8EE400A742020EE080AF7F7A4FFF5
:10B500003088CDE90004002332A201219420F7F70E
:10B5100031FD19E000EE100A3188CDE90014B8EED3
:10B52000400A00230222012120EE080A6B20F7F7CF
:10B530008BFF3088CDE90004002326A2012100E022
:10B540006CE09420F7F716FD3088CDE90004002365
:10B550002CA211216B20F7F70DFD3088CDE90004F6
:10B5600099F80C00002300EE100A02221121B8EE17
:10B57000400A742020EE280AF7F766FF308843E07F
:10B5800081E100006083FF1FA683FF1FB083FF1FC0
:10B59000C8B6FF1FF8620220AC83FF1F3083FF1F75
:10B5A0003C0000004083FF1F0000B0420000FE424C
:10B5B000000058433E000000CDCCCC3D00001643B7
:10B5C000000016430000D8423483FF1F00002041D2
:10B5D000A883FF1F560000003C83FF1FAA83FF1FA4
:10B5E000410000000000C84257000000CDCC4C3D97
:10B5F000442B00008883FF1F442D00008C83FF1F15
:10B600000AD7A33C300000000023AFF22C02CDE9A2
:10B61000000411219420F7F7ADFC3CE7B9F80A00CB
:10B6200000EE100AB8EE400A9FEDBA8A20EE080A32
:10B6300010EE101A414531DA30880023AFF23C0297
:10B64000CDE9000401216B20F7F794FC3088CDE9A7
:10B650000004B9F80A00002300EE100A02220121BA
:10B66000B8EE400A742020EE080AF7F7EDFE3088A5
:10B670000023AFF2A002CDE9000401219420F7F7E6
:10B6800079FC24E0F5E0EAE0DFE0D4E08BE080E064
:10B6900075E06AE05FE054E049E03EE000EE100A49
:10B6A0003188CDE90014B8EE400A002302220121BE
:10B6B00020EE080A6B20F7F7C7FE30880023AFF2B0
:10B6C000EC02CDE9000401219420F7F753FC308807
:10B6D0000023AFF2D002CDE9000411216B20F7F76F
:10B6E00049FC3088CDE9000499F80C00002300EEF5
:10B6F000100A02221121B8EE400A742020EE280A16
:10B70000F7F7A2FE30880023AFF22C12CDE9000437
:10B7100011219420F7F72EFCBDE62888CDE900041E
:10B7200000237DA221217020F7F724FCB4E02888B3
:10B73000CDE9000400237AA221217020F7F71AFC3A
:10B74000AAE02888CDE90004002377A221216C20FB
:10B75000F7F710FCA0E02888CDE90004002374A2CC
:10B7600021216C20F7F706FC96E02888CDE900043B
:10B77000002371A221216F20F7F7FCFB8CE02888C1
:10B78000CDE9000400236EA221217520F7F7F2FB1A
:10B7900082E02888CDE9000400236AA221217320D9
:10B7A000F7F7E8FB78E099F800000A2821D228880A
:10B7B000CDE90004002364A221217120F7F7DAFB10
:10B7C0002888CDE9000499F80000002300EE100A53
:10B7D0001A462121B8EE400A8620F7F735FE288860
:10B7E000CDE90004002351A221218F20F7F7C2FBED
:10B7F00052E02888CDE90004002353A221216C20C7
:10B80000F7F7B8FB2888CDE9000499F80000002379
:10B8100000EE100A1A462121B8EE400A8120F7F7FF
:10B8200013FE2888CDE90004002340A221219320A3
:10B83000F7F7A0FB30E02888CDE90004002343A2FD
:10B8400021217520F7F796FB26E02888CDE9000432
:10B8500000233FA221217420F7F78CFB1CE02888ED
:10B86000CDE9000400233BA221217520F7F782FBDC
:10B8700012E02888CDE90004002337A22121752099
:10B88000F7F778FB08E02888CDE90004002333A20D
:10B8900021216C20F7F76EFB3888CDE90004314890
:10B8A0000023012290ED000A31216D20F7F7CCFD35
:10B8B0003888CDE9000400232BA231218E20F7F730
:10B8C00059FB2A48007888B1012819D0022808D1EC
:10B8D0003888CDE90004002325A241217F20F7F715
:10B8E00049FB03B0BDEC028BBDE8F08F3888CDE991
:10B8F000000400231AA240218220F7F73BFBF0E767
:10B900003888CDE9000400231AA241217F20F7F7EF
:10B9100031FBE6E7CDCCCC3C51433556000000006E
:10B9200051433956000000005143313256000000A7
:10B9300051433230560000005143332E3000000096
:10B94000534350004D544B0050440000505053009E
:10B950004443500056415200415653002D2D2D2D89
:10B960002D2D2D008483FF1FA1E600002083FF1FE3
:10B97000434332004343310002490020087002492A
:10B98000487070476083FF1FB083FF1F2DE9F04FA1
:10B990002DED108B83B0FB480178FB4DFB4C4FF035
:10B9A000000A04290CD0017805290ED00178062957
:10B9B00010D001780A2912D001780B291CD025E07B
:10B9C00080F800A00220607020E080F800A084F8D9
:10B9D00001A01BE080F800A00A20607016E080F84B
:10B9E00000A0287880F001002870E9494870FFF72E
:10B9F00063F9FCF75FF909E080F800A0E548807B77
:10BA0000012812D005F0ADFA84F802A01020F7F753
:10BA1000A5FAE14E3088F7F7A7FAE0490A782878C6
:10BA200002423BD1097839B107E000210220FCF73E
:10BA30007BF8F9F7BFFFE9E778B394ED0F0AF0EE72
:10BA4000000A422130EE600ABCEEC00A10EE100A75
:10BA5000C0B2F7F77DFAD2A0F6F72CFF4FF0FF0B3C
:10BA60004F23682242215820CDE900ABF6F756FA61
:10BA7000DFF8308398ED000AB5EEC00AF1EE10FA57
:10BA800048DD94ED0F0AC84910EE100A884218DC10
:10BA90009FEDC60A84ED0F0A40E0FFE794ED0F0A20
:10BAA000DFEDC30A30EEC00ABDEEC00A10EE100A88
:10BAB0004221801EC0B2F7F74BFABEA0F6F7FAFE9D
:10BAC000CCE7D8ED000A10EE900AB0F17E5F06DAFE
:10BAD000DFEDB90A30EE600A84ED0F0A1EE0D8ED02
:10BAE000000AB64910EE900AF0EE040A88420CDA19
:10BAF00098ED001A21EE201ADFEDB11AC1EE210AED
:10BB000030EE600A84ED0F0A08E030EE600A84ED42
:10BB10000F0A03E09FEDAB0A84ED0F0AAA48AB4C75
:10BB20001C2790ED000AAA4D10EE101AA1420BDA64
:10BB30002988CDE90017002390ED000A0422194658
:10BB40001846F7F781FC0AE02988CDE900170023A1
:10BB500090ED000A032219461846F7F775FC28886D
:10BB6000CDE9000700239BA219465320F7F702FAFC
:10BB70009948DFF8689290ED000A10EE101AA14281
:10BB80000CDAB9F80010CDE90017002390ED000A97
:10BB900004221B211846F7F757FC0BE0B9F80010F8
:10BBA000CDE90017002390ED000A03221B2118465F
:10BBB000F7F74AFCB9F80000CDE90007002388A296
:10BBC0001B215320F7F7D6F998ED000A404610EEF6
:10BBD000102A21469FED83CB9FED84BB9FED85DB33
:10BBE000DFF818829FED86EB9FED87FB9FED889B2A
:10BBF0009FED89AB9FED8A8B10248A420BDA318846
:10BC0000CDE90017002390ED000A042237211846E1
:10BC1000F7F71AFC23E090ED000A10EE102A8A4292
:10BC200012DB90ED000A804A10EE101A91420BDAF6
:10BC30003188CDE90017002390ED000A0322372157
:10BC40001846F7F701FC0AE03188CDE90017002318
:10BC500090ED000A022237211846F7F7F5FB3088ED
:10BC6000CDE90007002371A237215320F7F782F9AD
:10BC7000B9F80000CDE9000B4F23682200216720AE
:10BC8000F6F74CF998ED000B53EC1B2B51EC100B15
:10BC9000F4F766FD09D22888CDE90004002364A2E8
:10BCA00019467220F7F766F908E02888CDE9000404
:10BCB000002361A219467820F7F75CF998ED000B94
:10BCC00053EC192B51EC100BF4F74AFD11D298EDFF
:10BCD000000B51EC100BF4F773FD00EE100A2888EE
:10BCE000CDE90004002304220E216B20F7F7ACFB02
:10BCF0005FE198ED000B53EC192B51EC100BF4F7AE
:10BD000047FD1AD898ED000B53EC1A2B51EC100B91
:10BD1000F4F726FD11D298ED000B51EC100BF4F75F
:10BD20004FFD00EE100A2888CDE90004002303220D
:10BD30000E216B20F7F788FB3BE198ED000B53ECED
:10BD40001A2B51EC100BF4F723FD77D898ED000B6C
:10BD500053EC182B51EC100BF4F702FD6ED298ED5A
:10BD6000000B51EC100BF4F72BFD00EE100A2888A5
:10BD7000CDE90004002302220E216B20F7F764FBBB
:10BD800017E15BE06083FF1FA683FF1FB083FF1FE7
:10BD9000F8620220C8B6FF1FAC83FF1F3083FF1F6D
:10BDA0003C0000004083FF1F0000B0420000FE4244
:10BDB000000058433E000000CDCCCC3D00001643AF
:10BDC000000016430000D8423483FF1F00002041CA
:10BDD000A883FF1F560000003C83FF1FAA83FF1F9C
:10BDE00041000000000000000088C3400000000087
:10BDF000006AF8400000000080842E415883FF1F35
:10BE00009A9999999999B93F000000000000F03F74
:10BE10000000000000002440000000000000594025
:10BE20000000000000408F400000C84257000000A2
:10BE30006D41683A0000000041683A0098ED000B3F
:10BE400053EC182B51EC100BF4F7A2FC1AD898ED18
:10BE5000000B53EC1C2B51EC100BF4F781FC11D2AE
:10BE600098ED000B51EC100BF4F7AAFC00EE100A51
:10BE70002888CDE90004002301220E216B20F7F76A
:10BE8000E3FA96E098ED000B53EC1C2B51EC100BF1
:10BE9000F4F77EFC1AD898ED000B53EC1B2B51ECF9
:10BEA000100BF4F75DFC11D298ED000B51EC100B68
:10BEB000F4F786FC00EE100A2888CDE90004002380
:10BEC0001A460E216B20F7F7BFFA72E098ED000BCF
:10BED00053EC1B2B51EC100BF4F75AFC22D898EDC5
:10BEE000000B53EC1D2B51EC100BF4F739FC19D25D
:10BEF000B0EE480AF0EE680A53EC102B98ED000BF8
:10BF000051EC100BF4F783FBF4F75AFC00EE100A27
:10BF10002888CDE90004002302220E216B20F7F7C8
:10BF200093FA46E098ED000B53EC1D2B51EC100BEF
:10BF3000F4F72EFC24D89FEDE20B53EC102B98ED78
:10BF4000000B51EC100BF4F70BFC19D2B0EE480AC1
:10BF5000F0EE680A53EC102B98ED000B51EC100B2F
:10BF6000F4F755FBF4F72CFC00EE100A2888CDE915
:10BF70000004002301220E216B20F7F765FA18E078
:10BF8000B0EE480AF0EE680A53EC102B98ED000B67
:10BF900051EC100BF4F73BFBF4F712FC00EE100A27
:10BFA0002888CDE9000400231A460E216B20F7F7FC
:10BFB0004BFAC54D53EC1F2B95ED000B51EC100BBC
:10BFC000F4F7CEFB0AD2B9F80000CDE90004002353
:10BFD000BEA21B217220F6F7CDFF09E0B9F80000E0
:10BFE000CDE900040023BBA21B217820F6F7C2FF95
:10BFF0009FEDB9BB95ED000B53EC1B2B51EC100BD7
:10C00000F4F7AEFB16D295ED000B53EC182B51EC68
:10C01000100BF4F78AFAF4F7D3FB00EE100AB9F824
:10C020000000CDE900040023042229216B20F7F74A
:10C030000BFAF7E095ED000B53EC1B2B51EC100BBA
:10C04000F4F7A6FB1FD895ED000B53EC1E2B51EC1B
:10C05000100BF4F785FB16D295ED000B53EC182B63
:10C0600051EC100BF4F761FAF4F7AAFB00EE100A9A
:10C07000B9F80000CDE900040023032229216B2038
:10C08000F7F7E2F9CEE095ED000B53EC1E2B51ECE7
:10C09000100BF4F77DFB1FD895ED000B53EC1F2B15
:10C0A00051EC100BF4F75CFB16D295ED000B53EC42
:10C0B000182B51EC100BF4F738FAF4F781FB00EE73
:10C0C000100AB9F80000CDE900040023022229215A
:10C0D0006B20F7F7B9F9A5E095ED000B53EC1F2B9A
:10C0E00051EC100BF4F754FB1BD895ED000B53ECFF
:10C0F000192B51EC100BF4F733FB12D295ED000B1A
:10C1000051EC100BF4F75CFB00EE100AB9F80000DC
:10C11000CDE900040023042229216B20F7F794F9CC
:10C1200080E095ED000B53EC192B51EC100BF4F75C
:10C130002FFB1BD895ED000B53EC1A2B51EC100B79
:10C14000F4F70EFB12D295ED000B51EC100BF4F747
:10C1500037FB00EE100AB9F80000CDE90004002317
:10C16000032229216B20F7F76FF95BE095ED000BB7
:10C1700053EC1A2B51EC100BF4F70AFB1BD895ED7E
:10C18000000B53EC182B51EC100BF4F7E9FA12D218
:10C1900095ED000B51EC100BF4F712FB00EE100ABA
:10C1A000B9F80000CDE900040023022229216B2008
:10C1B000F7F74AF936E095ED000B53EC182B51ECEC
:10C1C000100BF4F7E5FA1BD895ED000B53EC1C2B84
:10C1D00051EC100BF4F7C4FA12D295ED000B51ECB0
:10C1E000100BF4F7EDFA00EE100AB9F80000CDE9F3
:10C1F00000040023012229216B20F7F725F911E023
:10C2000095ED000B51EC100BF4F7DAFA00EE100A82
:10C21000B9F80000CDE9000400231A4629216B205B
:10C22000F7F712F930880C25CDE900A02C480295CB
:10C230000223027837216920F7F786F93088CDE9A3
:10C240000005002327A238217720F6F793FE3088D7
:10C250000295CDE900A024480223372102787D20F1
:10C26000F7F772F93088CDE9000500231DA23821C7
:10C270008B20F6F77FFE30880295CDE900A01B48A1
:10C280000223372102789120F7F75EF93088CDE953
:10C290000004174800231A4690ED000A42217C2032
:10C2A000F7F7D2F83088CDE90004002311A242212B
:10C2B0008E20F6F75FFE03B0BDEC108BBDE8F08F6B
:10C2C00000000000D01263415083FF1F6D57683A91
:10C2D0000000000057683A007B14AE47E17A843FC3
:10C2E000B58EFF1F3A000000B68EFF1FB78EFF1FEE
:10C2F0008483FF1FA1E600002DE9F04F2DED028B96
:10C3000083B0FC4801780025FB4EFC4C04290CD07E
:10C31000017805290CD0017806290DD001780A2969
:10C320000ED001780B2917D01EE0057065701BE058
:10C3300005700120607017E005700A20607013E03E
:10C340000570307880F001003070ED494870FEF7DC
:10C35000B3FCFBF7AFFC07E00570EA48807B0128DF
:10C3600011D004F0FEFDA5701020F6F7F7FDE64DA4
:10C370002888F6F7F9FDE5490A78307802422DD190
:10C38000097839B107E000210220FBF7CDFBF9F76E
:10C3900011FBE9E710B394ED100A0021BCEEC00ACE
:10C3A00010EE100AC0B2F6F7D3FDD9A0F6F782FA64
:10C3B000D84890ED000A9FEDD88AB5EEC00AF1EE9C
:10C3C00010FA46DD94ED100AD44A10EE101A91428C
:10C3D00016DC9FEDD30A84ED100A3CE094ED100AC0
:10C3E000DFEDD00A30EEC00ABDEEC00A10EE100A32
:10C3F0000021C0B2F6F7ACFDCBA0F6F75BFAD7E7A9
:10C40000D0ED000A10EE901AB1F17E5F06DADFED92
:10C41000C70A30EE600A84ED100A1CE0D0ED000A75
:10C42000C34A10EE901AF0EE040A91420CDA90ED35
:10C43000001A21EE201ADFEDBF1AC1EE210A30EEFC
:10C44000600A84ED100A06E030EE600A84ED100AFE
:10C4500001E084ED0F8A10242888CDE90004B64855
:10C4600000231A4690ED000A19466B20F6F7ECFF00
:10C470002888CDE900040023B0A219467D20F6F7F4
:10C4800079FDAF48AF4EDFF8C0B290ED000A10EE74
:10C49000101AB1420CDABBF80010CDE900140023E9
:10C4A00090ED000A032219461846F6F7CDFF0BE07F
:10C4B000BBF80010CDE90014002390ED000A022221
:10C4C00019461846F6F7C0FFBBF80000CDE9000496
:10C4D00000239EA219462920F6F74CFD9C48DFF860
:10C4E00074A290ED000A10EE101AB1420CDABAF8FC
:10C4F0000010CDE90014002390ED000A0322194634
:10C500003520F6F7A1FF0BE0BAF80010CDE90014D2
:10C51000002390ED000A022219463520F6F794FF19
:10C52000BAF80000CDE9000400238BA219465E2072
:10C53000F6F720FDFF20BAF80010CDE90010132314
:10C540009F2212210020F5F7E9FC4FF04209BBF8C9
:10C550000000CDE90009002380A217211846F6F754
:10C5600009FD804890ED000A10EE100AB0420ADA88
:10C57000BBF80000CDE90004002302221821192095
:10C58000F6F762FF09E0BBF80000CDE900040023E4
:10C59000012218211920F6F757FFBBF80000CDE95A
:10C5A0000004002369A218213920F6F7E3FC6E4845
:10C5B00090ED000A10EE100AB0420ADABBF8000053
:10C5C000CDE900040023022218214520F6F73CFFA4
:10C5D00009E0BBF80000CDE9000400230122182186
:10C5E0004520F6F731FFBBF80000CDE90004002339
:10C5F00059A218216520F6F7BDFC5C48514F4FF059
:10C60000D47890ED000A7F4210EE100AB0420ADAA8
:10C61000BBF80000CDE9000400230222182171209C
:10C62000F6F712FF19E010EE100A384440450AD21E
:10C63000BBF80000CDE9000400230122182171207D
:10C64000F6F702FF09E0BBF80000CDE90004002383
:10C650001A4618217120F6F7F7FEBBF80000CDE965
:10C660000004002342A218219120F6F783FCBAF8B7
:10C670000000CDE9000900233EA22B211846F6F761
:10C6800079FC3E4890ED000A10EE100AB0420ADA3A
:10C69000BAF80000CDE90004002302222C21192061
:10C6A000F6F7D2FE09E0BAF80000CDE90004002355
:10C6B00001222C211920F6F7C7FEBAF80000CDE9B7
:10C6C0000004002321A22C213920F6F753FC2C482A
:10C6D00090ED000A10EE100AB04253DABAF80000EA
:10C6E000CDE90004002302222C214520F6F7ACFE00
:10C6F00052E000006083FF1FA683FF1FB083FF1F6F
:10C70000F8620220C8B6FF1FAC83FF1F3083FF1FF3
:10C710003C0000004083FF1F000000000000F442C6
:10C7200000001F4300808C433E000000CDCCCC3D78
:10C7300000001643000016438483FF1FA1E600009B
:10C740003483FF1F00002041A883FF1F5600000014
:10C750003C83FF1FAA83FF1F41000000D7EEB8DF14
:10C7600000000000E48EFF1FE88EFF1FEC8EFF1F0D
:10C7700057000000C6BDBEF900000000F08EFF1F8C
:10C78000F48EFF1FBAF80000CDE900040023012257
:10C790002C214520F6F758FEBAF800000023AFF22E
:10C7A0004802CDE900042C216520F6F7E3FB794827
:10C7B00090ED000A10EE100AB0420ADABAF8000052
:10C7C000CDE90004002302222C217120F6F73CFE63
:10C7D00019E010EE100A384440450AD2BAF80000B9
:10C7E000CDE90004002301222C217120F6F72CFE54
:10C7F00009E0BAF80000CDE9000400231A462C2114
:10C800007120F6F721FEBAF800000023AFF2A00273
:10C81000CDE900042C219120F6F7ACFB2888CDE966
:10C82000000900235CA23F211846F6F7A3FB5C48F1
:10C83000DFF8709190ED000A10EE100A48450BD118
:10C840002888CDE9000400230222B0EE480A4021E6
:10C850001920F6F7F9FD16E010EE100AB04209DAD9
:10C860002888CDE900040023022240211920F6F790
:10C87000EBFD08E02888CDE90004002301224021D7
:10C880001920F6F7E1FD28880023AFF24012CDE928
:10C89000000440213920F6F76DFB434890ED000A73
:10C8A00010EE100A48450BD12888CDE9000400237A
:10C8B0000222B0EE480A40214520F6F7C5FD16E0F9
:10C8C00010EE100AB04209DA2888CDE900040023EE
:10C8D000022240214520F6F7B7FD08E02888CDE97F
:10C8E00000040023012240214520F6F7ADFD2888F1
:10C8F0000023AFF29C12CDE9000440216520F6F739
:10C9000039FB2A4890ED000A10EE100A48450BD179
:10C910002888CDE9000400230222B0EE480A402115
:10C920007120F6F791FD25E010EE100AB04209DA09
:10C930002888CDE900040023022240217120F6F767
:10C9400083FD17E010EE100A3844404509D22888CC
:10C95000CDE900040023012240217120F6F774FD87
:10C9600008E02888CDE9000400231A464021712000
:10C97000F6F76AFD28880023AFF20C22CDE9000407
:10C9800040219120F6F7F6FA03B0BDEC028BBDE82A
:10C99000F08F0000F88EFF1FD7EEB5CD000000002D
:10C9A000FC8EFF1F00007A44008FFF1F048FFF1FC3
:10C9B000F0EE401AB0EE410AF4EEE01AF1EE10FA91
:10C9C00007DDF4EEC01AF1EE10FA01DDB0EE610AF7
:10C9D0007047F4EEC00AF1EE10FAF9DDB0EE600A2D
:10C9E000704710B5AFF3008010BD00002DE9FC4189
:10C9F00000F05CF81020F6F7B1FA0024284D274E1D
:10CA000005F59A773088F6F7AFFA2007010E002077
:10CA1000F6F79EFAE87A844212D102210020F5F757
:10CA20004BFA0C20F6F79AFA1E480088F6F79CFAA3
:10CA30001DA0F5F73FFF6FF001010020F5F73CFA6C
:10CA40001020F6F78BFA287B204400EB400101EB25
:10CA5000001057F82000F5F7B5FB641CE4B2052C74
:10CA6000D0D3FF243088CDE900049E224F2300213B
:10CA70001046F5F753FA3088CDE90004E87A297BAF
:10CA80009F22084400EB400101EBC0039B1C0021E6
:10CA90009D20F5F743FABDE8FC810000AA83FF1F43
:10CAA000B083FF1FA883FF1F3E00000070B5324C0B
:10CAB0002578324A0023042DD07A117B0FD02678B6
:10CAC0000325052E19D02678062E12D108440828F1
:10CAD00050D2DFE800F01F21244144474A4D04288A
:10CAE00002D2401CD07203E0032903D0491C117309
:10CAF000237070BDD3721373FAE710B1401ED07269
:10CB000002E019B1491E1173237070BD0420D07268
:10CB10001573F9E755702DE0162050702AE018487B
:10CB2000807B022815D1907898B9164890ED000ABC
:10CB300010EE100AB0F17C5F0BDD13480168956BB5
:10CB4000491BB1F5487F15D9082111700068906321
:10CB500010E0072050700DE00E2050700AE0102009
:10CB6000507007E00D20507004E00F20507001E07D
:10CB700011205070237070BD6083FF1FB083FF1FB2
:10CB8000C8B6FF1F4083FF1F7C83FF1F034900209F
:10CB9000087003490A204870704700006083FF1F37
:10CBA000B083FF1F10B500F001F810BD10B5064CA2
:10CBB0002068002804D14FF4927104A0F8F708FC13
:10CBC0002068BDE810400047EC90FF1F2E2E5C2E21
:10CBD0002E5C2E2E5C2E2E5C2E2E5C647269766589
:10CBE000725C7372635C68633332663436305F65DF
:10CBF00078696E745F6E6D695F7377692E6300008C
:10CC00002DE9FC41F9480178F94D062905D10021AB
:10CC100001700120687702F079FF1020F6F79EF985
:10CC200000210846F6F794F9F2480088F6F79CF9D7
:10CC30006868F14C00287CD0F0A0F5F7C3FA0C200E
:10CC4000F6F78CF92088F6F78FF914210020F6F713
:10CC50007FF9EEA0F5F72EFE08212868F5F7A6FC6F
:10CC600020210020F6F774F9E8A0F5F723FE08214B
:10CC70006868F5F79BFC2C210020F6F769F9E3A022
:10CC8000F5F718FE0821A868F5F790FC3821002078
:10CC9000F6F75EF9DDA0F5F70DFE0821E868F5F777
:10CCA00085FC44210020F6F753F9D8A0F5F702FEE1
:10CCB00008212869F5F77AFCD54F3888F6F754F93A
:10CCC00014215220F6F744F968680C24C0F3C260BE
:10CCD0004FF4784603286CD004286FD0CDE9006467
:10CCE0000023CCA214215220F6F744F9142181200C
:10CCF000F6F72EF9E87F30B1C7A0F5F7DBFDE87F46
:10CD00000021F6F7DFF820215220F6F721F92869F3
:10CD1000410757D000F00700012857D0022859D00A
:10CD200003285BD0CDE9006400232021B9A2522062
:10CD300000E03AE1F6F71EF92C215220F6F708F947
:10CD40002869410A89074DD0C0F3412101294DD0FE
:10CD500002294FD06FEA502080074FD0CDE9006400
:10CD60000023ACA22C215220F6F704F90021082060
:10CD7000F5F7A2F8287CC0F34110012842D0022820
:10CD800044D0CDE900640023A2A22C217F20F6F735
:10CD9000F1F838215220F6F7DBF82869C0F3433068
:10CDA000092857D2DFE800F056363A3E42464A4E4E
:10CDB00052009AA0F5F706FA98E7FFE799A0F5F771
:10CDC00001FA93E799A0F5F775FDB5E799A0F5F796
:10CDD00071FDB1E79AA0F5F76DFDADE79BA0F5F702
:10CDE00069FDA9E79CA0F5F765FDBFE79BA0F5F7F6
:10CDF00061FDBBE79AA0F5F75DFDB7E799A0F5F7F0
:10CE000059FDB3E798A0F5F755FDC2E797A0F5F7F0
:10CE100051FDBEE796A0F5F74DFD23E095A0F5F78F
:10CE200049FD1FE094A0F5F745FD1BE093A0F5F741
:10CE300041FD17E092A0F5F73DFD13E091A0F5F755
:10CE400039FD0FE090A0F5F735FD0BE08EA0F5F76A
:10CE500031FD07E0CDE9006400236EA238215320A4
:10CE6000F6F788F82869800309D53888CDE90004E9
:10CE7000002386A238217620F6F77CF807E0CDE97A
:10CE80000064002381A238217620F6F773F844214C
:10CE90005220F6F75DF8A88842F6013280B2811A76
:10CEA00090425FD01DDC41F2EF72A0EB0201904294
:10CEB0004ED00BDCB0F57C7F45D0A0F5A060AC383F
:10CEC0005FD0A0F5506025381FD128E0E22935D089
:10CED000A1F52061EA392CD0A1F580613E3914D149
:10CEE0003BE0B1F5667F5BD009DC1C2953D0B1F57E
:10CEF000257F19D0A1F54071863906D146E0A1F50C
:10CF0000C0611B3933D0402936D061A0F5F7D2FC7F
:10CF1000A888BDE8FC4180B20421F5F747BBBDE815
:10CF2000FC415DA0F5F7C6BCBDE8FC415CA0F5F78F
:10CF3000C1BCBDE8FC415CA0F5F7BCBCBDE8FC4150
:10CF40005BA0F5F7B7BCBDE8FC415BA0F5F7B2BC50
:10CF5000BDE8FC4159A0F5F7ADBCBDE8FC4159A0C6
:10CF6000F5F7A8BCBDE8FC4158A0F5F7A3BCBDE8A7
:10CF7000FC4157A0F5F79EBCBDE8FC4157A0F5F772
:10CF800099BCBDE8FC4157A0F5F794BCBDE8FC4155
:10CF900056A0F5F78FBCBDE8FC4157A0F5F78ABC59
:10CFA000BDE8FC4156A0F5F785BC14A0F5F70AF9D9
:10CFB0002088F5F7D9FF687F78B128210020F5F7A0
:10CFC000C7FF51A0F5F7FEF83A210020F5F7C0FFA2
:10CFD000BDE8FC4151A0F5F7F5B832212320F5F763
:10CFE000B7FFBDE8FC4152A0F5F7ECB86083FF1F26
:10CFF000A8CC0120AA83FF1FA883FF1F452D4D61E8
:10D00000726B6572B2E2CAD4000000003078000092
:10D01000AC83FF1F45525200544254005061737359
:10D020006976650041637469766500005553423244
:10D030002E300000555342332E3247656E310000CA
:10D04000555342332E3247656E32000055534234F9
:10D0500047656E3300000000323056003330560012
:10D060003430560035305600334100003541000061
:10D070007E316D007E326D007E336D007E346D003A
:10D080007E356D007E366D007E376D004550520056
:10D09000556E6B6E6F7700004875617765690000AB
:10D0A0005669766F000000004F50504F000000009E
:10D0B000476F6F676C650000485000004C656E6FED
:10D0C000766F00005869616F4D6900005A4D490044
:10D0D000536F75746843686970000000596943684C
:10D0E0006F6E67004170706C65000000496E6A6F7A
:10D0F000696E6963000000004C696E74657300001E
:10D1000048796E6574656B00CEB4B6C1C8A1B5BD73
:10D11000456D61726B6572D0C5CFA200C7EBB0B42C
:10D1200027C8B7C8CF27BCFCD6D8CAD40000000097
:10D13000B0B427C8B7C8CF27BCFCBDF8D0D0B2E286
:10D14000CAD400002DE9F0470024FB4FDFF8EC8340
:10D15000F888F978421802EB420208EB8202528802
:10D16000C2F30235DFF8D8A39AF800C0F54AA14609
:10D170001288561ED31FBCF1040F05D09AF800C0C8
:10D18000BCF1050F23D03BE0DFF8ACC3072A9CF8C5
:10D1900003C00CF1010C0CF0FF0C07D2B14202DA13
:10D1A00087F803C010E087F803900DE0062902D24B
:10D1B00087F803C008E0984204D187F80390A7F8E5
:10D1C000069001E0401CF8808AF8009018E0DFF833
:10D1D00068C3072A9CF803C0ACF1010C0CF0FF0CEB
:10D1E00005D211B187F803C008E0FE7006E011B166
:10D1F00087F803C002E060B3401EF8808AF8009010
:10D200000C20F5F7ABFE00210846F5F7A1FEDFF88C
:10D210003893B9F80000F5F7A7FECCA0F5F74AFB64
:10D22000F878F98808440421F5F74CFE00210A201B
:10D23000F4F742FEF888F978084400EB400008EB68
:10D2400080004088C00508D5C1480088F5F78CFEED
:10D2500007E00620F870FB80D0E7BE480088F5F7AD
:10D2600083FEF888F978084400EB400008EB800062
:10D270004088C10B71D000F01F001F285DD2DFE88D
:10D2800000F05C1014181C2024282C3034383C404A
:10D2900044484C50545C5C5C5C5C5C5C5C5C5C5C1E
:10D2A0005800ADA0F5F706FB38E1AEA0F5F702FB9C
:10D2B00034E1AEA0F5F7FEFA30E1AFA0F5F7FAFAE7
:10D2C0002CE1ABA0F5F7F6FA28E1AEA0F5F7F2FAFB
:10D2D00024E1ADA0F5F7EEFA20E1AEA0F5F7EAFA09
:10D2E0001CE1B0A0F5F7E6FA18E1B2A0F5F7E2FA12
:10D2F00014E1B4A0F5F7DEFA10E1B6A0F5F7DAFA1A
:10D300000CE1B7A0F5F7D6FA08E1B9A0F5F7D2FA23
:10D3100004E1BBA0F5F7CEFA00E1BCA0F5F7CAFA2C
:10D32000FCE0BDA0F5F7C6FAF8E0BEA0F5F7C2FA3A
:10D33000F4E0C0A0F5F7BEFAF0E0C2A0F5F7BAFA43
:10D34000F888F978084400EB400008EB80000421DD
:10D350004088F5F72BF9E1E0FFE76DB100F01F0021
:10D36000102870D2DFE800F0C08C9094989CA0A4A4
:10D37000A8ACB0B4B8C0C0BC00F01F00192870D26F
:10D38000DFE800F06F0D1115191D2125292D31350C
:10D39000393D4145494D5155595D62666A00AAA023
:10D3A000F5F788FAAEE0AAA0F5F784FAAAE0AAA0F9
:10D3B000F5F780FAA6E0AAA0F5F77CFAA2E0AAA009
:10D3C000F5F778FA9EE0AAA0F5F774FA9AE0AAA019
:10D3D000F5F770FA96E0ABA0F5F76CFA92E0ADA025
:10D3E000F5F768FA8EE0ADA0F5F764FA8AE0ADA033
:10D3F000F5F760FA86E0AEA0F5F75CFA82E0AEA041
:10D40000F5F758FA7EE0AFA0F5F754FA7AE0B0A04D
:10D41000F5F750FA76E0B2A0F5F74CFA72E0B3A057
:10D42000F5F748FA6EE0B5A0F5F744FA6AE0B6A061
:10D43000F5F740FA66E0B6A0F5F73CFA62E0B8A06E
:10D44000F5F738FA5EE04FE0BAA0F5F733FA59E0A5
:10D45000BCA0F5F72FFA55E0BEA0F5F72BFA51E086
:10D46000FFE778A0F5F726FAF888F978084400EB8A
:10D47000400008EB800004214088F5F797F841E070
:10D4800066A0F5F717FA3DE0B6A0F5F713FA39E014
:10D49000B6A0F5F70FFA35E063A0F5F70BFA31E027
:10D4A000B4A0F5F707FA2DE0B6A0F5F703FA29E0E6
:10D4B000B6A0F5F7FFF925E0B9A0F5F7FBF921E0F3
:10D4C000BAA0F5F7F7F91DE0BBA0F5F7F3F919E0FD
:10D4D000BCA0F5F7EFF915E09FA0F5F7EBF911E027
:10D4E000BBA0F5F7E7F90DE056A0F5F7E3F9F888EA
:10D4F000F978084400EB400008EB800004214088E4
:10D50000F5F754F8F888F978084400EB400018F86B
:10D510002000E02802D2B2A0F5F7CCF94DB1012DE0
:10D5200008D00021B04AFE78AE481388FA88324409
:10D53000CDE15BE169E10000208FFF1F74B9FF1F9F
:10D540006083FF1F7083FF1FAA83FF1F4E3A0000F6
:10D55000AC83FF1FA883FF1F5352435F4341505FBB
:10D560004558000053746174757300004765745F1B
:10D570004261745F434150004765745F4261745F6C
:10D58000535441004765745F4D616E75665F496E27
:10D59000666F000053656375726974795F526571D7
:10D5A0000000000053656375726974795F5265739A
:10D5B000700000004669726D5F5570645F5265715E
:10D5C000000000004669726D5F5570645F526573BC
:10D5D000700000005050535F537461747573000005
:10D5E000436F756E7472795F496E666F000000005C
:10D5F000436F756E7472795F436F646573000000EA
:10D6000053696E6B5F4341505F45580045585F4317
:10D610006F6E74726F6C00004550525F5352435FDF
:10D62000434150004550525F53696E6B5F43415018
:10D630000000000056656E645F446566696E5F4574
:10D640005800000030780000476F6F644352430079
:10D65000476F746F4D696E004163636570740000BD
:10D6600052656A656374000050696E6700000000CF
:10D6700050535F52445900004765745F5352435FF3
:10D68000436170004765745F53696E6B5F436170FF
:10D690000000000044525F537761700050525F53A6
:10D6A0007761700056434F4E4E5F537761700000B4
:10D6B0005761697400000000536F66745F526573B0
:10D6C00065740000444154415F5265736574000005
:10D6D000444154415F52657365745F4F4B000000D5
:10D6E0004E6F745F537570706F7274004765745F2E
:10D6F0005352435F4361705F455800004765745F54
:10D70000537461747573000046525F537761700003
:10D710004765745F5050535F5374617475730000B4
:10D720004765745F436F756E7472795F436F6465AC
:10D73000000000004765745F53696E6B5F43617062
:10D740005F4558004765745F5352435F494E464FEB
:10D75000000000004765745F5265766973696F6EFB
:10D76000000000005265717565737400424953549E
:10D7700000000000426174746572795F53746174D3
:10D7800075730000416C6572740000004765745F3A
:10D79000436F756E7472795F496E666F00000000AA
:10D7A000456E7465725F5553420000004550525FEC
:10D7B00052657175657374004550525F4D6F6465B5
:10D7C000000000005352435F496E666F0000000086
:10D7D00056656E646F725F446566696E65640000CD
:10D7E0002A000000288E01207283FF1F0E21522084
:10D7F000F5F7AEFBA0A0F5F75DF800210420F4F7E3
:10D800005BFB9EA0F5F756F863E00A215220F5F77E
:10D810009FFBAFF2D010F5F74DF8F888F97808447F
:10D8200000EB400008EB800008214068F4F7BEFEE2
:10D83000F888F978084400EB400008EB8000808805
:10D8400084B246E01CD10A215220F5F781FBAFF2E9
:10D850000C20F5F72FF8F888F978084400EB400021
:10D8600008EB800008214068F4F7A0FEF888F978FA
:10D87000084400EB400008EB8000808884B228E078
:10D8800000EB4116B6F800C062451ED1002414E03A
:10D89000601C824600EB80004006010E5220F5F726
:10D8A00057FBAFF26020F5F705F806EB840008217E
:10D8B0004068F4F77BFE0AF0FF04AC42E8D36D1E2B
:10D8C00006EB8500808884B203E0491C89B2994246
:10D8D000B8D9B9F80000F5F747FB0E210020F5F79D
:10D8E00037FB68A0F4F7E6FFAFF2A820F4F7E2FFF9
:10D8F000F888F978084400EB400008EB8000042128
:10D900004088F4F753FE19210020F5F721FB5EA0B3
:10D91000F4F7D0FFF888F978084400EB400008EBF2
:10D92000800001218078C0F38110401CF5F7CAFA0D
:10D9300024210020F5F70CFB56A0F4F7BBFFF88874
:10D94000F978084400EB400008EB80000121408892
:10D95000C0F34220F5F7B6FA00210820F4F7ACFA3C
:10D96000F888F978084400EB4000022118F82000FC
:10D97000F4F71CFE2F210020F5F7EAFAF888F97871
:10D98000084400EB400018F82010E0290DD308EB04
:10D9900080004088000AC00703D03FA0F4F78AFF48
:10D9A00010E03EA0F4F786FF0CE008EB8000408812
:10D9B000000AC00703D03AA0F4F77CFF02E037A0CA
:10D9C000F4F778FF00210820F4F776FAF888F97860
:10D9D000084400EB400008EB800080784009C00755
:10D9E00003D030A0F4F766FF02E02FA0F4F762FF47
:10D9F000F888F978084400EB400008EB8000408884
:10DA0000C00B36D03A210020F5F7A2FA27A0F4F790
:10DA100051FFAFF2D030F4F74DFF04212046F4F768
:10DA2000C5FD45210020F5F793FAE00B03D021A0B6
:10DA3000F4F740FF02E020A0F4F73CFF00210420AF
:10DA4000F4F73AFAAFF2FC40F4F734FF0021C4F3E4
:10DA5000C320F5F737FA00210420F4F72DFA17A0B8
:10DA6000F4F728FFC4F30800BDE8F0470021F5F7FC
:10DA700029BABDE8F08700004E4F00004461746190
:10DA800000000000483A000056657273696F6E3AF4
:10DA90000000000049443A0053524300534E4B00EB
:10DAA0004361620044465000554650004558483A8C
:10DAB000000000004300000055430000533A0000FE
:10DAC0002DE9FC5FDFF8E49399F800B0F848F94DD0
:10DAD0004FF0010C0088EA78431EC41FE988DEB2CB
:10DAE0004FF0060AA7B24FF00008BBF1040F11D0A7
:10DAF00099F800B0BBF10A0F0CD099F80040052C42
:10DB00002FD099F800400B2C2BD099F80010062943
:10DB100043D04AE085F8028070B1DFF898C3072847
:10DB20009CF803C00CF1010C0CF0FF0C0AD29A42D5
:10DB300005DA85F803C038E085F802C035E085F8DD
:10DB4000038032E0062A02D285F803C02DE0A1420C
:10DB500004D185F80380A5F8068026E0491CE980F9
:10DB600023E085F8028040B1D24CE478641EE4B230
:10DB7000072807D222B1EC7017E085F802C014E044
:10DB8000EE7012E00AB1EC700FE011B1491EE980AD
:10DB90000BE085F803A0EF8007E030B1C64A122100
:10DBA000117085F8028089F8008099F80010042926
:10DBB00003D099F80010052901D189F80080A978CF
:10DBC00041B1062B01D2EE7004E0072802D3EF80AA
:10DBD00085F803A00C20F5F7C1F900210846F5F7F8
:10DBE000B7F9DFF8D892B9F80000F5F7BDF9B4A09D
:10DBF000F4F760FE00210420F4F75EF9B1A0F4F719
:10DC000059FEB24800210068F5F75CF9DFF8C0B2B0
:10DC10000C240023BBF80000CDE90004ADA2194696
:10DC20006620F5F7A7F9DFF8B0A20023ABA2BAF897
:10DC30000000CDE9000419468220F5F79BF9FF2486
:10DC4000B9F80000CDE900049E224F2300211046C0
:10DC5000F4F764F9964E3088012820D9401E00EE72
:10DC6000100AB8EEC00A9FED9E1AE878E988C1EE66
:10DC7000000A084400EE100A9F220021B8EE400A74
:10DC800020EE800ABCEEC00A10EE100A83B2B9F88A
:10DC90000000CDE900049D20F4F740F909E0B9F84F
:10DCA0000000CDE900044F239F2200219D20F4F7BE
:10DCB00035F93088072802D200F0FF0801E04FF064
:10DCC00007080024874E66E2B9F80000F5F74CF922
:10DCD000671C07EB8700FF2101EB4000C1B2002069
:10DCE000F5F736F9E88804212044F5F7EBF8E888E1
:10DCF000204400EB400006EB80004088C00504D5BE
:10DD0000BBF80000F5F730F903E0BAF80000F5F7CA
:10DD10002BF900210220F4F7CFF8E878844203D1F0
:10DD200071A0F4F7C7FD03E000210C20F4F7C4F85C
:10DD3000E888204400EB400006EB8000007A0128D0
:10DD400024D000210720F4F7B7F8E888204400EB3E
:10DD5000400006EB80004088C0F30231C20B74D053
:10DD600000F01F001F2861D2DFE800F06014181CCB
:10DD70002024282C3034383C4044484C50545860BF
:10DD8000606060606060606060605C0057A0F4F795
:10DD900091FDDAE756A0F4F78DFDF0E157A0F4F716
:10DDA00089FDECE157A0F4F785FDE8E158A0F4F710
:10DDB00081FDE4E154A0F4F77DFDE0E157A0F4F724
:10DDC00079FDDCE156A0F4F775FDD8E157A0F4F732
:10DDD00071FDD4E159A0F4F76DFDD0E15BA0F4F73B
:10DDE00069FDCCE15DA0F4F765FDC8E15FA0F4F743
:10DDF00061FDC4E160A0F4F75DFDC0E162A0F4F74D
:10DE000059FDBCE164A0F4F755FDB8E165A0F4F755
:10DE100051FDB4E166A0F4F74DFDB0E167A0F4F761
:10DE200049FDACE169A0F4F745FDA8E16BA0F4F76A
:10DE300041FDE8880421204400EB400006EB80000F
:10DE40004088F4F7B3FB9AE1FFE769B100F01F00E7
:10DE5000102828D2DFE800F027EFEEEDECEBEAE93E
:10DE6000E8E7E6E5E427272900F01F0019281BD280
:10DE7000DFE800F01A0D1115C2C6CACED2F2F6FACA
:10DE8000FEEDECEBEAE9E8E7E6E5E4E3E20054A0C6
:10DE9000F4F710FD73E154A0F4F70CFD6FE154A00A
:10DEA000F4F708FD6BE15CE116E156E16083FF1FCA
:10DEB0007083FF1F208FFF1FB183FF1FAA83FF1FE7
:10DEC000504400005061636B733A00007883FF1F79
:10DED000AC83FF1F53524300A883FF1F534E4B00D8
:10DEE00000009E4274B9FF1F3E000000A1CC00005C
:10DEF0005352435F4341505F45580000537461746F
:10DF0000757300004765745F4261745F4341500060
:10DF10004765745F4261745F535441004765745FA5
:10DF20004D616E75665F496E666F0000536563757F
:10DF3000726974795F526571000000005365637502
:10DF4000726974795F526573700000004669726D82
:10DF50005F5570645F526571000000004669726D24
:10DF60005F5570645F526573700000005050535FDE
:10DF70005374617475730000436F756E7472795FCA
:10DF8000496E666F00000000436F756E7472795FB2
:10DF9000436F64657300000053696E6B5F434150CB
:10DFA0005F45580045585F436F6E74726F6C000098
:10DFB0004550525F5352435F434150004550525FBA
:10DFC00053696E6B5F4341500000000056656E64FC
:10DFD0005F446566696E5F45580000003078000058
:10DFE000476F6F6443524300476F746F4D696E0013
:10DFF000416363657074000069A0F4F75BFCBEE0E8
:10E0000069A0F4F757FCBAE069A0F4F753FCB6E056
:10E0100069A0F4F74FFCB2E06AA0F4F74BFCAEE065
:10E0200097E092E08DE088E083E07EE079E074E0C4
:10E030006EE069E064E05EE04AE045E040E03BE03D
:10E0400036E031E02CE027E022E01DE018E013E0AC
:10E050000EE009E004E0FFE75EA0F4F72BFC8EE0A1
:10E060005EA0F4F727FC8AE05EA0F4F723FC86E0CC
:10E070005FA0F4F71FFC82E05FA0F4F71BFC7EE0DA
:10E0800060A0F4F717FC7AE061A0F4F713FC76E0E7
:10E0900063A0F4F70FFC72E064A0F4F70BFC6EE0F1
:10E0A00066A0F4F707FC6AE067A0F4F703FC66E0FB
:10E0B00067A0F4F7FFFB62E069A0F4F7FBFB5EE00A
:10E0C0006CA0F4F7F7FB5AE06EA0F4F7F3FB56E010
:10E0D00070A0F4F7EFFB52E0AFF20010F4F7EAFBA8
:10E0E000E8880421204400EB400006EB80004088D3
:10E0F000F4F75CFA43E0AFF24410F4F7DBFB3EE0E8
:10E1000068A0F4F7D7FB3AE068A0F4F7D3FB36E059
:10E11000AFF25410F4F7CEFB31E066A0F4F7CAFB7F
:10E120002DE068A0F4F7C6FB29E068A0F4F7C2FB75
:10E1300025E06BA0F4F7BEFB21E06CA0F4F7BAFB7E
:10E140001DE06DA0F4F7B6FB19E06EA0F4F7B2FB8A
:10E1500015E051A0F4F7AEFB11E06DA0F4F7AAFBB7
:10E160000DE0AFF28810F4F7A5FBE8880421204405
:10E1700000EB400006EB80004088F4F717FAE888CF
:10E18000204400EB400016F82000E02802D264A0F2
:10E19000F4F790FBFCB24445FFF496ADBDE8FC9F5C
:10E1A00052656A656374000050696E670000000084
:10E1B00050535F52445900004765745F5352435FA8
:10E1C000436170004765745F53696E6B5F436170B4
:10E1D0000000000044525F537761700050525F535B
:10E1E0007761700056434F4E4E5F53776170000069
:10E1F0005761697400000000536F66745F52657365
:10E2000065740000444154415F52657365740000B9
:10E21000444154415F52657365745F4F4B00000089
:10E220004E6F745F537570706F7274004765745FE2
:10E230005352435F4361705F455800004765745F08
:10E24000537461747573000046525F5377617000B8
:10E250004765745F5050535F537461747573000069
:10E260004765745F436F756E7472795F436F646561
:10E27000000000004765745F53696E6B5F43617017
:10E280005F4558004765745F5352435F494E464FA0
:10E29000000000004765745F5265766973696F6EB0
:10E2A0000000000052657175657374004249535453
:10E2B00000000000426174746572795F5374617488
:10E2C00075730000416C6572740000004765745FEF
:10E2D000436F756E7472795F496E666F000000005F
:10E2E000456E7465725F5553420000004550525FA1
:10E2F00052657175657374004550525F4D6F64656A
:10E30000000000005352435F496E666F000000003A
:10E3100056656E646F725F446566696E6564000081
:10E320002A000000034900200870034910200870EB
:10E33000704700006083FF1FB183FF1F2DE9F04786
:10E340002DED028B0C20F4F709FED7480088F4F776
:10E350000BFE00210846F4F7FBFDDFF850A39AF806
:10E36000190001281BD09AF81A00E0B1D0A0F4F7E8
:10E37000A1FAD14E96F8280096F8291008440021F9
:10E38000F4F7A0FD00212B20F4F7E2FDDFF82C8349
:10E3900098F8080001280AD002282AD06DE0C8A009
:10E3A000F4F788FAE5E7C7A0F4F784FAE1E7C7A035
:10E3B000F4F780FA98F800000221F4F783FDC5A075
:10E3C000F4F778FAC4A0F4F775FA00210820F3F7FF
:10E3D00073FD98ED010A0221BDEEC00A10EE100A8D
:10E3E000F4F770FDBBA0F4F765FABCA0F4F762FA8D
:10E3F00043E0BBA0F4F75EFAB8F80A009FEDBA8BD1
:10E40000B0F5FA7F12D2BAA0F4F754FAB8F80A00BD
:10E41000F2F76CF953EC182BF2F787F8F2F7D0F912
:10E4200000EE100A0220F4F7DBFC0CE0F2F75EF9D4
:10E4300053EC182BF2F779F8F2F7C2F900EE100A54
:10E440000220F4F7CDFCA4A0F4F734FA0021082050
:10E45000F3F732FDA6A0F4F72DFA98F80C0000EEC1
:10E46000100AB8EE400ADFEDA30A022020EE200ACF
:10E47000F4F7B6FC99A0F4F71DFA98F80800032801
:10E4800020D19DA0F4F716FA98F800000221F4F7C5
:10E4900019FD90A0F4F70EFA8FA0F4F70BFA002103
:10E4A0000820F3F709FD98ED010A0221BDEEC00A2C
:10E4B00010EE100AF4F706FD86A0F4F7FBF987A02A
:10E4C000F4F7F8F90A210020F4F742FD0025DFF8FF
:10E4D0003092DCE006EB850494ED0B0AD4ED150ACE
:10E4E00020EE200AD6ED3D0AB4EEE00AF1EE10FA75
:10E4F00001DD86ED3D0A98F81900A84204D1814853
:10E500000088F4F731FD03E07F480088F4F72CFD24
:10E510006F1C07EB87004006010E0020F4F718FD82
:10E52000354495F8F800012806D0022829D00328A0
:10E5300027D004287DD0A9E094ED0B0A0220F4F73F
:10E540004FFC65A0F4F7B6F900210720F3F7B4FCFF
:10E5500094ED150A0220F4F743FC60A0F4F7AAF941
:10E5600000210720F3F7A8FC94ED0B0AD4ED150A5F
:10E57000022020EE200AF4F733FC64A0F4F79AF9A5
:10E5800084E094ED330A0220F4F72AFC60A0F4F74B
:10E5900091F994ED290A0220F4F722FC4EA0F4F739
:10E5A00089F900210720F3F787FC94ED150A022072
:10E5B000F4F716FC49A0F4F77DF900210720F3F7E2
:10E5C0007BFC95F8020120B394ED290AD4ED150ADD
:10E5D00060EE200A96ED3D0AF4EEC00AF1EE10FA64
:10E5E00017D39AF81900012813D010EE100A4845E5
:10E5F00002DA0120F4F7F4FB96ED3D0A10EE100A62
:10E60000484502DB0020F4F7EBFB40A0F4F752F999
:10E610003CE094ED290AD4ED150A20EE200A10EE14
:10E62000100A484502DA0120F4F7DAFB94ED290AD2
:10E6300000E00BE0D4ED150A20EE200A10EE100ADF
:10E640004845E2DB0020F4F7CBFBDEE794ED330A2C
:10E650000220F4F7C5FB2EA0F4F72CF994ED290A5B
:10E660000220F4F7BDFB1CA0F4F724F900210720D9
:10E67000F3F722FC96ED3D0A0021BDEEC00A10EE34
:10E68000100AF4F71FFC21A0F4F714F9FDB296F874
:10E69000280096F829100844A8423FF61BAFBDECAD
:10E6A000028BBDE8F0870000AC83FF1FA8CC0120DF
:10E6B0004550523A0000000068B8FF1FC8B6FF1F5F
:10E6C0004D493A0050444F3A000000004649583A3C
:10E6D000000000002E303000560000004100000015
:10E6E0005050533A000000007B14AE47E17A943F4B
:10E6F00030000000CDCC4C3D5661723A0000000065
:10E700000000C842A883FF1FAA83FF1F5700000014
:10E710007E0000002DE9FC5F00F028FA0C20F4F7E1
:10E720001DFCF94C2088F4F71FFC00210846F4F783
:10E730000FFCDFF8D8A39AF81900012820D09AF826
:10E740001A0008B3F2A0F4F7B5F8F34F97F82800D1
:10E7500097F8291008440021F4F7B4FB00212D207C
:10E76000F4F7F6FBED49EE4D91ED000A10EE100ABC
:10E77000A8420DDA032091ED000AF4F731FB0CE01A
:10E78000E8A0F4F797F8E0E7E7A0F4F793F8DCE700
:10E79000022091ED000AF4F723FBE5A0F4F78AF8D4
:10E7A00000210820F3F788FBE24991ED000A10EE02
:10E7B000100AA84205DA032091ED000AF4F710FBD5
:10E7C00004E0022091ED000AF4F70AFBDAA0F4F766
:10E7D00071F8DFF8688398F80000D94E4FF00C0507
:10E7E0003178084208D02088CDE900050023D5A261
:10E7F00019468A20F4F7BEFB98F800003178884368
:10E8000008D02088CDE900050023CFA219468A2030
:10E81000F4F7B0FB307898F80010884308D02088CF
:10E82000CDE900050023C8A219468A20F4F7A2FB0F
:10E8300098F8000050B9307840B92088CDE900053B
:10E840000023C0A219468A20F4F794FB0A21002075
:10E85000F4F77EFB97F8280097F82910084407285A
:10E8600001D9072600E0C6B20024DFF8E0B2DFF8E5
:10E87000E092DFF8E08211E198F80100204407EB14
:10E88000800090ED0B0AD0ED150A20EE200AD7ED9E
:10E890003D0AB4EEE00AF1EE10FA01DD87ED3D0A23
:10E8A000651C05EB85004006010E0020F4F750FBC7
:10E8B000A948007EA04207D1A8480088F4F754FB7D
:10E8C000A0A0F3F7F7FF03E0BBF80000F4F74CFB60
:10E8D00098F801002044C11991F8F810012906D0D8
:10E8E000022935D0032933D004297DD0D5E007EBA8
:10E8F000800090ED0B0A0220F4F772FA8CA0F3F777
:10E90000D9FF00210720F3F7D7FA98F80100204437
:10E9100007EB800090ED150A0220F4F761FA86A05B
:10E92000F3F7C8FF00210720F3F7C6FA98F80100B3
:10E93000204407EB800090ED0B0AD0ED150A022071
:10E9400020EE200AF4F74CFA85A0F3F7B3FFA4E019
:10E9500007EB800090ED330A0120F4F741FA81A023
:10E96000F3F7A8FF98F80100204407EB800090ED32
:10E97000290A0120F4F734FA6DA0F3F79BFF002178
:10E980000720F3F799FA98F80100204407EB80007C
:10E9900090ED150A0220F4F723FA67A0F3F78AFF37
:10E9A00000210720F3F788FA98F801002044C119E4
:10E9B00091F8021141B307EB800191ED290AD1EDE5
:10E9C000150A60EE200A97ED3D0AF4EEC00AF1EE5A
:10E9D00010FA19D39AF81910012915D010EE100A5F
:10E9E000484504DA012000E030E0F4F7F9F997ED4A
:10E9F0003D0A10EE100A484502DB0020F4F7F0F95A
:10EA000057A0F3F757FF48E007EB800090ED290A85
:10EA1000D0ED150A20EE200A10EE100A484502DA61
:10EA20000120F4F7DDF998F80100204407EB80009D
:10EA300090ED290AD0ED150A20EE200A10EE100AFA
:10EA40004845DDDB0020F4F7CBF9D9E707EB800080
:10EA500090ED330A0220F4F7C3F942A0F3F72AFF3E
:10EA600098F80100204407EB800090ED290A02206D
:10EA7000F4F7B6F92EA0F3F71DFF00210720F3F7F6
:10EA80001BFA97ED3D0A0021BDEEC00A10EE100AF8
:10EA9000F4F718FA32A0F3F70DFFECB2B442FFF42A
:10EAA000EBAEFF24BBF80000CDE900049E224F230B
:10EAB00000211046F3F732FA17F8280F9FED2A1AB3
:10EAC00079789F220844401E00EE100A224898F8E8
:10EAD0000110B8EEC00A007E0844C1EE000A00EE44
:10EAE000100A0021B8EE400A20EE800ABCEEC00AEF
:10EAF00010EE100A83B2BBF80000CDE900049D209F
:10EB0000F3F70CFABDE8FC9FAC83FF1FA8CC0120F3
:10EB10004550523A0000000068B8FF1F3483FF1FC1
:10EB2000000020414D493A0050444F3A0000000097
:10EB3000560000003C83FF1F410000003083FF1F90
:10EB4000A683FF1F3E0000003C000000AA83FF1FB9
:10EB50000000C842208FFF1FC8B6FF1FA883FF1FF9
:10EB6000570000007E00000000009E422DE9F041A9
:10EB70002A4CA07B032801D10120A073284E96F8CF
:10EB800000802848DFF8A0C00027417800784518A9
:10EB90002248EB1F6A1E007E9CF80110B8F1040F9A
:10EBA00015D096F80080B8F1050F24D03278062AE7
:10EBB0000BD10844C0B26076F8F70EF994F834002F
:10EBC00010B11A49092008703770BDE8F0818242FF
:10EBD00004DD062802D2401C20760AE08B4201D0D8
:10EBE000824203D127768CF8017002E0491C8CF830
:10EBF00001103770E9E710B1401E207603E021B123
:10EC0000491E8CF801103770DFE7072D04D9062064
:10EC100020768CF80130F6E72276F4E7C8B6FF1FBD
:10EC20006083FF1F90B8FF1F208FFF1FB183FF1F5E
:10EC3000034900200870034908200870704700004D
:10EC40006083FF1FB183FF1F2DE9FC4100F0A4F892
:10EC50001020F4F783F942480088F4F785F9002181
:10EC60000846F4F775F93FA0F3F7ACFA0024DFF893
:10EC700004813F4FA8F254453888F4F775F9601CB9
:10EC800006460007010E0020F4F762F9687C844212
:10EC900012D101210020F3F70FF90C20F4F75EF9EF
:10ECA00035480088F4F760F934A0F3F703FE4FF01D
:10ECB000FF310020F3F700F91020F4F74FF904EBCF
:10ECC000C40058F83000F3F77DFA34B1012C0ED0AF
:10ECD000022C14D0032C23D11AE0A87C18B128A050
:10ECE000F3F770FA1CE028A0F3F76CFA18E00021A3
:10ECF000E87CF4F7E7F826A0F3F7DCFD10E002204B
:10ED000095ED120AF4F76CF821A0F3F7D3FD07E0B4
:10ED1000022095ED130AF4F763F81EA0F3F7CAFD7D
:10ED2000F4B2042CA8D3FF243888CDE900049E2235
:10ED30004F2300211046F3F7F1F83888CDE900049D
:10ED4000687C9F2200EB800101EBC000012101EBF8
:10ED5000400300219D20F3F7E1F8BDE8FC810000AD
:10ED6000AC83FF1F5044D3D5C6ADC9E8D6C300005D
:10ED7000AA83FF1F0488FF1FA883FF1F3E00000017
:10ED80005050532F415653004649582F455052007A
:10ED900056000000410000002DE9F041574D2A784F
:10EDA00001279FED571ADFED571A9FED572A574C51
:10EDB0000026042AE07C94ED120AD4ED130A617C4B
:10EDC0000FD02A780A2A0CD02A78052A34D02A783B
:10EDD0000B2A31D02A78062A59D02878092879D0E8
:10EDE0007FE031B1012906D0022909D0032978D169
:10EDF00018E0A77475E0242873D2401CE07470E01A
:10EE000010EE100A424988426BDA28780A2804D0AA
:10EE100030EE210A84ED120A63E030EE010A84ED3F
:10EE2000120A5EE010EE900AB0F1824F59DA30EE2D
:10EE3000820A84ED130A54E031B1012906D0022977
:10EE400009D003294DD118E0A6744AE0052848D915
:10EE5000401EE07445E010EE100A2E49884240DD65
:10EE600028780B2804D030EE610A84ED120A38E0CD
:10EE700030EE410A84ED120A33E010EE900A264982
:10EE800088422EDD30EEC20A84ED130A29E0491CC7
:10EE9000C9B26174042924D1217811BB03216174A2
:10EEA0001E49A27CCA7108720920F8F74DFF94ED43
:10EEB000130A0D20F8F748FFF8F7FCFE1848016820
:10EEC000A26B891AB1F5487F0BD927700068A0633F
:10EED00007E0FFE711B1491E617401E01120607085
:10EEE0002E702878062805D02878052802D02878A2
:10EEF000042800D12E70BDE8F08100006083FF1F60
:10EF0000CDCCCC3D0AD7A33CCDCC4C3DB083FF1F2C
:10EF100000001042333353408FC2753DF862022027
:10EF20007C83FF1F2DE9F04F2DED048B85B0DFF8BA
:10EF30000084B8F8040000EBC009FE4B03EB890025
:10EF400090F8211001297CD1D8F80810491CC8F884
:10EF5000081090F820604246F74CB2F800C0012536
:10EF60000CEB4C0204EB820A012E04D18AF8085003
:10EF7000491CC8F80810EF4911F82930EE4901F88A
:10EF800022304188AAF802104188C1F30232418838
:10EF9000E74B5FEAD13BEA4FB3F802E00EF1010123
:10EFA00089B20491198801F1010189B20391E34901
:10EFB00001EB4E139FEDE39ADFEDE38A9FEDE38AC9
:10EFC000DFEDE39AE349E44CE44E91F82810029116
:10EFD000A17B7DD0012A05D0BEF5FA7F19D24FF072
:10EFE00000090FE04368CAF8043012E000EB890A18
:10EFF000DAF804A003EB890BCBF804A009F10109AE
:10F0000009F0FF099145F1D3A3F800C0049BA8F8CB
:10F01000023042F20F739C4502D2039BA8F80030E5
:10F02000521E00EB82035B681FFA83F9438803F0EA
:10F030001F03102B7ED0112B7DD14088C0057BD5BE
:10F0400000E0FDE319F4F04F76D0C24880F82920A3
:10F05000DDF808A003E1B8F80420AAEB000002EBF9
:10F06000C203B44A02EB830202EB8000406841F81D
:10F070002A00820F03D0C243920F2ED0EBE001EBA7
:10F080000A0080F8F85051F82A0001EB8A01C0F319
:10F09000892200EE102AB8EE400A20EE280A81EDFF
:10F0A0000B0AC0F3090000EE900AF8EE600A60EE69
:10F0B000880AC1ED150AF87900280DD1387A00EEDA
:10F0C000900AF8EE600AB4EEE00AF1EE10FA00E001
:10F0D000F2E001D884F81AA0BDE0C00053D501EBDE
:10F0E0000A02042002F8F80F51F82A0001EB8A0BFB
:10F0F000C0F3484300EE103AB8EE400A20EE090A89
:10F100008BED290AC0F3072100EE101AB8EE400A71
:10F1100020EE090A8BED330A9072F879012831D17B
:10F120000920F8F7B7FDDBED330AB4EEE00AF1EEA3
:10F1300010FA02E0BBE0ACE09AE023DB0920F8F72C
:10F14000A9FDDBED290AB4EEE00AF1EE10FA19D8B8
:10F1500084F81AA00920F8F79DFD30EE080ADFEDCB
:10F16000800A80EE201ABCEEC10A10EE100A6081FF
:10F170000D20F8F78FFDC0EE280ABCEEE00A10EE75
:10F18000100A207367E001EB0A00032200F8F82F51
:10F1900051F82A20C2F3C062827251F82A0001EBB2
:10F1A0008A0BC0F3474200EE102AB8EE400A20EE68
:10F1B000090A8BED290AC0F3072100EE101AB8EEF8
:10F1C000400A20EE090A8BED330AC0B200EE100AA5
:10F1D000B8EE400A20EE280A8BED150AF8790128CE
:10F1E00039D10920F8F756FDDBED330AB4EEE00A19
:10F1F000F1EE10FA2FDB0920F8F74CFDDBED290AC0
:10F20000B4EEE00AF1EE10FA25D8207B58B10D20BB
:10F21000F8F740FDDBED150A70EE880AB4EEE00A5F
:10F22000F1EE10FA17D884F81AA00920F8F732FD89
:10F2300070EE080A80EEA90ABCEEC00A10EE100AB1
:10F2400060810D20F8F726FDC0EE280ABCEEE00A2A
:10F2500010EE100A20730AF1010A0AF0FF0A3D4974
:10F2600091F8280091F82920024452453FF6F3AE68
:10F27000B07E01280DD1A07B0128FBD1B07F48B919
:10F28000C9F30801182905D9F7F750FDB07F401CD4
:10F29000B0776EE00128FCD1A07EF7F79DFDA07E3F
:10F2A0002076607625742F4800686062F6E30129B5
:10F2B000EFD10020A074F1E3DFF8A0B09BF817B005
:10F2C000CDF804B03AB1012A7ED0BEF5FA7F7CD2E7
:10F2D0004FF0000A14E142F20F72944502D2039AF1
:10F2E000A8F80020DFF84CC040881C4A00F01F0A34
:10F2F0001948137D927D477C807EBAF1110FC8D2E8
:10F30000DFE80AF0370937386A37793791373796A7
:10F3100037C73737E700B8F800000128B9D9811E90
:10F3200001EB4102044901EB82010A7A002A1BE049
:10F330007083FF1F00B7FF1F74B9FF1F288E0120C5
:10F34000F8620220CDCCCC3DCDCC4C3D0AD7233C3D
:10F350000AD7A33C68B8FF1FC8B6FF1FA8CC01207E
:10F36000CDCCCC3C7C83FF1F93D10D72401EA8F8FE
:10F37000000093E301298CD1707D012800D113B1E5
:10F38000012A04D005E03575F8F744FA86E30198C0
:10F3900010B1012A08D081E30020B075F57586F818
:10F3A0002050F7F715FA79E301980128E1D1002000
:10F3B000B075F075707E012808D0F9480068000229
:10F3C000D7D5F6F7FDFE69E38AE0A0E0F8F7DCF9AF
:10F3D0000C2086F8200061E30129CAD1012AC8D196
:10F3E0000021B175002FC4D1F7F7F6FCA07E20767E
:10F3F0006076657452E30129BBD117B1307E38B114
:10F400000EE0F7F7E9FCA07E20766076657407E0F1
:10F41000E4480078012803D93576F6F727FEB5755C
:10F420000020A0743AE30129A3D1F8F7ABFA35E341
:10F430004BB10020F6F74EFDDB48007801281CD0C8
:10F4400002281FD022E00020F6F744FDD6480078BD
:10F45000012802D0022805D008E025210220F8F773
:10F4600063FB03E01A210220F8F75EFBF8F7D2F9FC
:10F470003575CE480068A06210E305210220F8F738
:10F4800053FB03E00A210220F8F74EFB0020307501
:10F4900004E31CF82900DF2812D84FF400510220A1
:10F4A00000F020FC01288ED1C14C207800288AD0A1
:10F4B000C049002008700120F6F70CFD2570EDE230
:10F4C000012988D1BC48002101700020F6F702FD17
:10F4D000E4E201298ED1012A8CD10020B075DDE251
:10F4E0004368CAF8043012E000EB8A0BDBF804B082
:10F4F00003EB8A0ECEF804B00AF1010A0AF0FF0A03
:10F500009245F1D3A3F800C0049BA8F8023042F260
:10F510000F739C4502D2039BA8F80030DFF89CB221
:10F520004388DFF89CC203F01F034FF0020A102B40
:10F53000A2D2DFE803F0FD08FCFDFDFDFDFDFDFBB3
:10F54000FAFDFDFDFDF9964E86F82820002106E023
:10F5500000EB8102526846F82120491CC9B296F896
:10F5600028208A42F4D84FF00009C9E056F8290053
:10F57000810F29D0BAEB907F51D106EB090080F8BA
:10F58000F8A056F82900C0F3095100EE101A06EB56
:10F590008901B8EE400A20EE280A81ED290AC0F35D
:10F5A000892200EE102AB8EE400A20EE280A81EDEA
:10F5B000330AC0F3090000EE100AB8EE400A20EE4C
:10F5C000080A81ED150A97E006EB090080F8F8506B
:10F5D00056F82900C0F3892100EE101A06EB8901C4
:10F5E000B8EE400A20EE280A81ED0B0AC0F30900AC
:10F5F00000EE900AF8EE600A60EE880AC1ED150A86
:10F60000F879E8BB387A00EE900AF8EE600AB4EEBA
:10F61000E00AF1EE10FA6FD884F81A906CE0C0435B
:10F62000800F69D106EB0900032100F8F81F56F896
:10F630002910C1F3C061817256F8290006EB890BCD
:10F64000C0F3474100EE101AB8EE400A20EE090A56
:10F650008BED290AC0F3072100EE101AB8EE400A1C
:10F6600020EE090A8BED330AC0B200EE100AB8EEA4
:10F67000400A20EE280A8BED150AF879012800E0EF
:10F680003AE039D10920F8F705FBDBED330AB4EE97
:10F69000E00AF1EE10FA2FDB0920F8F7FBFADBEDB8
:10F6A000290AB4EEE00AF1EE10FA25D8207B58B111
:10F6B0000D20F8F7EFFADBED150A70EE880AB4EECC
:10F6C000E00AF1EE10FA17D884F81A900920F8F73A
:10F6D000E1FA70EE080A80EEA90ABCEEC00A10EE4C
:10F6E000100A60810D20F8F7D5FAC0EE280ABCEEAA
:10F6F000E00A10EE100A207309F1010909F0FF0970
:10F7000096F8280048453FF631AFA07B01280FD17D
:10F71000B8F8040000EBC001284800EB810090F825
:10F7200020000128F3D104E0DFE0B5E06BE00DE05C
:10F7300088E0607C30B1A07EF7F74EFBA07E20769B
:10F740006076ABE10020F7F747FBA7E14168C1F322
:10F7500002718CF8001009B14A1E6276104B5A18DB
:10F7600092F8F720012A04D0032A2BD0022A32D0A3
:10F7700094E12572491E03EB810191ED0B0ABCEE69
:10F78000C00A10EE101A21704068C0F3892000EE04
:10F79000100AB8EE400A20EE080A84ED010A7DE165
:10F7A00068B8FF1F2283FF1F2083FF1F7C83FF1F7A
:10F7B0002183FF1F2483FF1F2383FF1F00B7FF1F29
:10F7C0002583FF1F84F808A04168C1F34A216181A5
:10F7D0004068207362E103222272491E03EB81011B
:10F7E00091ED290ABCEEC00A10EE101A2170406893
:10F7F000C0F3892000EE100AB8EE400A20EE080A95
:10F8000084ED010A4AE10299B04B00291AD04168FF
:10F81000090F8CF80010072904D9029AC91F114456
:10F820008CF800109CF8001009B14A1E62765A1834
:10F8300092F8F720012A06D0032A1BD0042A00E000
:10F840003EE120D02AE12572491E03EB810191EDB2
:10F850000B0ABCEEC00A10EE101A21704068C0F30B
:10F86000892000EE100AB8EE400A20EE080A84ED66
:10F87000010A13E184F808A04168C1F34A216181BB
:10F88000406820730AE1042121724168C1F34A21D2
:10F8900061814068207301E14268BAEB126F01D1C7
:10F8A000012906D042680321B1EB126F15D1B5765C
:10F8B000F4E087480078012802D0022805D008E04B
:10F8C00001210320F8F730F903E002210320F8F7C3
:10F8D0002BF9804904200870E0E040680521B1EB75
:10F8E000106F01D10020B076D8E01BF82920A02AA3
:10F8F0007BD31BF82920DF2A77D84FF40051022050
:10F9000000F0F0F9012802D0F07E80B338E0B8F8BA
:10F91000040000EBC0000BEB800041684AF20102DA
:10F9200089B2914202D1F7F75DFCB7E0416889B234
:10F93000A1F50042023A11D0416889B2A1F5004216
:10F94000033A0ED0416889B2B1F5827F10D0406889
:10F9500080B2A0F521411F3906D09FE0F7F770FD76
:10F960009CE0F7F7CFFD99E0F7F7A8FE96E002E0FC
:10F97000F7F73EFE92E0317F11B9717F012905D082
:10F9800001281AD0307F01281ED087E0B8F8040083
:10F9900000EBC0000BEB8000416831608168716052
:10F9A000C268B2600269F26040693061480175D591
:10F9B0000120F7F775FFF57670E00220F7F770FF8A
:10F9C0000020F076357769E0B8F8040000EBC0005D
:10F9D0000BEB80008168C1F30341032906D08068E6
:10F9E000C0F303400B2804D005E007E00320F077C4
:10F9F00001E00420F077002030774FE0012902D1A8
:10FA0000019A012A02D0012940D047E096F820103F
:10FA1000022903D1826872840069B084708CA0F5D9
:10FA20001C52173A03D042F6013290422AD1B08CD0
:10FA3000A0F52440753814D0112806D007291CD011
:10FA400005292BD8F6F7C4FE28E00B2904D00A2993
:10FA500024D8F6F70BFC21E0F6F708FB7576B575B0
:10FA60001CE00B2904D00A2918D8F6F7FFFB15E093
:10FA7000F6F7FCFA7576B57510E0F6F7F7FA7576D5
:10FA8000B5750BE0F6F7F2FAB57507E0406880B29D
:10FA9000A0F52041023901D1F7F7CCF8B8F80400FD
:10FAA0000D4A00EBC00302EB8302002182F8211013
:10FAB000401C80B2A8F804000A2801D1A8F804105C
:10FAC00005B0BDEC048BBDE8F08F000068B8FF1FE7
:10FAD0002083FF1F2183FF1F00B7FF1F0449C87841
:10FAE000401CC0B2C870072801D90020C8707047F8
:10FAF0002083FF1F04490879401CC0B20871072801
:10FB000001D90020087170472083FF1F2DE9F041C3
:10FB10001D4E1E4C1E48B27B012500786168012AEB
:10FB20000BD0002914D16575012827D002280FD1E8
:10FB3000BDE8F0411821F7F7F7BF627D002A07D131
:10FB4000002905D1217D134F21B165753868B06258
:10FB5000BDE8F081012802D0022805D008E0252167
:10FB60000220F7F7E1FF03E01A210220F7F7DCFF9C
:10FB7000F7F77EFF65753868B062E9E7BDE8F041E8
:10FB800024210220F7F7D0BFC8B6FF1FA8CC012060
:10FB90002083FF1F7C83FF1F2DE9F041304F314C44
:10FBA000314D97F82000062807D1E86A28B121686E
:10FBB000081A2D2801D9F6F70BFE95F83400012814
:10FBC0000DD1287C58B9286A2168081A42F22831D8
:10FBD000884204D9687EF7F7FFF820682862287CFD
:10FBE00001280ED1686A2168091A40F2EE2081428C
:10FBF00007D9F6F78DFA206868620120A87420689A
:10FC00002863787D002601280FD1A86A2168081A88
:10FC100096280AD97E750020F7F742FE97F8210052
:10FC2000012802D1022087F82100A87B012808D1F1
:10FC3000A87C30B9E87C012803D1687EF7F7CCF8BE
:10FC4000EE74A87B012809D1A87C012806D1286B75
:10FC50002168081AB0F5FA7F00D9AE74BDE8F081CA
:10FC6000A8CC01207C83FF1FC8B6FF1F70B50546D6
:10FC70000C461F2D04D940F223110EA0F5F7A8FB66
:10FC800034B1012C04D04FF492710AA0F5F7A0FB17
:10FC900000F036FA124905F01F00012C06D00A8840
:10FCA00082430A8000F050F9002070BD0A880243A8
:10FCB0000A80F7E72E2E5C2E2E5C2E2E5C2E2E5CFC
:10FCC0002E2E5C6472697665725C7372635C686325
:10FCD0003332663436305F6770696F2E6300000020
:10FCE000F43B054070B505460C46002D0ED0012DA5
:10FCF0000CD0022D0AD0032D08D0042D06D0052DDE
:10FD000004D04FF4C8711CA0F5F762FB012C2AD077
:10FD1000022C28D0042C26D0082C24D0102C22D041
:10FD2000202C20D0402C1ED0802C1CD0B4F5807FFD
:10FD300019D0B4F5007F16D0B4F5806F13D0B4F5A8
:10FD4000006F10D0B4F5805F0DD0B4F5005F0AD01D
:10FD5000B4F5804F07D0B4F5004F04D040F29111B4
:10FD600005A0F5F735FB0F4800EB051000682040B3
:10FD700000D0012070BD00002E2E5C2E2E5C2E2E99
:10FD80005C2E2E5C2E2E5C6472697665725C7372DA
:10FD9000635C68633332663436305F6770696F2E38
:10FDA00063000000003805402DE9F04106460F468B
:10FDB00014460025002E0DD0012E0BD0022E09D0A6
:10FDC000032E07D0042E05D0052E03D0AC2152A05F
:10FDD000F5F7FEFA207838B1012805D0022803D0C3
:10FDE000AE214DA0F5F7F4FA607938B1012805D0BD
:10FDF000022803D0AF2148A0F5F7EAFAA07928B18C
:10FE0000012803D0B02144A0F5F7E2FA607828B1C8
:10FE1000012803D0B12140A0F5F7DAFAA07828B183
:10FE2000012803D0B2213CA0F5F7D2FAE07828B13E
:10FE3000012803D0B32138A0F5F7CAFA207928B1F8
:10FE4000012803D0B42134A0F5F7C2FAE07928B133
:10FE5000012803D0B52130A0F5F7BAFA00F050F927
:10FE6000012101FA05F038424CD0B001354A00EBCF
:10FE700085008318921C024494F801C018886CF322
:10FE80008E30188094F802C018886CF30C301880FB
:10FE900094F803C018886CF34920188094F804C0C3
:10FEA00018886CF38610188094F806C018886CF3D4
:10FEB0008200188094F805C018886CF3051018802B
:10FEC000207820B101280BD0022816D111E0188823
:10FED00020F400401880188820F0020018800CE000
:10FEE000188820F400401880188840F0020018801C
:10FEF00003E0188840F400401880E379108863F329
:10FF0000082010806D1CEDB2102DAAD300F01CF853
:10FF10000020BDE8F08100002E2E5C2E2E5C2E2EDF
:10FF20005C2E2E5C2E2E5C6472697665725C737238
:10FF3000635C68633332663436305F6770696F2E96
:10FF400063000000003C054002494FF42540088052
:10FF500070470000FC3B054070B504460D46002C80
:10FF60000ED0012C0CD0022C0AD0032C08D0042C6B
:10FF700006D0052C04D040F20F2105A0F5F728FA91
:10FF80000E4800EB041002882A430280002070BD56
:10FF90002E2E5C2E2E5C2E2E5C2E2E5C2E2E5C6465
:10FFA00072697665725C7372635C6863333266345F
:10FFB00036305F6770696F2E630000000A380540B5
:10FFC00070B504460D46002C0ED0012C0CD0022C2E
:10FFD0000AD0032C08D0042C06D0052C04D040F203
:10FFE000F71105A0F5F7F4F90E4800EB04100288AC
:10FFF0002A430280002070BD2E2E5C2E2E5C2E2EF9
:020000040002F8
:100000005C2E2E5C2E2E5C6472697665725C737257
:10001000635C68633332663436305F6770696F2EB5
:1000200063000000083805402DE9F0410646884687
:1000300015461F460024002E0ED0012E0CD0022E95
:100040000AD0032E08D0042E06D0052E04D04FF47B
:100050001A711FA0F5F7BCF975B1681E09280BD9F4
:100060000E2D09D00F2D07D01F381B2804D940F2C0
:10007000692117A0F5F7ACF937B1012F04D040F290
:100080006A2113A0F5F7A4F900F03AF80123B101B1
:100090001A4E03FA04F010EA080F0CD001EB8400AA
:1000A0003044028865F305020280012F0CD00288DB
:1000B00022F480720280641CE4B2102CE9D3FFF7B2
:1000C00043FF0020BDE8F081028842F48072F1E72E
:1000D0002E2E5C2E2E5C2E2E5C2E2E5C2E2E5C6424
:1000E00072697665725C7372635C6863333266341E
:1000F00036305F6770696F2E63000000023C054078
:1001000002494AF20150088070470000FC3B05405C
:100110002DE9F0412DED028B82B000F0C3F9C74804
:10012000C74F1C2490ED000AC64D10EE101AB942BC
:100130000BDA2988CDE90014002390ED000A04228F
:1001400019461846F3F780F90AE02988CDE900142A
:10015000002390ED000A032219461846F3F774F9BC
:100160002888CDE900040023B7A219465320F2F7EE
:1001700001FFB648DFF8D88290ED000A10EE101AA1
:10018000B9420CDAB8F80010CDE90014002390ED64
:10019000000A04221B211846F3F756F90BE0B8F8C1
:1001A0000010CDE90014002390ED000A03221B216A
:1001B0001846F3F749F9B8F80000CDE90004002328
:1001C000A4A21B215320F2F7D5FEA348A34E90ED25
:1001D000000A10EE101AB9420BDA3188CDE900148A
:1001E000002390ED000A042237211846F3F72CF97A
:1001F00023E090ED000A10EE101AB94212DB90EDE8
:10020000000A974A10EE101A91420BDA3188CDE9B4
:100210000014002390ED000A032237211846F3F75B
:1002200013F90AE03188CDE90014002390ED000AAB
:10023000022237211846F3F707F93088CDE9000488
:10024000002388A237215320F2F794FEFF20B8F84C
:100250000010CDE900104F23682200216720F1F73C
:100260005DFE3088F2F780FE02217720F2F770FE03
:100270001020F2F773FE7C4C207A04280CD07BA06F
:10028000F2F718FB7A480078072838D2DFE800F048
:10029000370810182028300076A0F2F70BFBF1E7A2
:1002A0002888F2F761FE19217520F2F751FE26E049
:1002B0002888F2F759FE19218320F2F749FE1EE043
:1002C0002888F2F751FE19218C20F2F741FE16E042
:1002D0003088F2F749FE2D217520F2F739FE0EE045
:1002E0003088F2F741FE2D218320F2F731FE06E03F
:1002F0003088F2F739FE2D218C20F2F729FE5EA01E
:10030000F2F7D8FA2888F2F72FFE17216C20F2F7BF
:100310001FFE608900EE100AB8EE400ADFED570AB2
:1003200020EE208A217A042907D100EE100AB8EEC7
:10033000400ADFED530A20EE208A18EE100AB84278
:100340000BDA50A0F2F7B6FA0220B0EE480AF2F744
:1003500047FD3DA0F2F7AEFA07E00220B0EE480AF2
:10036000F2F73EFD38A0F2F7A5FAB8F80000F2F770
:10037000FBFD2B216C20F2F7EBFD207B00EE100A39
:10038000B8EE400ADFED400A20EE208A3DA0F2F7E9
:1003900091FA0220B0EE480AF2F722FD2DA0F2F702
:1003A00089FA3088F2F7E0FD384F3878384D4FF051
:1003B00010042978084208D03088CDE900040023D1
:1003C00034A23F216A20F2F7D5FD38782978884396
:1003D00008D03088CDE9000400232FA23F216A20F5
:1003E000F2F7C8FD28783978884308D03088CDE9FD
:1003F0000004002328A23F216A20F2F7BBFD3878D1
:1004000050B9287840B93088CDE90004002321A2F2
:100410003F216A20F2F7AEFD40217C20F2F798FDE3
:100420001E49002091ED000AF2F7DAFC02B01CA090
:10043000BDEC028BBDE8F041F2F73CBA3483FF1FFC
:1004400000002041A883FF1F560000003C83FF1FCF
:10045000AA83FF1F410000004083FF1FAC83FF1FE2
:100460000000C84257000000C8B6FF1F505053009C
:10047000208FFF1F415653005F0000000AD7A33CA6
:10048000CDCCCC3C30000000CDCC4C3D3083FF1FA8
:10049000A683FF1F3E0000003C0000008483FF1F76
:1004A000A1E600002DE9F0410021484CDFF820C111
:1004B000207A9CF80020042807D0072A22D2DFE8FF
:1004C00002F02116181A1C1E2000072A1AD2DFE893
:1004D00002F019040619080A0C00282112E0042170
:1004E00010E014210EE002210CE001210AE032218B
:1004F00008E0052106E0012104E0142102E00221C8
:1005000000E00121334E96F800803048304FB8F1BA
:10051000040F037E7F7845891F44037BF8B211D016
:1005200037780A2F0ED096F800800127B8F1050F12
:1005300020D096F80080B8F10B0F1BD03078062839
:100540002FD036E0032A0AD8294489B26181A28AD1
:10055000914200D962816076F6F73EFC29E01944A9
:10056000C9B22173627B914200D922736076F6F79B
:1005700033FC1EE0042A0AD2691A89B26181E28A38
:10058000914200D262816076F6F726FC11E08B4240
:1005900002D9591A217300E027736076F6F71CFC24
:1005A00007E0521CD0B28CF80000062801D98CF864
:1005B00000703078062805D03078052802D03078D1
:1005C000042801D100203070BDE8F081C8B6FF1FBB
:1005D000208FFF1F6083FF1F70B504460D46104833
:1005E000044200D124B940F286210EA0F4F7F0FEB7
:1005F00035B1012D04D040F287210AA0F4F7E8FEBE
:10060000144813490161012D06D00168214301609E
:100610000F49491E016170BD0168A1430160F7E700
:10062000EE3A0C702E2E5C2E2E5C2E2E5C2E2E5C46
:100630002E2E5C6472697665725C7372635C6863AB
:100640003332663436305F7077632E63000000000B
:100650000100A5A50080044070B504460D460E4873
:10066000044200D124B940F2BF210CA0F4F7B0FE3F
:1006700035B1012D04D04FF4307108A0F4F7A8FE75
:100680001148012D03D041682143416070BD41688C
:10069000A143416070BD00008602F0F02E2E5C2E5A
:1006A0002E5C2E2E5C2E2E5C2E2E5C64726976657E
:1006B000725C7372635C68633332663436305F70C9
:1006C00077632E63000000000080044070B504468C
:1006D0000D460E48044200D124B94FF43C710CA0E1
:1006E000F4F776FE35B1012D04D040F2F12108A0D7
:1006F000F4F76EFE1148012D03D08168214381601B
:1007000070BD8168A143816070BD00000078F8FF72
:100710002E2E5C2E2E5C2E2E5C2E2E5C2E2E5C64DD
:1007200072697665725C7372635C686333326634D7
:1007300036305F7077632E63000000000080044055
:1007400070B504460D4641F2131034EA000000D1A2
:1007500024B940F215310BA0F4F73AFE35B1012D62
:1007600004D040F2163107A0F4F732FE1048012DF4
:1007700003D0C1682143C16070BDC168A143C1609D
:1007800070BD00002E2E5C2E2E5C2E2E5C2E2E5C5C
:100790002E2E5C6472697665725C7372635C68634A
:1007A0003332663436305F7077632E6300000000AA
:1007B0000080044010B50446002C06D0012C04D063
:1007C0004FF416710FA0F4F703FE194AB2F8FE03B6
:1007D0004AF202510843A2F8FE031649012C0CD03C
:1007E000087820F080000870B2F8FE0320F00200C4
:1007F00040F42540A2F8FE0310BD087840F08000C8
:10080000F1E700002E2E5C2E2E5C2E2E5C2E2E5C30
:100810002E2E5C6472697665725C7372635C6863C9
:100820003332663436305F7077632E630000000029
:10083000004005400A44054010B5AFF3008010BDEC
:100840001CB500200090019001208DF800000220CE
:100850008DF8050001026A460120FFF7A5FA6A46F5
:1008600010210120FFF7A0FAF4F76CFDF4F746FD24
:100870001CBD1CB500200090019001208DF80000E7
:1008800002208DF8050001026A460120FFF78CFA6C
:100890006A4610210120FFF787FAF4F75FFDF4F7AD
:1008A00039FD1CBD2DE9FC4799490A78DFF86482BF
:1008B0000024042A98F8030006D00A78052A0DD0EF
:1008C0000978062914D03CE0042803D2401C88F89B
:1008D000030001E088F803400C7032E018B1401EBC
:1008E00088F8030002E0042088F803000C7028E078
:1008F00098F8041041B1042806D000F0E9FAC820A5
:10090000F4F786FD88F8044098F80300052818D20B
:10091000DFE800F00306090C0F0000F0D9FA10E040
:1009200000F0EFFA0DE0FFF78BFF0AE0FFF7A1FF01
:1009300007E000F01DF90C2088F80100012088F87C
:1009400004001020F2F70AFB734D2888F2F70CFB25
:1009500000210846F2F7FCFA70A0F1F7ABFF002186
:100960005820F2F7F5FA6F49012091ED000AF2F7ED
:1009700037FA6DA0F1F79EFF6C4E30786C4F4FF058
:1009800010043978084208D02888CDE900040023F3
:1009900068A219469020F2F7EDFA3078397888434A
:1009A00008D02888CDE90004002363A219469020CE
:1009B000F2F7E0FA38783178884308D02888CDE912
:1009C000000400235CA219469020F2F7D3FA307895
:1009D00050B9387840B92888CDE90004002355A2E1
:1009E00019469020F2F7C6FA15210020F2F7B0FA66
:1009F0000024DFF82091514F514E09F1D009308881
:100A0000F2F7B2FA98F80300844202D13888F2F77C
:100A1000ABFA04EB840059F82000F1F74BFF0021FA
:100A20000920F1F749FA641CE4B2062CE7D3282127
:100A30000520F2F78DFA2888F2F796FA41A0F1F72F
:100A400039FF4149022091ED000AF2F7C9F93FA0B0
:100A5000F1F730FF00211120F1F72EFA3CA0F1F759
:100A600029FF3C49022091ED000AF2F7B9F937A0BD
:100A7000F1F720FF3888F2F777FA3C210020F2F7EF
:100A800067FA354C354D94ED000A10EE100AA84275
:100A90000BDA33A0F1F70EFF032094ED000AF2F712
:100AA0009FF92AA0F1F706FF0AE02DA0F1F702FF57
:100AB000022094ED000AF2F793F924A0F1F7FAFE70
:100AC00000210F20F1F7F8F93088F2F74DFA2649A6
:100AD00091ED000A10EE100AA84205DA032091ED0C
:100AE000000AF2F77DF904E0022091ED000AF2F726
:100AF00077F91EA0F1F7DEFEFF203188CDE9001066
:100B000010239F2219460020F1F708FABDE8FC8760
:100B10006083FF1FB083FF1FAC83FF1F5143322E42
:100B2000300000008483FF1FA1E600003083FF1F18
:100B3000A683FF1F3E0000003C000000A883FF1FAB
:100B4000AA83FF1F442B3A008883FF1F5600000032
:100B5000442D3A008C83FF1F3483FF1F0000204187
:100B60004E4F573A000000003C83FF1F4100000039
:100B70001CB500200090019001208DF8000002209B
:100B80008DF8050001026A460120FFF70DF96A465B
:100B900010210120FFF708F9F4F7D4FBF4F7BAFBB2
:100BA0001CBD00002DE9FC47A44E3078042809D074
:100BB00030780A2806D03078052806D030780B28FF
:100BC00003D004E000F076F901E000F065F9307838
:100BD000042802D03078052801D1002030709848D0
:100BE000DFF860921C2490ED000ADFF85C8210EEC2
:100BF000101A49450CDAB8F80010CDE900140023AA
:100C000090ED000A042219461846F2F71DFC0BE08D
:100C1000B8F80010CDE90014002390ED000A03227B
:100C200019461846F2F710FCB8F80000CDE90004A8
:100C3000002386A219465320F2F79CF98448854F79
:100C400090ED000A10EE101A49450BDA3988CDE90B
:100C50000014002390ED000A04221B211846F2F72D
:100C6000F3FB0AE03988CDE90014002390ED000A77
:100C700003221B211846F2F7E7FB3888CDE9000470
:100C8000002375A21B215320F2F774F97348744DA9
:100C900090ED000A10EE101A49450BDA2988CDE9CB
:100CA0000014002390ED000A042237211846F2F7C1
:100CB000CBFB23E090ED000A10EE101A494512DB41
:100CC00090ED000A674A10EE101A91420BDA29885B
:100CD000CDE90014002390ED000A032237211846C5
:100CE000F2F7B2FB0AE02988CDE90014002390ED69
:100CF000000A022237211846F2F7A6FB2888CDE920
:100D00000004002358A237215320F2F733F9FF20C3
:100D10003988CDE900104F23682200216720F1F7C0
:100D2000FDF810242888CDE9000400234FA20321F8
:100D30007720F2F71FF93078012846D030780A285A
:100D400043D03888CDE90004002349A217216F2041
:100D5000F2F710F93078022842D030780B283FD0D3
:100D60003888CDE90004002343A22B217020F2F73C
:100D700001F9434F3878434E3178084208D028882B
:100D8000CDE90004002340A23F216A20F2F7F2F8E7
:100D900038783178884308D02888CDE900040023CA
:100DA0003AA23F216A20F2F7E5F830783978884393
:100DB00008D02888CDE90004002334A23F216A200E
:100DC000F2F7D8F83878B0B120E0B8F80000CDE9F3
:100DD0000004002326A217216F20F2F7CBF8B9E711
:100DE000B8F80000CDE90004002323A22B217020D5
:100DF000F2F7C0F8BDE7307840B92888CDE90004A3
:100E0000002321A23F216A20F2F7B4F82888CDE917
:100E100000041F4800231A4690ED000A3F217C2061
:100E2000F2F712FB2888CDE90004002319A23F2124
:100E30008E20F2F79FF8BDE8FC8700006083FF1F5B
:100E40003483FF1F00002041A883FF1F56000000CD
:100E50003C83FF1FAA83FF1F410000004083FF1F48
:100E6000AC83FF1F0000C84257000000514333000D
:100E70002B302E32560000002D302E32560000004E
:100E80003083FF1FA683FF1F3E0000003C000000D0
:100E90008483FF1FA1E6000010B5F4F753FAF4F7BE
:100EA0002DFA0A20F4F7B4FAF4F74CFABDE8104032
:100EB000F4F730BA10B5F4F751FAF4F72BFA0A2028
:100EC000F4F7A6FAF4F73EFABDE81040F4F722BAB8
:100ED0001CB500200090019001208DF80000022038
:100EE0008DF8050001026A460120FEF75DFF6A46A3
:100EF00010210120FEF758FFF4F724FAF4F7F2F975
:100F00001CBD1CB500200090019001208DF8000050
:100F100002208DF8050001026A460120FEF744FF19
:100F20006A4610210120FEF73FFFF4F717FAF4F7A5
:100F3000E5F91CBD1CB500200090019001208DF842
:100F4000000002208DF80500C1016A460120FEF76D
:100F50002BFF6A4608210120FEF726FFF4F7F2F97D
:100F60001CBD1CB5002400940194F4F7DFF9F4F7DC
:100F7000B9F90A20F4F74CFA8DF800406A464FF4AC
:100F800080710120FEF710FF6A4608210120FEF75C
:100F90000BFF6A464FF400710120FEF705FF6A4619
:100FA00010210120FEF700FF1CBD00002DE9F05FBD
:100FB000FD480178DFF8F4830026FD4FFD4D002940
:100FC00012D00178052905D00178042902D00178D2
:100FD000062907D1297929B106702E7198F80400E5
:100FE000F9F736FE3868286298F8030001240728CC
:100FF0005CD05BD2DFE800F004111E2B37434F00BA
:101000003868296A401A43F6982188424ED92C71D3
:1010100098F80500F9F71CFE48E03868296A401A7C
:1010200047F23051884241D92C7198F80500F9F700
:101030000FFE3BE03868296A401A4EF6602188426C
:1010400034D92C7198F80500F9F702FE2EE03868C3
:10105000296A401AD849884228D92C7198F8050085
:10106000F9F7F6FD22E03868296A401AD349884228
:101070001CD92C7198F80500F9F7EAFD16E03868DC
:10108000296A401ACE49884210D92C7198F8050077
:10109000F9F7DEFD0AE03868296A401AC949884232
:1010A00004D92C7198F80500F9F7D2FDDFF8188300
:1010B000DFF81893DFF818A398ED000A10EE100A75
:1010C000B0F1804F39DA3868B0F57A7F35D999F8C0
:1010D0000E0020B172B6F4F76DFC62B623E09AF808
:1010E0000000152804D09AF800000D280ED01AE050
:1010F00072B6F4F7DFFC62B699F80E00032812D13D
:1011000089F80E4015208AF800000CE072B6F4F75A
:10111000D1FC99F80E00032804D189F80E400D2067
:101120008AF8000062B6DFF8AC9299F8000090B13E
:10113000FFF717FF89F800600DE098ED000AA64957
:1011400010EE100A884206DB99F80E0018B972B644
:10115000F4F776FC62B63868A96E401AC8287DD3C9
:10116000EFF7F6FF08F034FD9AF80000DFED9B1A68
:10117000DFF86C92032804D09AF800000F2855D0AD
:10118000A6E0002200219748007820B11E2300200D
:10119000DFF854B20CE095480078401CC3B2F6E783
:1011A0003BF810C08C4500D961466244401CC0B277
:1011B0009842F5D38E48DFF83CC200880A2818D23E
:1011C000B2FBF3F000EE100AB8EE400ADFED8A0A37
:1011D00060EE200A00EE101AB8EE400A9FED871A62
:1011E00040EE010ABCEEE00A10EE100AACF8000076
:1011F00017E0B2FBF3F000EE100AB8EE400ADFEDA4
:10120000800A60EE200A00EE101AB8EE400A9FED48
:101210007D1A40EE010ABCEEE00A10EE100AACF8AE
:101220000000794879490088088051E0784890EDBD
:10123000000A7848D0ED000A9FED771A7748B4EE9F
:10124000E00A7749F1EE10FA22DD30EE600AC0EED6
:10125000010A90ED000A60EE800A00E0ABE199ED32
:10126000001AA87980EE810A01EB800120EE210AA4
:1012700081ED000A062802D2401CA87128E0012254
:101280000721674802F0B4F885ED180AAE711FE037
:1012900030EEC00AC0EE010A90ED000A99ED001A86
:1012A000A87901EB800160EE800A80EE810A20EED1
:1012B000210A81ED000A062802D2401CA87107E02D
:1012C00003220721564802F093F885ED180AAE7103
:1012D00098ED000A288960EE210A00EE100AB8EEA7
:1012E000400AF4EEC00AF1EE10FA08DD98ED000AAB
:1012F00020EE210ABCEEC00A10EE100A288199EDFA
:10130000000A688960EE210A00EE100AB8EE400A71
:10131000F4EEC00AF1EE10FA08DD99ED000A20EEB5
:10132000210ABCEEC00A10EE100A6881A889401C90
:1013300080B2A8813A49EB891C3101F5A07298422C
:1013400017D198ED000AE87920EE210ABCEEC00A18
:1013500010EE10CA21F810C099ED000A20EE210A03
:10136000BCEEC00A10EE10CA22F810C0401CE87192
:10137000AE81E879A02813D15020E8714FF6FF70B4
:1013800000EA4300E881002031F8203021F81030D5
:1013900032F8203022F81030401CC0B25028F3D36D
:1013A000DFF880B0204E48E06083FF1FF862022023
:1013B0007C83FF1FB48EFF1FC0D40100E0930400A4
:1013C000C027090040771B003483FF1FC8B6FF1FEA
:1013D000B183FF1FB283FF1F0000404000007A442A
:1013E0003C83FF1FB883FF1FD03A0220B783FF1F43
:1013F000D683FF1FDA83FF1F9A99193FCDCCCC3ECD
:101400003333333F9A99993EDC83FF1FDE83FF1FFE
:101410009083FF1F9483FF1F00F07F458083FF1F91
:101420005C600220D483FF1FD383FF1F1E208AF835
:101430000000F9F749F901F003FB9BF8000031784F
:101440000843F3D09BF8000058B93868E96A401A9D
:101450005A49884205D9307818B100F0B3F8386895
:10146000E8629BF8000058B9386840F6B831884205
:1014700006D9307820B1687910B900F0A3F86C7102
:10148000A869B0F5FA6F7DD998ED000AD5ED0C0A80
:10149000B4EEE00AF1EE10FA04DD98ED000A85EDF5
:1014A0000C0A0CE098ED000AD5ED120AB4EEE00A41
:1014B000F1EE10FA03D298ED000A85ED120A99EDCB
:1014C000000AD5ED0D0AB4EEE00AF1EE10FA04DDE3
:1014D00099ED000A85ED0D0A0CE099ED000AD5EDB5
:1014E000130AB4EEE00AF1EE10FA03D299ED000A05
:1014F00085ED130A324AD5ED0E0A92ED000AB4EEDC
:10150000E00AF1EE10FA04DD92ED000A85ED0E0A14
:101510000CE092ED000AD5ED140AB4EEE00AF1EE0B
:1015200010FA03D292ED000A85ED140A696E98ED67
:10153000001A411A00EE101AF8EE400A95ED150A4D
:1015400001EE200A85ED150A00EE901AD9ED001A79
:10155000B8EE601AD5ED160A41EE810AC5ED160AFD
:1015600001EE101A92ED002AF8EE411A95ED171AC5
:1015700002EE211A85ED171A6866A0F5FA6001EEF1
:10158000900A00E015E0F8EE611A80EE212A85ED60
:101590000F2A00EE100AB8EE400AC0EE801AC5ED20
:1015A000101A00EE100AB8EE400AC1EE000AC5EDAE
:1015B000110A3868A866BDE8F09F000080CBA4003F
:1015C0004083FF1FF8B547480090474C47480099B3
:1015D000084483E0217800297FD023781A46082523
:1015E00002E05B086D1EEDB2DE07FAD0F82A22D0C9
:1015F00008DC802A27D0C02A23D0E02A1FD0F02A76
:1016000006D11AE0FC2A14D0FE2A10D0FF2A0CD0F2
:101610000022364B009E083333449C421DD31846AB
:10162000231A12D0012B4ED112E0FE22F1E7FC2248
:10163000EFE7F822EDE7F022EBE7E022E9E7C0224E
:10164000E7E78022E5E70022E3E7294911433AE092
:101650006FF47F4141EA022135E0244B009E1B1DBF
:101660003344FF264FF6FF776FF07F4C9C4214D334
:101670001846231A06D0012B06D0022B07D0032BC5
:1016800021D107E011461EE046EA02211BE007EBEC
:10169000024118E04CEA026115E0844213D3231A98
:1016A00006D0012B06D0022B08D0032B0BD108E06B
:1016B000114608E046EA022105E00EE007EB024190
:1016C00001E04CEA0261F6F749FB00980949201A4B
:1016D000C01C05EBC0000870F8BD641E8442BFF456
:1016E00079AFF8BD53AE0043190C0003BD5DFFBFD9
:1016F0000000FFFFD383FF1F2DE9F04F2DED048B7A
:1017000083B0002440F6FF750026A1469FEDF88ABD
:10171000F8490878DFF8E0B3A246062805D00A7831
:101720005846042AC08C09D044E09BF8090080F098
:1017300001008BF8090081F800A07EE04FF4A07250
:10174000904237D2082816D04FF6FF7303EA4000C4
:10175000ABF8260001208BF8090081F800A0BBF847
:101760002600082869D950281CD008DC14280ED07F
:10177000282862D112E01420ABF82600EAE7A0285E
:1017800014D0904259D1E32001F01CF855E001201B
:10179000F0F7B6F9112001F015F84EE00220F0F74D
:1017A000AFF94AE02F2001F00DF846E06B2001F080
:1017B00009F842E00A78052A3FD101283DD91428CA
:1017C00015D04008ABF8260001208BF8090081F8FD
:1017D00000A0BBF8260004282FD9502822D00ADC0C
:1017E00008280ED0142813D0282826D117E0082066
:1017F000ABF82600E8E7A02818D0B0F5A07F1CD1F0
:1018000018E00020F0F77CF90B2000F0DBFF14E07B
:101810000120F0F775F9112000F0D4FF0DE002204F
:10182000F0F76EF92F2000F0CDFF06E06B2000F0FE
:10183000C9FF02E0E32000F0C5FF4FF0500848F672
:101840001047CDE900780A22462300211046F0F720
:1018500065FBCDE900781422462300211046F0F7FD
:101860005DFBCDE900781E22462300211046F0F7EB
:1018700055FBCDE900782822462300211046F0F7D9
:101880004DFBCDE900783222462300211046F0F7C7
:1018900045FBCDE900783C22462300211046F0F7B5
:1018A0003DFB4623CDE900781A4600211846F0F7A3
:1018B00035FBCDE900785022462300211046F0F791
:1018C0002DFBCDE900785A22462300211046F0F77F
:1018D00025FBCDE900786422462300211046F0F76D
:1018E0001DFBCDE900780A236E2219460020F0F78F
:1018F00015FBCDE9007814236E2219460020F0F77D
:101900000DFBCDE900781E236E2219460020F0F76A
:1019100005FBCDE9007828236E2219460020F0F758
:10192000FDFACDE9007832236E2219460020F0F747
:10193000F5FACDE900783C236E2219460020F0F735
:10194000EDFA4FF0FF08CDE900786D224623002123
:101950001046F0F7E3FACDE900786E224623002125
:101960001046F0F7DBFA0022CDE900784623114655
:101970001046F0F7D3FACDE9007801224623002182
:101980001046F0F7CBFA0023CDE900786E22194615
:101990001846F0F7C3FACDE9007801236E22194604
:1019A0000020F0F7BBFACDE9007845236E221946F6
:1019B0000020F0F7B3FACDE9007846236E221946ED
:1019C0000020F0F7ABFA00214C4F4FF4A06237F83B
:1019D0001100A04201D9044602E0A84200D2054607
:1019E0008144491C89B29142F1D3B9FBF2F03988A4
:1019F0004FF4806281421CD2002137F811308342BB
:101A000013D201F1080337F8133083420DD201F1EC
:101A1000100337F81330834207D201F1180337F867
:101A20001330834201D2CEB203E0491C89B2914205
:101A3000E3D3314619E037F81130834213D901F16D
:101A4000080337F8133083420DD901F1100337F83A
:101A50001330834207D901F1180337F8133083425A
:101A600001D9CEB203E0491C89B29142E3D39BF87D
:101A70000900DFF88C9070B38BED118A601B4FF476
:101A80007A71484340F6FF7190FBF1F000EE100AC6
:101A90001C48B8EEC00AD0ED000A1B4860EE200AD0
:101AA00090ED001A80EE810AF6EE000A30EE200A70
:101AB000BCEEC00A10EE100A81B2ABF828109BF8F9
:101AC000050000EB80138B4206D28BF806A0401C69
:101AD0008BF805001CE09EE0401EC0EB0010B1EB4F
:101AE000800F13DA9BF80600401C8BF806000FE00D
:101AF000000000006083FF1FB083FF1FD0CC0120D7
:101B00000C5B02208083FF1F9883FF1F8BF806A0C9
:101B10009BF80600322806D19BF80500401E8BF882
:101B200005008BF806A00020F94B37F8101000EEE6
:101B3000101A03EBC001B8EE400A81ED000A81EDF6
:101B4000018A401C80B29042EFD301230022F04969
:101B5000F04805F064F84FF4AA742246EE49EC48C8
:101B600005F0F6FB0120594609EB8002D1ED110A80
:101B700092ED000AB4EEE00AF1EE10FA02DD88857B
:101B800081ED110A401C80B2A042EDD3C88C5028D0
:101B900028D004DC142817D0282805D11BE0A02861
:101BA00027D0B0F5A07F2AD0888DDC4A5043000CA6
:101BB0008885D74BC8793C3B0A8D23F810201D2817
:101BC00025D2401CC87126E0888D4FF4FA3250436C
:101BD000000C8885EDE7888D4FF47A725043800AB7
:101BE0008885E6E7888D4FF4FA725043800A88852D
:101BF000DFE7888DFA225043800A8885D9E7888DEF
